:100000000C94FC060C9440070C9440070C94400799
:100010000C9440070C9440070C9440070C94400744
:100020000C9440070C9498180C9440070C944007CB
:100030000C94A12E0C9440070C9440070C9440079C
:100040000C9440070C9440070C9425170C9440071F
:100050000C948A0E0C9440070C94510E0C9440079B
:100060000C94DB1D0C9440070C94382D0C94400725
:100070000C946F750C9440070C946470F91127115F
:1000800027112711271127112711271127112711B0
:1000900027112711271127112711271127112711A0
:1000A0002711271127112711ED11AA110711C111CD
:1000B00027112711BD11D8112711271127117211EE
:1000C0002711271127112711271127112711841113
:1000D000271180114912F810F810F810F810F810D4
:1000E000F810F810F810F810F810F810F810F810D0
:1000F000F810F810F810F810F810F810F810F810C0
:10010000F810F810F810F810F8101612F810F8108F
:10011000F810F810F810F81040116111F8100913D8
:100120000D13F810E312CC12F810F810F810F810B4
:100130006612851E781E6C1E521E381E141E261E48
:100140008921BD20BA20141EA7208D206D204D20AE
:10015000FB1FA91F911E0723BF284C28E3292E2926
:100160002226B8254725FA24A8244924E9238923EF
:10017000EA274C27502AE226B12DA02DFB2DD92DA0
:10018000C92D5A2D6F2D6F2D762D922D8D2D722DFF
:100190007A2D762D892D962D722D7A2D762D852D01
:1001A0009B2D722D0D2E0A0D426174743A0020337E
:1001B0002043656C6C7320200020342043656C6CF8
:1001C00073202000204C6F77207761726E696E6714
:1001D000206C6576656C3A2025642E2564000A0D36
:1001E00047656E65726174696E67206465666175E6
:1001F0006C74204D69786572205461626C65000AE8
:100200000D4D697865722D436F6E6669673A2027D8
:1002100025732720282575204D6F746F7273290070
:100220000A0D466F756E6420424C2D4374726C3A11
:100230002000256420000A0D0A0D2121204D49537C
:1002400053494E4720424C2D4354524C3A2025648A
:10025000202121000A0D3D3D3D3D3D3D3D3D3D3DC3
:100260003D3D3D3D3D3D3D3D3D3D3D3D3D3D3D3DBE
:100270003D3D3D3D3D3D3D3D3D000A0D496E6974AE
:100280002E20454550524F4D003A2047656E65720D
:100290006174696E672044656661756C742D506188
:1002A00072616D65746572207573696E67206F6C1D
:1002B0006420537469636B2053657474696E67734B
:1002C000000A0D466C696768742D74696D65202598
:1002D00075206D696E2020546F74616C3A2575200D
:1002E0006D696E000A0D414343206E6F7420636197
:1002F0006C696272617465642021000A0D5573692E
:100300006E6720706172616D6574657273657420CB
:100310002564000A0D43616C6962726174696E67DD
:100320002070726573737572652073656E736F727A
:100330002E2E004F4B0A0D000A0D436F6E74726F24
:100340006C3A200048656164696E67486F6C6400B0
:100350004E6F726D616C20284143432D4D6F646573
:1003600029000A0D3D3D3D3D3D3D3D3D3D3D3D3D71
:100370003D3D3D3D3D3D3D3D3D3D3D3D3D3D3D3DAD
:100380003D3D3D3D3D3D3D0A0D00416E676C654E76
:1003900069636B20202020202020416E676C65520D
:1003A0006F6C6C202020202020204163634E696305
:1003B0006B202020202020202020416363526F6C7E
:1003C0006C2020202020202020205961774779723E
:1003D0006F20202020202020202048656967687435
:1003E0002056616C7565202020204163635A2020CF
:1003F0002020202020202020202047617320202042
:1004000020202020202020202020436F6D70617349
:10041000732056616C7565202020566F6C7461677F
:1004200065205B302E31565D20205265636569760C
:100430006572204C6576656C20204779726F204389
:100440006F6D70617373202020204D6F746F722068
:10045000312020202020202020204D6F746F72201A
:10046000322020202020202020204D6F746F722009
:10047000332020202020202020204D6F746F7220F8
:100480003420202020202020202020202020202058
:10049000202020202020202020202020202020205C
:1004A00020202020202020202020566172696F4DBE
:1004B000657465722020202020204D4B334D6167EC
:1004C0002043616C537461746520536572766F20AC
:1004D00020202020202020202020486F7665726771
:1004E0006173202020202020202043757272656EC9
:1004F00074205B302E31415D20204361706163695F
:100500007479205B6D41685D202020202020202010
:1005100020202020202020202020202020202020DB
:1005200020202020202020202020202020202020CB
:1005300020202020202020202020202020202020BB
:10054000202020202020202020204932432D4572C9
:10055000726F7220202020202020202020202020A8
:10056000202020202020202020204750535F4E694B
:10057000636B20202020202020204750535F526FA3
:100580006C6C202020202020202021212120494E79
:10059000434F4D50415449424C4520212121002ECA
:1005A000000A0D20444143206F7220493243204508
:1005B00052524F522120436865636B204932432CCD
:1005C0002033567265662C2044414320616E6420BE
:1005D000424C2D4374726C005B25695D005B25699C
:1005E0005D002B204D696B726F4B6F7074657220CC
:1005F0002B0048573A5625642E25642053573A2538
:10060000642E256425630053657474696E673A250A
:100610006420257300493243204552524F52212114
:1006200021004D697373696E6720424C2D437472CB
:100630006C3A25642121004865696768743A202076
:1006400025356900536574706F696E743A25356994
:100650000050726573737572653A253569004F668F
:10066000667365743A2020253569004865696768B6
:100670007420636F6E74726F6C0044495341424C36
:1006800045440048656967687420636F6E74726FD3
:100690006C0044495341424C4544006163742E2030
:1006A00062656172696E67004E69636B3A20202053
:1006B00020202025356900526F6C6C3A20202020C4
:1006C000202025356900436F6D706173733A2020D7
:1006D00020253569004B313A25346920204B323AC8
:1006E00025346920004B333A25346920204B343AB5
:1006F00025346920004B353A25346920204B363AA1
:1007000025346920004B373A25346920204B383A8C
:1007100025346920004E693A2534692020526F3A09
:10072000253469200047733A253469202047693A07
:10073000253469200050313A253469202050323A5E
:10074000253469200050333A253469202050343A4A
:1007500025346920004779726F202D2053656E7310
:100760006F72004E69636B25346920282533692E2A
:1007700025692900526F6C6C25346920282533695E
:100780002E2569290047696572253469202825339B
:100790006929004E69636B20253469202825336957
:1007A0002E25782900526F6C6C202534692028256D
:1007B00033692E2578290059617720202534692056
:1007C0002825336929004E69636B20253469202868
:1007D00025336929282533692900526F6C6C20253F
:1007E000346920282533692928253369290059616E
:1007F0007720202534692028253369292825336965
:100800002900414343202D2053656E736F72004EC3
:1008100069636B2025346920282533692900526FCC
:100820006C6C20253469202825336929005A202042
:10083000202025346920282533692900566F6C74DF
:100840006167653A2020202533692E2531695600DD
:1008500043757272656E743A2020202533692E2507
:1008600031694100506F7765723A202020202025A1
:10087000346957004469736368617267653A20257B
:1008800035696D416800526563656976657200522D
:10089000432D525353493A202020202534690052D9
:1008A000432D5175616C6974793A20253469005281
:1008B000432D4368616E6E656C733A25346900435D
:1008C0006F6D706173730048656164696E673A208B
:1008D000202535690056616C75653A202020202559
:1008E00035690053746172743A20202020253569DF
:1008F00000506F7469313A202025336900506F74BD
:1009000069323A202025336900506F7469333A20E8
:100910002025336900506F7469343A2020253369EB
:1009200000506F7469353A202025336900506F7488
:1009300069363A202025336900506F7469373A20B0
:100940002025336900506F7469383A2020253369B7
:1009500000536572766F202000536574706F696E66
:1009600074202025336900506F736974696F6E3A83
:10097000202533690052616E67653A2533692D255C
:1009800033690045787465726E436F6E74726F6C74
:100990002020004E693A2534692020526F3A2534D0
:1009A00069200047733A253469202047693A253485
:1009B00069200048693A253469202043663A253485
:1009C000692000424C2D4374726C204572726F7224
:1009D00073200025336420253364202533642025CB
:1009E00033642000253364202533642025336420BC
:1009F00025336420002533642025336420253364A7
:100A0000202533642000424C2D4374726C20666FA5
:100A1000756E64200020256320202025632020207F
:100A20002563202020256320002025632020202509
:100A300063202020256320202025632000202563BB
:100A40002020202D2020202D2020202D200031307E
:100A500000313100313200466C696768742D546989
:100A60006D65202000546F74616C3A2535756D6991
:100A70006E004163743A20202535756D696E00283B
:100A8000726573657429000A0D506C656173652089
:100A9000636F6E6E656374205370656B7472756DF1
:100AA00020726563656976657220666F722062697F
:100AB0006E64696E67204E4F572E2E2E006F6B2E80
:100AC0000A0D0054696D656F75742E0A0D000000E3
:100AD0008F001E01AD013B02CA025803E6037404F5
:100AE00002058F051B06A7063307BE074808D20874
:100AF0005B09E3096B0AF20A780BFD0B810C040D0C
:100B0000860D070E870E060F840F00107B10F51060
:100B10006E11E5115B12CF124213B313231492141A
:100B2000FE146A15D3153B16A11605176717C817CB
:100B300027188318DE1837198E19E319361A871A01
:100B4000D61A231B6E1BB61BFD1B411C831CC31C2A
:100B5000001D3C1D751DAB1DE01D121E421E6F1EAB
:100B60009A1EC31EE91E0D1F2E1F4D1F691F841FD5
:100B70009B1FB01FC31FD31FE11FEC1FF51FFB1FDF
:100B8000FF1F002003010000FD6900020101C46A8B
:100B900001030202356B02000303926B2532692EBA
:100BA0002531695600253033646D202530336425A6
:100BB00063005374617475730025346920253269AC
:100BC0003A25303269002534696D2563004E69632A
:100BD0006B20526F6C6C202059617700253469209E
:100BE00025346920253469002532692E253169565E
:100BF00020202533692E253169410025346957208D
:100C00002536696D4168005361743A2530326400BD
:100C10004E6F46697800324446697800334446692D
:100C200078003F3F466978002F4447505300486F93
:100C30006D653A253033646D2025303364256300BB
:100C40004E6F204E6176694374726C21000A0D77F5
:100C500077772E4D696B726F4B6F707465722E646F
:100C6000652028632920486953797374656D732062
:100C7000476D6248000A0D74686520757365206FC2
:100C800066207468697320736F667477617265207B
:100C90006973206F6E6C79207065726D697474650C
:100CA00064200A0D6F6E206F726967696E616C2037
:100CB0004D696B726F4B6F707465722D4861726411
:100CC00077617265004143542044534C004A657477
:100CD0006920736174656C6C6974005370656B7422
:100CE00072756D20736174656C6C697420284C6F2B
:100CF00077207265736F6C7574696F6E290053701D
:100D0000656B7472756D20736174656C6C697420A9
:100D1000283230343829005370656B7472756D2039
:100D2000736174656C6C6974004D756C746973697A
:100D3000676E616C2050504D000A0D526563656905
:100D40007665723A2000756E6B6E6F776E2E205549
:100D500073696E672050504D2E2E2E006E6F7420DA
:100D6000737570706F727465642062792068617247
:100D7000647761726521000A0D3D3D3D3D3D3D3D7D
:100D80003D3D3D3D3D3D3D3D3D3D3D3D3D3D3D3D93
:100D90003D3D3D3D3D3D3D3D3D3D3D3D000A0D461A
:100DA0006C69676874436F6E74726F6C0A0D48618A
:100DB0007264776172653A25642E25640A0D536F5B
:100DC0006674776172653A5625642E256425632022
:100DD000000A0D3D3D3D3D3D3D3D3D3D3D3D3D3DE3
:100DE0003D3D3D3D3D3D3D3D3D3D3D3D3D3D3D3D33
:100DF0003D3D3D3D3D3D000011241FBECFEFD0E104
:100E0000DEBFCDBF11E0A0E0B1E0ECE0FFEE02C03C
:100E100005900D92A43DB107D9F718E0A4EDB1E01B
:100E200001C01D92A833B107E1F76AEAE2E0F0E001
:100E300081E2809357007491AE014F5F5F4F20EFC6
:100E40003FEFDA019FE0F9012F5F3F4F84918D93CF
:100E5000915097FFF8CF773911F40000FECFFA01D7
:100E60009EE0819168276095915097FFFACF88891D
:100E7000681721F0773911F40000FECF0C94810837
:100E80000C940000282FFB018150853008F023E0EE
:100E9000842F9927332721503040829FD001839F90
:100EA000B00D929FB00D1124AC59BF4F019724F0A3
:100EB0000E9468770192FACF0E94226608958630D8
:100EC00038F085E0A2E0B0E0082E0E947577089522
:100ED0008823C1F70895582F863048F155E0842FB4
:100EE0009927252F332721503040829FD001839F9F
:100EF000B00D929FB00D1124AC59BF4FFB0101976B
:100F000024F001900E947577FACFA2E6B0E0042E9B
:100F10000E947577A0E5B0E08CE0FB01182E0E94DE
:100F20008177852F0E945F070E942266089588239B
:100F3000B1F60895CF93A2E0B0E00E946877802DCB
:100F4000C82F8150853020F0C3E08C2F0E945F07AE
:100F50008C2F9927CF9108958091C806E82FFF27FD
:100F6000EE0FFF1FE75AF94F808191818D5E9F4FF1
:100F700014F010920301808191818A5B9F4F24F4C9
:100F800080910301882319F02091850417C081E026
:100F90008093030120918504280F20938504253038
:100FA00038F088EE93E0909303028093020206C02B
:100FB00066E970E0822F0E94CB33E6CF822F99271B
:100FC0009093FF058093FE0508951F93CF93DF93C1
:100FD000182F882351F48091EA068233D8F0809349
:100FE0000001112309F489C046C086EA91E09F936D
:100FF0008F9381E294E19F938F93E0910404F091A9
:10100000050409950F900F900F900F908091EA06BC
:10101000823328F784EF91E00E941618EC01112327
:1010200009F04BC0809125019091260182389105ED
:101030000CF04FC08091EA0623E0829FC00111248A
:1010400080930001112369F268EC70E0822F0E9406
:10105000CB338EEA91E09F938F9381E294E19F934B
:101060008F93E0910404F091050409950F900F907F
:101070000F900F90B6CF809100016AE00E94BB767E
:10108000892F99279F938F93809100010E94BB76AF
:1010900099279F938F9384EC91E09F938F9381E2A4
:1010A00094E19F938F93E0910404F09105040995D6
:1010B0008DB79EB708968DBF20C0CE010E941F1825
:1010C000882309F0AFCFCE010E941F188823A9F30F
:1010D000A9CF8091EA069927880F991F880F991F39
:1010E00080930001112309F47CCF68EC70E084E068
:1010F0000E94CB3389EB91E0AECFDF91CF911F916E
:101100000895CFEFD0E1DEBFCDBFCC24DD24FF2496
:10111000F4B8F5B807EE13E00253104017FFFCCF08
:10112000189B77C1199B9EC12DE02093020181E895
:1011300087B93E9A8FEF88B98BE184B981E085B990
:101140008EE38AB987E48BB9469A84B7877F84BFD8
:10115000809160008861809360001092600080ED53
:1011600097E090930302809302021092EE02109295
:10117000ED0210925E0610925D061092F00210923F
:10118000EF021092F2021092F102243108F447C1EA
:1011900088E894E0A0E0B0E080937E0190937F0126
:1011A000A0938001B09381012A3009F45DC12431FC
:1011B00009F45AC1289A0E9481180E9452180E946C
:1011C00029140E94852E0E949D1C0E94F72C0E94CB
:1011D00002620E94966C0E94A274809102018C307F
:1011E00008F01BC1299A78944DE068EC76E083E022
:1011F0000E944207C8EED3E0DE010E946877802D8E
:10120000813009F411C18EED91E09F938F9381E2BB
:1012100094E19F938F93E0910404F0910504099564
:101220000F900F900F900F9026E034E0F9018FE0BF
:10123000158616861786108A8150349687FFF8CF58
:1012400080E4809313048093140410921504809317
:1012500016048093170490EC9093180410921904CC
:1012600080931A0480931B0410921C0490931D0415
:1012700090931E0480931F041092200480932104F5
:101280009093220481E08093060447E054E08BE0D1
:10129000E4E0F1E0DA0101900D928A95E1F78DE446
:1012A000DE01F901182E0E9481778F2D99279F93D7
:1012B0008F935F934F938FEF91E09F938F9381E292
:1012C00094E19F938F93E0910404F09105040995B4
:1012D00010924C02109206020E94EC3FADB7BEB7CE
:1012E0001896ADBF809106028823E1F310924C025C
:1012F00080E292E09F938F93E1E2F4E1FF93EF931A
:10130000E0910404F0910504099580EA9FE00E94B1
:1013100016188C01AA24BB240F900F900F900F90E9
:10132000E2E38E2EE2E09E2E109206020E94EC3F37
:10133000809106028823E1F37501EE0CFF1CEE0C90
:10134000FF1CF701EA5FFB4F85851816D4F4E7010F
:10135000C85DD94FC8010E941F18982F882389F4AF
:101360008981882374F0909306020E94EC3F80915B
:1013700006028823E1F3C8010E941F18982F8823D2
:1013800079F388E296E0E80EF91EF701818187FD86
:101390006FC0E50121965E012C9730F2AA24BB2490
:1013A00066E3862E62E0962E11E01FC0E5012196CD
:1013B000DF93CF939F928F92E1E2F4E1FF93EF935B
:1013C000E0910404F09105040995109300028DB793
:1013D0009EB706968DBFF701E85DF94F8181807851
:1013E00081835E012C9708F057C07501EE0CFF1C3D
:1013F000EE0CFF1CF701E85DF94F818187FD06C007
:10140000F701EA5FFB4F8585181684F2E501219606
:10141000E2CF199B2BC024E188CE2998E4CE8BE043
:1014200095E0A0E0B0E0B8CEA1E0B0E00E9468771F
:10143000802D8F3F09F4E7CE26E034E08DE4DE0115
:10144000F901182E0E947077F9013D969FE0808186
:10145000349618160CF4F394915097FFF8CF47E0A8
:1014600054E023CF2BE061CE2898A5CE2AE05DCEB4
:10147000E5012196DF93CF939F928F9281E294E1D1
:101480009F938F93E0910404F09105040995ADB703
:10149000BEB71696ADBF7FCF84E592E09F938F9342
:1014A000A1E2B4E1BF93AF93E0910404F09105048D
:1014B00009950E94EC3F0F900F900F900F90A1E0C4
:1014C000B0E00E946877802D823509F0CFC2AEE08F
:1014D000EA2EA0E0FA2ED7010E946877802D992786
:1014E000582F442737010894611C711CD3010E94B6
:1014F0006877802D480F511DECEFAE2EEFEFBE2E1A
:10150000AE0CBF1CD5010E946877802D9927382F1B
:1015100022276DEF862E6FEF962E8E0C9F1CD40126
:101520000E946877802D280F311D8FEF2F3F3807DD
:1015300009F4AEC39FEF4F3F590709F4A9C3309395
:10154000D7012093D6015093D9014093D8018091BF
:10155000D6019091D7019F938F938091D80190915C
:10156000D9019F938F9381EC92E09F938F93C1E277
:10157000D4E1DF93CF93E0910404F0910504099541
:10158000ADB7BEB71896ADBFA4E0B0E00E946877D3
:10159000802D853008F06CC30E949A074CE668ECF9
:1015A00076E00E9442070E949A0799279F938F93A3
:1015B0008BEF92E09F938F93DF93CF93E09104049E
:1015C000F091050409958DB79EB706968DBF83E10E
:1015D00093E09F938F93DF93CF93E0910404F09176
:1015E0000504099588EE93E00E9416188C010E946C
:1015F000A31C0F900F900F900F90C8010E941F180E
:101600008823D9F383E393E09F938F93A1E2B4E11E
:10161000BF93AF93E0910404F091050409950E94F3
:101620007E3D809102010F900F900F900F908A30B5
:1016300009F41CC3843109F419C3289A80ED97E09A
:10164000909303028093020285E58093870488E3E8
:1016500093E09F938F93E1E2F4E1FF93EF93E091A6
:101660000404F091050409958091D4060F900F9021
:101670000F900F9082FFF7C284E493E09F938F93C3
:1016800081E294E19F938F93E0910404F09105042B
:1016900009950F900F900F900F900E946C2288E890
:1016A00093E19093A5018093A40181E08093860447
:1016B0000E94E5070E94017482E693E09F938F9356
:1016C000A1E2B4E1BF93AF93E0910404F09105046B
:1016D000099580ED97E00E9416188C018AEF90E042
:1016E0000E941618EC010F900F900F900F90CE01F2
:1016F0000E941F18882309F0B5C080910602882334
:1017000009F4A3C080911701882309F49EC01092A8
:10171000060280918504882309F4B2C00E94AC07B8
:101720000E94EC3F209102012A3009F4B2C024311A
:1017300009F4AFC0289A8091F402882309F49AC072
:101740008091F40281508093F4028091A4019091E1
:10175000A50101979093A5018093A4018091A40114
:101760009091A501892B29F080914B02882309F4DF
:1017700092C08091A4019091A501892B09F42BC1FD
:1017800080911001909111018F5F9F4F09F441C129
:1017900080910602882321F08091EA02882311F4C7
:1017A0000E946D140E94E710C8010E941F18882330
:1017B00009F447C00C5E1F4F80910D01882309F486
:1017C000E2C0815080930D018091D903882309F4F0
:1017D000BAC081508093D9038091C3028F7B8093DC
:1017E000C30280910001282F332780912501909119
:1017F0002601821793070CF0B9C08091C302806262
:101800008093C30280911001909111018F5F9F4FCF
:1018100009F413C10E94496584E08093010280911C
:10182000EA02882309F04BC05AEAC52E55E0D52EAE
:101830000894C11CD11C22E7C2162BE0D20609F481
:101840004FC00E9431660E94AB6C809101028823D8
:1018500009F04DCF0E948D65CE010E941F1888238C
:1018600009F44BCF84E690E00E941618EC010E9428
:101870005E7543CF80916F00806280936F0065CF6B
:101880000E946B420E94EC3F209102012A3009F035
:101890004ECF289850CF2A3009F4CDC0243109F416
:1018A000CAC0289A8091020290910302892B09F004
:1018B0006FCF8091C3028F778093C30269CF8091ED
:1018C000DA018F5F813309F4C5C08093DA0108948F
:1018D000C11CD11C22E7C2162BE0D20609F0B1CF01
:1018E000CC24DD242091D8013091D9012F5F3F4FC6
:1018F0003093D9012093D8018091D6019091D701DE
:1019000001969093D7018093D601832F9927D70111
:10191000082E0E9475778091D801D301082E0E946D
:1019200075778091D701D501082E0E947577809137
:10193000D601D401082E0E94757784E190E00E94C0
:1019400016188C017ECF1092D7031092D6031092F6
:10195000D5031092D4038091020290910302892B47
:1019600009F03FCF8091C302806439CF8091020299
:1019700090910302892B09F04DCF8091C3028F7D96
:101980008093C30247CF809391041092CF021092AC
:10199000CE021092CD021092CC021092CB02109285
:1019A000CA0280911001909111018F5F9F4F09F041
:1019B0000BCF8091F402882309F006CF88E99AE3DF
:1019C000909303028093020280E09CE090931101C7
:1019D00080931001F9CE0E940D2D85E090E0909348
:1019E000A5018093A40180911006909111060196A3
:1019F00090931106809310068091C30280688093B3
:101A0000C30280911001909111018F5F9F4F09F0E7
:101A1000BFCE8091EA02882309F4BACE80E197E232
:101A2000909303028093020280E890E0909311016A
:101A300080931001ADCE289835CF80E797E1909341
:101A400003028093020280E093E09093110180935F
:101A50001001E0CE1092DA018091D4019091D5016D
:101A600001969093D5018093D401E2CE0E943D313E
:101A70008AE792E09F938F93E1E2F4E1FF93EF9383
:101A8000E0910404F0910504099541E0742E0F9053
:101A90000F900F900F90C0E5D0E08E010F5F1F4FA9
:101AA00032E0E32EF12CEC0EFD1E23E0A22EB12C31
:101AB000AC0EBD1E94E0492E512C4C0E5D1E85E0EF
:101AC000282E312C2C0E3D1EB8E08B2E912C8C0E26
:101AD0009D1EF2E07F1609F4B5C023E0721609F4EA
:101AE000BFC083E0871508F4ADC080910201843146
:101AF00068F085E08093E706109208078BE18093F9
:101B0000E3068EE48093050780930607DE010E94BA
:101B10006877802D8C3008F092C0D8010E946877D9
:101B2000802D8C3008F08BC0D7010E946877802D03
:101B30008C3008F084C0D5010E946877802D8C30ED
:101B400008F07DC0DE010E946877802D8093C80672
:101B5000D8010E946877802D8093C906D7010E9422
:101B60006877802D8093CA06D5010E946877802D02
:101B70008093CB06D2010E946877802D8093CC069B
:101B8000D1010E946877802D8093CD06A6E5B0E054
:101B90000E946877802D8093CE06A7E5B0E00E9472
:101BA0006877802D8093CF06D4010E946877802DBE
:101BB0008F3F09F44AC0D4010E946877802D80933A
:101BC000D006A9E5B0E00E946877802D8093D10609
:101BD000AAE5B0E00E946877802D8093D206ABE53D
:101BE000B0E00E946877802D8093D30691E079164B
:101BF00089F4A9E8B2E0BF93AF93E1E2F4E1FF9387
:101C0000EF93E0910404F091050409950F900F9073
:101C10000F900F904CE668EC76E0872D0E946B07E2
:101C20007394F5E0F71508F054CF83E00E945F0746
:101C300082E5A1E0B0E0082E0E94757748CC0E94B2
:101C40001831E8CF0E94113250CF89E08093D0063E
:101C50008AE08093D1068BE08093D2068CE0C4CFDB
:101C60000E94E33242CF80E593E008CD2898E6CC8D
:101C700084EE92E09F938F93DF93CF93E0910404DF
:101C8000F091050409950F900F900F900F9084CC60
:101C90001092D9011092D8011092D7011092D6015A
:101CA00056CC1F920F920FB60F9211248F939F93D1
:101CB000EF93FF9380910F018823A9F48091F401A1
:101CC0009091F5010196FC01EA5CFA4FE081ED305C
:101CD00079F0803A910561F09093F5018093F401D9
:101CE000E093C6000EC01092F5011092F40109C0F5
:101CF0001092F5011092F40181E080930F01E093BE
:101D0000C600FF91EF919F918F910F900FBE0F90A2
:101D10001F9018951F920F920FB60F9211242F93B8
:101D20003F934F935F936F937F938F939F93AF9363
:101D3000BF93CF93EF93FF9390E08091C600809381
:101D4000EC015091FA01503A10F09093FB01809110
:101D5000EC018D3091F02091FB01822F9927813089
:101D6000910509F46EC0823091050CF490C0029781
:101D700009F481C01092FB01AAC02091FB0122301E
:101D800061F79093FB01852F99278C569B4FFC019F
:101D9000329740812091F6013091F701241B3109DF
:101DA000DC0111978C91281B3109C9019F70909318
:101DB000F7018093F6010024880F991F001C880FFB
:101DC000991F001C892F902D982F935C9093F801F8
:101DD0002F733070235C2093F9018081891709F4F7
:101DE00070C090E08091E9018F5F8093E901C0911C
:101DF000EB01CC2309F06BC0992309F468C081E0A2
:101E00008093EB01580F5093E8015150E52FFF27C5
:101E1000EC56FB4F8DE0808380919604823509F06B
:101E200056C00E946C2288E190E02CE00FB6F89436
:101E3000A895809360000FBE20936000C0930002BD
:101E400046C02F5F2093FB01E52FFF27EC56FB4F89
:101E50008091EC0180835F5F5093FA012091EC0147
:101E60008091F6019091F701820F911D9093F701F7
:101E70008093F6012CC0E52FFF27EC56FB4F809195
:101E8000EC018083503A38F31092FB01E7CF892BA5
:101E900009F070CF8091EC01833259F08091EC0110
:101EA0008093940481E08093FA018091EC0199275A
:101EB000DDCF8091EB01882389F781E08093FB01DE
:101EC000EDCF8C91821709F08CCF91E090CFFF91EC
:101ED000EF91CF91BF91AF919F918F917F916F9132
:101EE0005F914F913F912F910F900FBE0F901F90D8
:101EF0001895AC01A0E0B0E09D01A817B90748F41F
:101F0000E6E3F5E08191280F311D1196A417B5077E
:101F1000C8F33F70FD01EA5CFA4FC9010024880F45
:101F2000991F001C880F991F001C892F902D835C1E
:101F300080831196FD01EA5CFA4F2F733070822F77
:101F4000835C8083A95CBA4F8DE08C9310920F0163
:101F5000809136058093C6000895A0E0B0E0E3EBE1
:101F6000FFE00C9434772C859D857E85BB2483E22D
:101F7000809336059F59909337052093380503E0E9
:101F800010E0772309F4ADC0CF84D88843E1E42E74
:101F9000F12CEC0EFD1EA989BA897150109709F435
:101FA000A0C0109709F43CC0F601EB0DF11DB394ED
:101FB0009081119789F47723A1F1F70122E030E0B5
:101FC000E20EF31ED701C080D180E20EF31E0D9009
:101FD000BC91A02DBB247150109719F1F601EB0DA7
:101FE000F11DB3944081119709F466C01097D1F0A8
:101FF000F601EB0DF11DB39460811197A1F47723E5
:1020000091F0F7013296D701CD90DC9032E0E32ECB
:10201000F12CEE0EFF1EA081B181BB24715003C0D4
:1020200090E040E060E0F801EA5CFA4F892F869585
:102030008695835C80830F5F1F4FF801EA5CFA4F3F
:10204000892F99278370907082959295907F982719
:10205000807F982755279A01329522952F70232744
:102060003F702327822B835C80830F5F1F4FF80113
:10207000EA5CFA4F4F705070440F551F440F551FC4
:10208000862F99270024880F991F001C880F991FFD
:10209000001C892F902D842B835C80830F5F1F4F42
:1020A000F801EA5CFA4F6F73635C60830F5F1F4F48
:1020B000109709F076CF15C0772309F4B3CFF70155
:1020C000A2E0B0E0EA0EFB1ED701C080D18022E082
:1020D00030E0E20EF31E0D90BC91A02DBB24715098
:1020E00085CFC8010E94790FE9E00C945077A3E0F6
:1020F0007A2F4091E801465009F45FC0E72FFF278F
:10210000EC56FB4F80818D537F5FE72FFF27EC5606
:10211000FB4F20812D537F5FE72FFF27EC56FB4FAE
:1021200030813D537F5FE72FFF27EC56FB4F6081E7
:102130006D537F5F9927880F991F880F991F522F22
:1021400052955F70582B822F99278F7090708295CF
:102150009295907F9827807F9827232F2695269504
:10216000282B832F9927837090700024969587954C
:102170000794969587950794982F802D682B41504A
:102180004F3FD9F0EA2FFF27EC56FB4F5083AF5F4C
:1021900041504F3F91F0EA2FFF27EC56FB4F208331
:1021A000AF5F41504F3F49F0EA2FFF27EC56FB4FFE
:1021B0006083AF5F442309F0A1CF87E994E0909357
:1021C000E7018093E601A350A093E5010895A2E002
:1021D000B0E0EDEEF0E10C943B778091EB018823C9
:1021E00009F42BC30E947710809195048236C1F1C7
:1021F000809196049927AA27BB27FC01EB54F04055
:10220000EC32F10520F5E25CFF4F0C94627780918F
:10221000DF019091E001892B09F099C2A091E601BC
:10222000B091E7019C91992309F087C29C918AE0C3
:10223000989FC00111249093E0018093DF0180EA10
:102240009FE00E9416189093DC018093DB011092AE
:10225000EB011092E7011092E6011092E501EDC248
:10226000809196049927AA27BB27FC01EB54F040E4
:10227000EF32F10508F0BCCFE659FF4F0C946277BE
:1022800080910F018823E1F3A091E601B091E7016D
:102290009C91913009F4B4C2198281E090E09F933F
:1022A0008F93CE0101969F938F9381E08F938F93AD
:1022B0008DE48F930E94AD0F8DB79EB707968DBFAB
:1022C00097CF80910F018823E1F38DE490E09F93F5
:1022D0008F9386E094E09F938F9381E08F938F9309
:1022E0008EE4E7CF8FEF80930D01E091E601F0914E
:1022F000E70180818093470281E08093F201A7CFBC
:1023000081E08093EF01A3CF8091E801853108F44B
:1023100026C2E091E601F091E70180E1AFE6B4E08A
:1023200001900D928A95E1F780910F018823E1F3E6
:102330001F9280910C018F9384E58F930E94AD0FC3
:102340008AEF8093E3018FEF80930D010F900F9040
:102350000F907DCFA091E601B091E7018BE0E7E817
:10236000F4E00D9001928A95E1F7809190048093BA
:1023700018068FEF80930D016ACF81E08093F301FF
:1023800066CF8FEF80930D01E091E601F091E701B8
:1023900090818AE0989FC00111249093E20180937C
:1023A000E101892B09F44BCF81E08093F00147CF05
:1023B0008FEF80930D01E091E601F091E7019081AC
:1023C00097FDFBC182E08093ED011092DE01109237
:1023D000DD0181E08093F1013ACFE091E601F091D7
:1023E000E701E081E03208F4B7C18FE180930E018C
:1023F000C0CFE091E601F091E70180819181909357
:102400000703809306032091040330910503821B88
:10241000930B845E9D4F68E671E00E94DB76845BDF
:102420009040909303038093020311CFA091E601A3
:10243000B091E7019C91892F8150853008F4D8C173
:102440008C9189834CE668EC76E00E94420780918B
:102450000F018823E1F381E090E09F938F93CE01F9
:1024600001969F938F9381E08F938F9386E48F9350
:102470000E94AD0F8DB79EB707968DBF8091EA027F
:10248000882309F47DC180E00E94E5070E94017461
:10249000AFCEA091E601B091E7018D919C91909310
:1024A0000703809306032091040330910503821BE8
:1024B000930B845E9D4F68E671E00E94DB76845B3F
:1024C0009040909303038093020392CEA091E60183
:1024D000B091E7018C91992787FD909590937406B0
:1024E00080937306FD018181992787FD90959093D4
:1024F0007606809375068281992787FD9095909343
:102500007806809377068381992787FD909590932D
:102510007A06809379068481992787FD9095909318
:102520007C0680937B068581992787FD9095909303
:102530007E0680937D068681992787FD90959093EE
:10254000800680937F068781992787FD90959093D9
:102550008206809381068085992787FD90959093C8
:102560008406809383068185992787FD90959093B3
:102570008606809385068285992787FD909590939E
:102580008806809387068385992787FD9095909389
:102590008A06809389062CCE8091E801853108F463
:1025A000FAC0A091E601B091E70180E1EFE6F4E026
:1025B0000D9001928A95E1F780EF8093E3018FEF10
:1025C00080930D0115CE2091E6013091E701F901CC
:1025D00080818150853020F48181823509F465C085
:1025E000198280910F018823E1F381E090E09F93AD
:1025F0008F93CE0101969F938F9381E08F938F935A
:1026000083E58F930E94AD0FEDB7FEB73796EDBF10
:1026100035CF81E08093EE01D2CFA091E601B09159
:10262000E7018C918F3F09F4FCC08C91882309F05D
:10263000ADC081E08C93A091E601B091E7014CE63A
:1026400068EC76E08C910E94420780910F0188230C
:10265000E1F3E091E601F091E7018081898382E571
:102660008A838CE690E09F938F9388EC96E09F930B
:102670008F9321E030E03F932F93CE0102969F93FA
:102680008F933F932F93CE01820F931F9F938F932E
:1026900083E08F9381E08F9381E58F930E94AD0F4C
:1026A000ADB7BEB71F96ADBFA3CD68EC76E08CE6A4
:1026B0002E5F3F4FDB01F901982F01900D929A9503
:1026C000E1F722503040482FD9018C910E946B07CE
:1026D000809105079927AA27BB27BC01CD0124ECCF
:1026E00039E040E050E00E949C76DC01CB01809311
:1026F0009E0190939F01A093A001B093A1018091AE
:1027000006079927AA27BB27BC01CD010E949C760A
:10271000DC01CB0180939A0190939B01A0939C01D3
:10272000B0939D01E091E601F091E70180810E9464
:102730005F070E949A07898354CF8AE0989FC0015F
:1027400011240E9416189093620480936104A09152
:10275000E601B091E7016ACDE0930E010ACEE09167
:10276000E601F091E70180819181A281B38180939C
:102770006F0490937004A0937104B0937204D4CD4D
:102780006EE670E089810E94CB337DCE863008F4FE
:1027900056CF85E04FCFA091E601B091E7018D9132
:1027A0009D910D90BC91A02D80936F049093700427
:1027B000A0937104B0937204FFCE9095809146026D
:1027C000982B9093460291818AE0989FC001112432
:1027D0009093DE018093DD0184E08093ED0180EA37
:1027E0009FE00E9416189093DC018093DB01F1CDED
:1027F000892F0E945F07A091E601B091E70120CEEA
:1028000046E054E08DE4FA01282F0D9001922A95BC
:10281000E1F7A8EEB3E0FA01182E0E9481779983C0
:102820003CCD0E949A07E091E601F091E701808398
:10283000A091E601B091E701F8CEE2E0CE5F0C9402
:102840005777982F8091C00085FFFCCF9093C600EA
:1028500008950F931F9388E18093C1008091C00079
:1028600082608093C0008091C10080688093C10025
:102870008091C10080648093C10000E010E000936B
:10288000C5008AE290E08093C4008091E1019091BC
:10289000E2010E94161890936404809363048CED07
:1028A00090E00E94161890939304809392041092E3
:1028B00065048EE48093660485E0809369048BE070
:1028C00080936704109268041093E7010093E60177
:1028D0001092E5011F910F910895A0E1B0E0E3E7A8
:1028E000F4E10C94377780910F01882309F4A9C291
:1028F0008091DB019091DC010E941F18882309F070
:10290000F2C08091DD019091DE01892B09F088C130
:102910008091F101882309F44BC080910F01882335
:1029200009F446C08091ED01843008F0A6C11092F0
:1029300048028AE895E09F938F9385E792E29F9300
:102940008F93E0910404F0910504099584E190E0EF
:102950009F938F9388E291E09F938F9381E090E023
:102960009F938F938DEE91E09F938F9382E08F934F
:1029700081E08F9388E48F930E94AD0F8091ED01E9
:10298000982F9F5F2DB73EB7215F3F4F2DBF8430FB
:1029900008F454C21092ED018091DD019091DE01A6
:1029A0000E94161890933505809334051092F1011A
:1029B0008091F201882329F080910F01882309F08A
:1029C00073C18091EF01882329F080910F01882342
:1029D00009F01DC28091F301882329F080910F0135
:1029E000882309F0FCC180919204909193040E9485
:1029F0001F18882329F080910F01882309F092C1C4
:102A00008091E1019091E201892B09F0FFC0809152
:102A1000F001882329F080910F01882309F00AC171
:102A20008091DF019091E001892B09F069C08091CC
:102A30000E018F3F79F1992782959295907F982783
:102A4000807F982786579C4F40E150E0BC01CE0123
:102A500001960E94A87580E190E09F938F93CE012C
:102A600001969F938F9381E090E09F938F938EE0E8
:102A700091E09F938F9382E08F9381E08F9381E425
:102A80008F930E94AD0F8FEF80930E018DB79EB78D
:102A90000B968DBF80911806882329F080910F0135
:102AA000882309F028C18091EE01882309F4C9C167
:102AB00080910F01882309F4C4C184E390E09F93BF
:102AC0008F9389E596E09F938F9381E08F938F9307
:102AD00080E58F930E94AD0F1092EE018DB79EB7E7
:102AE00007968DBFAEC11092DE011092DD011092EB
:102AF000E2011092E1011092E0011092DF0101CF9A
:102B000080916104909162040E941F18882309F447
:102B10008ECF80910F01882309F489CF8091E3063D
:102B20009927880F991F880F991F7C010027F7FCB0
:102B30000095102F8091400390914103A091420392
:102B4000B0914303BC01CD01A80197010E94107709
:102B500030935404209353048091380390913903A7
:102B6000A0913A03B0913B03BC01CD01A8019701AC
:102B70000E941077309356042093550420918F07BC
:102B8000309190074091910750919207DA01C90165
:102B900003E0880F991FAA1FBB1F0A95D1F7820F68
:102BA000931FA41FB51F820F931FA41FB51F209151
:102BB0007E0130917F014091800150918101BC01E3
:102BC000CD010E94107730935804209357048EE073
:102BD00090E09F938F9383E594E09F938F9381E0A0
:102BE0008F938F9383E48F930E94AD0F8091DF01C9
:102BF0009091E0010E941618909362048093610402
:102C00002DB73EB7295F3F4F2DBF11CF8091630491
:102C1000909164040E941F18882309F0FCCEF7CE1F
:102C200080913405909135050E941F18882309F082
:102C300074CE6ECE82E490E09F938F9386ED95E004
:102C40009F938F9381E08F938F9384E48F930E945F
:102C5000AD0F1092F0018DB79EB707968DBF809192
:102C6000E1019091E201009709F4DACE0E94161872
:102C70009093640480936304D3CE0E94802280E505
:102C800090E09F938F9388E291E09F938F9381E0F0
:102C90008F938F9388E48F930E94AD0F2DB73EB72B
:102CA000295F3F4F2DBF78CE0E94802280E590E0C3
:102CB0009F938F9388E291E09F938F9321E030E080
:102CC0003F932F9387E291E09F938F933F932F93AE
:102CD00087E492E09F938F9383E08F9381E08F93BB
:102CE0008CE48F930E94AD0F1092F2018DB79EB7C6
:102CF0000F968DBF66CE81E090E09F938F9388E121
:102D000096E09F938F9381E08F938F9382E48F93CC
:102D10000E94AD0F109218062DB73EB7295F3F4FA6
:102D20002DBFC1CE8091E3069927880F991F880F88
:102D3000991F7C010027F7FC0095102F809140031C
:102D400090914103A0914203B0914303BC01CD0196
:102D5000A80197010E9410773093800420937F048C
:102D60008091380390913903A0913A03B0913B03CD
:102D7000BC01CD01A80197010E9410773093820415
:102D8000209381048091D702809383048091D6029E
:102D90008093840488E090E09F938F938FE794E082
:102DA0009F938F9381E08F9383E08F9387E78F9337
:102DB0000E94AD0F809185042DB73EB7295F3F4F2C
:102DC0002DBF853018F086E08093850483E690E07F
:102DD0000E941618909393048093920411CE8BE076
:102DE00090E09F938F9387E894E09F938F9381E087
:102DF0008F9380910C018F9387E48F930E94AD0F86
:102E00001092F3018DB79EB707968DBFECCD8AE087
:102E100090E09F938F9385E694E09F938F9381E05A
:102E20008F938F9386E58F930E94AD0F1092EF01E1
:102E30002DB73EB7295F3F4F2DBFCCCD9093ED010D
:102E4000ABCDE6E0C05F0C9453771F920F920FB6A4
:102E50000F9211242F933F935F936F937F938F93E0
:102E60009F93AF93BF93EF93FF93809101028823C9
:102E700029F0809101028150809301028091E70343
:102E8000882319F081508093E703809109028150D3
:102E90008F3F09F490C080930902809102029091C3
:102EA0000302892B09F1809102029091030201979C
:102EB0009093030280930202809102029091030298
:102EC000209110013091110182239323892B91F0DD
:102ED000809102018A3009F492C0479A8091D90307
:102EE000882309F093C011C08FEF9FEF90931101D9
:102EF00080931001809102018A3009F474C04798D0
:102F00008091D903882309F081C08091D40683FF82
:102F10007DC086B19927FC01E071F07084FD65C029
:102F20008091040290910502892B09F43FC08091A1
:102F30000402909105028A569140C0F580910402E6
:102F40009091050269E270E00E94C77680910402C8
:102F500090910502860F971F9093050280930402BB
:102F600080910402909105020B9708F44AC0809169
:102F70000402909105020A97909307038093060339
:102F8000809106039091070320910403309105037B
:102F9000821B930B845E9D4F68E671E00E94DB7696
:102FA000845B904090930303809302031092050288
:102FB000109204022BC089E08093090280911201D3
:102FC0008F5F817080931201882319F481E08093D0
:102FD00006028091070290910802019690930802E0
:102FE000809307025ACF5A988BCF80910402909118
:102FF00005020196909305028093040207C05A9A35
:103000007FCFF0930703E0930603BACFFF91EF91D0
:10301000BF91AF919F918F917F916F915F913F9100
:103020002F910F900FBE0F901F90189520910702BF
:1030300030910802280F391FC90101960895209187
:10304000070230910802821B930B892F99278695DE
:10305000807490700895CF93DF930E941618EC014E
:10306000CE010E941F188823D9F3DF91CF910895D4
:103070001F93CF93DF930E941618EC011FEC08C03A
:1030800080911701882321F09093170110937A0003
:10309000CE010E941F18982F882391F3DF91CF91C2
:1030A0001F9108959FB7F8945F983E9A469A809131
:1030B000B0008F708093B0008091B00083608093E7
:1030C000B0008091B1008B738093B1008091B1000A
:1030D0008B608093B1001092B2008FEF8093B300A9
:1030E0008091B00080688093B000809170008A7FEA
:1030F00080937000809170008260809370009FBF09
:1031000008958AE090E00E9416189093110280932F
:10311000100282E085BD83EA84BD17BC88E788BDC4
:1031200086E086BD80916E00816080936E00089578
:103130001F920F920FB60F9211242F933F934F932C
:103140005F936F937F938F939F93AF93BF93EF930F
:10315000FF93809102018431C0F480910A02882398
:1031600009F446C020910B0230910C0241E02F3748
:10317000340708F49CC08FEF8093B3002F5F30407A
:1031800030930C0220930B02C7C380910A0288235C
:1031900049F78091B00086FFADC08091B0008F7B71
:1031A0008093B000E0910F02EE2309F0EFC0809110
:1031B000FB06282F33278DED96E0289FA001299F3D
:1031C000500D389F500D1124CA0120910D023091ED
:1031D0000E02821B930B90930C0280930B021092B1
:1031E0000E0210920D02469A81E080930A02BACF35
:1031F0008091B00086FFA8C08091B0008F7B809343
:10320000B00089EA93E090930C0280930B028091C6
:103210001301909114019C01220F331F280F391FB5
:1032200080918A019927880F991F880F991F280F6D
:10323000391F37FDA0C1C90195958795959587954B
:1032400090931401809313019093FF018093FE01EA
:103250008091260780FFE5C08091F406682F7727CC
:1032600088279927209140033091410340914203E0
:103270005091430357FD61C1A7E055954795379598
:103280002795AA95D1F70E949C769B01AC0197FDEA
:1032900083C1F6E05595479537952795FA95D1F76F
:1032A0008091FE019091FF01820F931FE4C02F3F98
:1032B000310569F060F0A9014F5F50404F3751056B
:1032C00088F480E88093B3002058304059CF809133
:1032D0000B028093B30010920C0210920B0210921A
:1032E0000A021AC38FEF8093B30050930C024093ED
:1032F0000B0212C38091B00080648093B0008CEB0D
:1033000090E090930C0280930B0280910D029091BB
:103310000E0284549F4F90930E0280930D02809171
:103320000002882329F08091F402853B08F0F9C05F
:10333000469A90910F029F5F8091FB06891708F0D3
:10334000EDC010920F0250CF8091B0008064809346
:10335000B0008091FB06282F33278DED96E0289F43
:10336000A001299F500D389F500D1124CA012091B2
:103370000D0230910E02821B930B90930C028093EE
:103380000B029C0181E080930A02F0CE29EA33E02F
:103390008E2F99278330910509F4C5C0843091059B
:1033A0000CF0EEC030930C0220930B02813091059B
:1033B00009F4FCC0029709F490C1FF27EE0FFF1F2C
:1033C000E75AF94F80819181880F991F20910B0254
:1033D00030910C02820F931F90930C0280930B028A
:1033E00020910B0230910C0255E02D3D350708F479
:1033F000B5C08CED95E090930C0280930B029C017C
:103400002C5B304030930C0220930B0280910D0214
:1034100090910E02820F931F90930E0280930D02E3
:10342000E3CE8091F406682F77278827992720918B
:10343000400330914103409142035091430357FDB3
:1034400081C0E7E05595479537952795EA95D1F7DF
:103450000E949C769B01AC0197FDA3C076E0559538
:103460004795379527957A95D1F78091FE019091F0
:10347000FF01821B930B9093FF018093FE018091CB
:10348000F506282F3327220F331F220F331F809179
:10349000FE019091FF01821793077CF08091F60660
:1034A000282F3327220F331F220F331F8091FE0155
:1034B0009091FF012817390724F43093FF012093DE
:1034C000FE012091FE013091FF0180910B0290914D
:1034D0000C02280F391F205032408091FE0190913C
:1034E000FF0197FD4BC0959587959595879590938E
:1034F000FF018093FE0145E02D3D340740F18CED46
:1035000095E090930C0280930B0220910B02309176
:103510000C0230930E0220930D0234CF90930F02D1
:1035200063CE469806CF80915B079927880F991F35
:10353000880F991F87559E4F4FCF21583F4F4F4FB0
:103540005F4F9ACE21583F4F4F4F5F4F7ACF51E098
:103550002737350758F487E791E0D3CF81E0273745
:10356000380708F04DCF87E791E045CF30930C0244
:1035700020930B02CACF2D5F3F4F5DCE0396B3CF92
:103580008430910509F4A6C0059709F43AC1309337
:103590000C0220930B0211CF215C3F4F4F4F5F4F26
:1035A00078CE215C3F4F4F4F5F4F58CF8091130132
:1035B000909114019C01220F331F280F391F809115
:1035C0008A019927880F991F880F991F280F391F83
:1035D00037FD70C1C901959587959595879590930D
:1035E0001401809313019093FF018093FE01809159
:1035F000260780FF09C18091F406682F7727882766
:10360000992720914003309141034091420350910A
:10361000430357FD5EC1E7E05595479537952795DC
:10362000EA95D1F70E949C769B01AC0197FD4CC1B5
:10363000B6E05595479537952795BA95D1F780917E
:10364000FE019091FF01820F931F9093FF018093E1
:10365000FE018091F506282F3327220F331F220FFA
:10366000331F8091FE019091FF01821793077CF038
:103670008091F606282F3327220F331F220F331F86
:103680008091FE019091FF012817390724F43093AF
:10369000FF012093FE018091FE019091FF01209196
:1036A0000B0230910C02820F931F80509240909336
:1036B0000C0280930B028091FE019091FF0197FD17
:1036C000FCC095958795959587959093FF0180937C
:1036D000FE0186CE8091C70628CF8091150190917A
:1036E00016019C01220F331F280F391F8091890179
:1036F0009927880F991F880F991F280F391F37FDA9
:10370000E0C0C90195958795959587959093160189
:10371000809315019093FD018093FC018091260711
:1037200081FF9DC08091F806682F77278827992709
:10373000209138033091390340913A0350913B0373
:1037400057FDD6C0A7E05595479537952795AA957B
:10375000D1F70E949C769B01AC0197FDCEC0F6E0AC
:103760005595479537952795FA95D1F78091FC01A6
:103770009091FD01820F931F9093FD018093FC01B6
:103780008091F906282F3327220F331F220F331F72
:103790008091FC019091FD01821793077CF080914C
:1037A000FA06282F3327220F331F220F331F809151
:1037B000FC019091FD012817390724F43093FD0195
:1037C0002093FC018091FC019091FD0120910B025E
:1037D00030910C02820F931F8050924090930C0204
:1037E00080930B028091FC019091FD0197FD67C0D1
:1037F00095958795959587959093FD018093FC010C
:10380000EFCD8091650791CE8091F406682F7727E0
:10381000882799272091400330914103409142032A
:103820005091430357FD5FC0A7E0559547953795E5
:103830002795AA95D1F70E949C769B01AC0197FD34
:103840004DC0F6E05595479537952795FA95D1F7F0
:103850008091FE019091FF01821B930BF6CE809127
:10386000F806682F77278827992720913803309109
:10387000390340913A0350913B0357FD48C0E7E0BC
:103880005595479537952795EA95D1F70E949C76EF
:103890009B01AC0197FD36C076E05595479537956D
:1038A00027957A95D1F78091FC019091FD01821BBB
:1038B000930B62CF2D5F3F4F8DCE039602CF0396C1
:1038C00097CF2D5F3F4F1DCF215C3F4F4F4F5F4F35
:1038D000AFCE21583F4F4F4F5F4F9DCE215C3F4FA2
:1038E0004F4F5F4FAECF21583F4F4F4F5F4F9CCF51
:1038F00021583F4F4F4F5F4F25CF215C3F4F4F4FD8
:103900005F4F2DCF215C3F4F4F4F5F4FC5CF2158A9
:103910003F4F4F4F5F4FB3CFFF91EF91BF91AF91AB
:103920009F918F917F916F915F914F913F912F91D7
:103930000F900FBE0F901F90189510927C008FEC87
:1039400080937A000895A0E0B0E0E9EAFCE10C94ED
:10395000357703E010E0D8010E946877802DC82FEA
:10396000DD27C531D10508F02A97C7BD109219028D
:1039700084E690E00E94381880911B0190911C0110
:103980008052934010F4C0E0D0E0CA3FD10528F542
:103990009FE9C92E95E0D92E81E2E82E84E1F82E28
:1039A000C7BD82E390E00E943818DF92CF92FF9269
:1039B000EF92E0910404F0910504099580911B01B8
:1039C00090911C010F900F900F900F908052934098
:1039D00020F02196CA3FD10518F3D8010C2E0E9481
:1039E0007577C09325068CE291E00E943818E8E0D4
:1039F000CDB7DEB70C945177EF92FF920F931F93E0
:103A0000CF93DF9300E0009314020093130200931E
:103A1000120280ED97E00E941618EC011CE831E0DC
:103A2000F32E25EFE22E033009F4B2C000E08091BE
:103A3000290290912A028C5F93400CF098C08091EB
:103A40001A01815080931A018091270290912802D7
:103A50008C5F93400CF080C080911901815080935D
:103A6000190180912502909126028C5F93400CF001
:103A700051C08091180181508093180188E0809393
:103A80004E020E94FD2C80911A018A3008F05CC021
:103A9000F09214028AE080931A01809119018A3011
:103AA00008F04AC0F09213028AE0809319018091D5
:103AB00018018A30D0F5F09212028AE08093180142
:103AC00080914E028823B1F0CE010E941F188823F6
:103AD000B9F381EA95E09F938F9381E294E19F93FC
:103AE0008F93E0910404F091050409950F900F90D5
:103AF0000F900F90109217018FEC80937A008091B5
:103B000017018823E1F31A3008F447C0115009F077
:103B10008ACF48C080912502909126028750944018
:103B20008CF1809118018F5FA7CF863F48F2F09209
:103B30001202E0921801C4CF863F08F4B8CFF09289
:103B40001302E0921901B3CF863F08F4A6CFF0929A
:103B50001402E0921A01A1CF8091270290912802CD
:103B6000875094408CF0809119018F5F78CF8091BD
:103B7000290290912A028750944044F080911A01C2
:103B80008F5F60CF0F5F7ACF0F5F6BCF01E05CCFAD
:103B90001B3008F44BCF19E049CF8AE090E00E9437
:103BA0003818B4CF86E490E00E943818E6E0CDB72C
:103BB000DEB70C9453771F920F920FB60F92112419
:103BC000AF92BF92CF92DF92EF92FF920F931F932B
:103BD0002F933F934F935F936F937F938F939F9315
:103BE000AF93BF93EF93FF9320913202822F9927D7
:103BF000AA27BB272F5FFC01429720F4E756FF4F0F
:103C00000C9462771092320282E0809331028091AC
:103C1000310280937C0080913202882309F443C4EE
:103C20008FEC80937A003FC4209332028091780019
:103C3000909179002091370230913802820F931FC2
:103C4000909338028093370281E0DFCF20933202D5
:103C50008091780090917900209135023091360260
:103C6000820F931F909336028093350284E0CDCF6C
:103C700020933202809178009091790020914E0338
:103C800030914F03821B930B90932406809323065D
:103C900080912306909124069093400280933F02E6
:103CA00082E0B3CF2093320280914C0390914D0378
:103CB0002091780030917900821B930B90931A0623
:103CC000809319068091190690911A0690933E02EE
:103CD00080933D0287E099CF209332028091780053
:103CE00090917900909334028093330286E08DCFD7
:103CF000209332022091780030917900309336027F
:103D0000209335021092310282CF2093320220910B
:103D1000780030917900309338022093370281E0A7
:103D200074CF1092320281E08093170180911502C6
:103D3000909116020196909316028093150280913D
:103D400078009091790090931C0180931B018091E1
:103D50001B0190911C015C01CC24DD248091410267
:103D600090914202A0914302B0914402A80EB91E64
:103D7000CA1EDB1E809145028F5F823108F4E8C2C3
:103D800080911D0190911E01A0911F01B091200111
:103D90007C018D0123E0EE0CFF1C001F111F2A95F2
:103DA000D1F7E81AF90A0A0B1B0BEA0CFB1C0C1DD5
:103DB0001D1D80911902992787FD9095A92FB92F74
:103DC000BC01CD0126EC34E240E050E00E949C763C
:103DD000DC01CB01E81AF90A0A0B1B0BD801C70159
:103DE0000496A11DB11DB7FD23C313E0B595A7959A
:103DF000979587951A95D1F780931D0190931E0191
:103E0000A0931F01B093200180911D0690911E0682
:103E10007C010027F7FC0095102F80911D019091E7
:103E20001E01A0911F01B0912001E81AF90A0A0BA6
:103E30001B0BE092E602F092E7020093E802109377
:103E4000E90220911A0230911B0240911C0250910C
:103E50001D0257FDFDC2B4E055954795379527954E
:103E6000BA95D1F780911A0290911B02A0911C0281
:103E7000B0911D02821B930BA40BB50B80931A0209
:103E800090931B02A0931C02B0931D0280911A0212
:103E900090911B02A0911C02B0911D028E0D9F1DDE
:103EA000A01FB11F80931A0290931B02A0931C02C3
:103EB000B0931D028091170290911802BC01629587
:103EC0007295707F7627607F7627681B790B20912B
:103ED0001A0230911B0240911C0250911D0257FDA5
:103EE000B2C2F4E05595479537952795FA95D1F7E5
:103EF0008091E6029091E702821B930B880F991F35
:103F0000880F991F880F991F860F971F97FDA9C2C9
:103F10009595879595958795959587959595879589
:103F20009093180280931702D601C501D7FC95C261
:103F3000B595A795979587958093410290934202F6
:103F4000A0934302B093440289E08093450282E04B
:103F50005CCE2093320220917800309179008091DC
:103F6000350290913602280F391F809102018A3064
:103F700009F448C2220F331F220F331F3093360239
:103F800020933502C90137FD73C2959587959595A4
:103F90008795959587959093280280932702809125
:103FA0003B0290913C02820F931F97FD66C295954C
:103FB000879590933C0280933B0220915603309169
:103FC0005703821B930B9093220180932101209130
:103FD0002D0230912E028091210190912201280F13
:103FE000391F37FD47C23595279530932E02209310
:103FF0002D0283E00ACE2093320220917800309186
:1040000079008091370290913802280F391F8091F2
:1040100002018A3009F407C2220F331F220F331F17
:104020003093380220933702C90137FDFFC19595BF
:104030008795959587959595879590932A02809376
:1040400029028091390290913A02820F931F97FDC5
:104050000DC29595879590933A02809339022091ED
:10406000580330915903821B930B90932401809342
:10407000230120912F0230913002809123019091F1
:104080002401280F391F37FDEEC135952795309350
:10409000300220932F0281E0B8CD2093320280912C
:1040A00078009091790020914E0330914F03821B4C
:1040B000930B90932406809323068091230690917E
:1040C000240620913F0230914002820F931F90936B
:1040D00022028093210282E098CD209332028091C7
:1040E0004C0390914D032091780030917900821B10
:1040F000930B90931A06809319068091190690915C
:104100001A0620913D0230913E02820F931F909338
:1041100024028093230287E078CD2093320280919D
:1041200002018A3009F471C1843109F4A8C1809177
:104130007800909179002091330230913402820FFF
:10414000931F909326028093250286E05ECD2093F4
:10415000320280917800909179002091350230915F
:104160003602820F931F909336028093350210928D
:1041700031024DCD20933202E2CD20933202809164
:10418000780090917900AA2797FDA095BA2FBC01DD
:10419000CD010E9422767B018C0180914603909193
:1041A0004703A0914803B09149039C01AD01C801A8
:1041B000B7010E94C275DC01CB01BC01CD010E9498
:1041C0000576DC01CB019093200280931F02809141
:1041D0001F029091200202970CF4C6C08091460302
:1041E00090914703A0914803B091490320E030E843
:1041F0004BE354E4BC01CD010E942C768823DCF50E
:104200008091460390914703A0914803B0914903E0
:104210002AE037ED43EA5CE3BC01CD010E94C3759F
:10422000DC01CB018093460390934703A09348039E
:10423000B09349038091C4029091C502845F91407C
:10424000D0F48091460390914703A0914803B09128
:1042500049032DEC3CEC4CEC5DE3BC01CD010E942C
:10426000C375DC01CB018093460390934703A09371
:104270004803B093490381E080931E028091780047
:104280009091790090931C0680931B0680911F02E9
:1042900090912002AA2797FDA095BA2F209108039C
:1042A0003091090340910A0350910B03820F931F31
:1042B000A41FB51F8093080390930903A0930A03DA
:1042C000B0930B03209108033091090340910A0336
:1042D00050910B0357FDB2C00AE0559547953795AD
:1042E00027950A95D1F78091080390910903A09131
:1042F0000A03B0910B03821B930BA40BB50B8093A5
:10430000080390930903A0930A03B0930B0383E07F
:104310007CCC2093320280912501909126019C0152
:10432000220F331F280F391F809178009091790058
:1043300063E070E00E94C776260F371F36952795F9
:1043400036952795309326012093250185E05DCC95
:1043500080934502A0924102B0924202C092430271
:10436000D092440282E051CC80911F0290912002B1
:104370008F5F9F4F0CF07FCF809146039091470352
:10438000A0914803B091490320E030E849E054E4AB
:10439000BC01CD010E942F7618160CF06CCF8091D5
:1043A000460390914703A0914803B09149032AE046
:1043B00037ED43EA5CE3BC01CD010E94C275DC012C
:1043C000CB018093460390934703A0934803B09397
:1043D00049038091C4029091C502845F914008F026
:1043E0004ACF8091460390914703A0914803B09132
:1043F00049032DEC3CEC4CEC5DE3BC01CD010E948B
:10440000C2752FCF220F331FB9CD809178009091C4
:1044100079002091330230913402820F931F01966C
:10442000969587958ECE220F331FFACD0796FFCD36
:10443000D801C7010B96A11DB11DD7CC21503C4F0F
:104440004F4F5F4F49CF215F3F4F4F4F5F4F49CD98
:10445000215F3F4F4F4F5F4FFECC0196A11DB11D15
:1044600067CD0F9655CD2F5F3F4F0FCE0196F1CD03
:1044700007968BCD2F5F3F4FB6CD019698CD80919B
:104480007800909179002091330230913402820FAC
:10449000931F2FEF37E0281B390B30932602209310
:1044A000250286E0B2CBFF91EF91BF91AF919F9132
:1044B0008F917F916F915F914F913F912F911F91BC
:1044C0000F91FF90EF90DF90CF90BF90AF900F9043
:1044D0000FBE0F901F90189590E2E8E2F1E08FE494
:1044E0009193815087FFFCCF089590914802E8E2B4
:1044F000F1E0E90FF11D80839F5F909348020895DA
:104500000F931F93CF93DF932091460220FF08C0A3
:1045100080914702882309F46BC081508093470241
:1045200021FF0AC09091470280912701981709F452
:104530006BC09F5F90934702822F992780FF02C034
:1045400081FD5BC00E946C22909147029A3030F549
:1045500081E180934802892F99279F938F9388ED5B
:1045600095E09F938F93C5E7D2E2DF93CF93E091DD
:104570000404F091050409952DB73EB72A5F3F4F1B
:104580002DBF20914702822F9927AA27BB27FC0124
:10459000419730F5E555FF4F0C94627780E18093A9
:1045A0004802892F99279F938F938DED95E09F93D4
:1045B0008F93C5E7D2E2DF93CF93E0910404F091AB
:1045C000050409956DB77EB76A5F7F4F6DBF209177
:1045D0004702822F9927AA27BB27FC014197D0F2D7
:1045E00080912701281761F0109247020C94F02C5B
:1045F000809127018093470293CF10924702A2CF68
:10460000215020932701F0CF1092470295CF1092AE
:10461000480282EE95E09F938F93DF93CF93E091D2
:104620000404F0910504099584E1809348020F90F9
:104630000F900F900F9086E690E09F938F938EE4FB
:1046400090E09F938F931F921F92809102016AE0E6
:104650000E94BB76892F99279F938F9380910201A7
:104660000E94BB7699279F938F9382EF95E09F934B
:104670008F93DF93CF93E0910404F09105040995A3
:1046800088E2809348028DB79EB70E968DBF87E073
:1046900094E09F938F930E949A0799279F938F93FB
:1046A00087E096E09F938F93DF93CF93E09104048C
:1046B000F091050409958091A4019091A5012DB771
:1046C0003EB7285F3F4F2DBF069710F40C94132C74
:1046D00090914B02992311F40C94F02C8CE380936D
:1046E0004802892F99279F938F9382E296E09F93A8
:1046F0008F9385E792E29F938F93E0910404F0916A
:10470000050409956DB77EB76A5F7F4F6DBF0C9446
:10471000F02C1092480281E599E09F938F93DF93EC
:10472000CF93E0910404F0910504099584E180930E
:1047300048020F900F900F900F9080918A01992757
:104740009F938F9389E599E09F938F93DF93CF9306
:10475000E0910404F0910504099588E280934802F1
:104760006DB77EB76A5F7F4F6DBF8091FE019091FC
:10477000FF019F938F9387E699E09F938F93DF9339
:10478000CF93E0910404F091050409958CE38093A4
:1047900048028DB79EB706968DBF8091F606992781
:1047A0009F938F938091F50699279F938F9385E729
:1047B00099E09F938F93DF93CF93E0910404F0915E
:1047C000050409952DB73EB7285F3F4F2DBF0C94C8
:1047D000F02C109248028091F90299279F938F93B1
:1047E00081E299E09F938F93DF93CF93E09104044C
:1047F000F0910504099584E1809348022DB73EB7F6
:104800002A5F3F4F2DBF8091FA0299279F938F9384
:104810008DE299E09F938F93DF93CF93E09104040F
:10482000F0910504099588E2809348026DB77EB740
:104830006A5F7F4F6DBF8091FB0299279F938F9393
:1048400089E399E09F938F93DF93CF93E0910404E2
:10485000F091050409958CE3809348028DB79EB7CB
:1048600006968DBF8091FC0299279F938F9385E4D4
:1048700099E09F938F93DF93CF93E0910404F0919D
:10488000050409952DB73EB72A5F3F4F2DBF0C9405
:10489000F02C109248028091F50299279F938F93F4
:1048A00081EF98E09F938F93DF93CF93E09104047F
:1048B000F0910504099584E1809348028DB79EB775
:1048C00006968DBF8091F60299279F938F938DEF67
:1048D00098E09F938F93DF93CF93E0910404F0913E
:1048E0000504099588E2809348022DB73EB72A5FF8
:1048F0003F4F2DBF8091F70299279F938F9389E0B7
:1049000099E09F938F93DF93CF93E0910404F0910C
:10491000050409958CE3809348026DB77EB76A5F02
:104920007F4F6DBF8091F80299279F938F9385E108
:1049300099E09F938F93DF93CF93E0910404F091DC
:10494000050409958DB79EB706968DBF0C94F02C83
:10495000109248028FEB98E09F938F93DF93CF9351
:10496000E0910404F0910504099584E180934802E4
:104970000F900F900F900F9080910203909103037E
:104980009F938F9387EC98E09F938F93DF93CF93C0
:10499000E0910404F0910504099588E280934802AF
:1049A0008DB79EB706968DBF809106039091070341
:1049B0009F938F9385ED98E09F938F93DF93CF9391
:1049C000E0910404F091050409958CE3809348027A
:1049D0002DB73EB72A5F3F4F2DBF809104039091C2
:1049E00005039F938F9383EE98E09F938F93DF93BC
:1049F000CF9383CE1092480286E898E09F938F93DE
:104A0000DF93CF93E0910404F0910504099584E1CC
:104A1000809348020F900F900F900F90809159064D
:104A200090915A069F938F938FE898E09F938F936E
:104A3000DF93CF93E0910404F0910504099588E297
:104A4000809348028DB79EB706968DBF8091F40281
:104A500099279F938F938FE998E09F938F93DF938C
:104A6000CF93E0910404F091050409958CE38093C1
:104A700048022DB73EB72A5F3F4F2DBF80915806A1
:104A8000992701979F938F938FEA98E0AECF10926A
:104A9000480280912501909126016AE070E00E9411
:104AA000DB769F938F9380912501909126016AE098
:104AB00070E00E94DB767F936F938CE398E09F9386
:104AC0008F93DF93CF93E0910404F091050409954F
:104AD00084E1809348026DB77EB7685F7F4F6DBFFA
:104AE00080910508909106086AE070E00E94C77600
:104AF0009F938F9380910508909106086AE070E07B
:104B00000E94C7767F936F9380E598E09F938F9381
:104B1000DF93CF93E0910404F0910504099588E2B6
:104B2000809348028DB79EB708968DBF8091070885
:104B3000909108089F938F9384E698E09F938F93BA
:104B4000DF93CF93E0910404F091050409958CE381
:104B5000809348022DB73EB72A5F3F4F2DBF80910B
:104B6000090890910A089F938F9384E798E03DCFBE
:104B70001092480282E098E09F938F93DF93CF9347
:104B8000E0910404F0910504099584E180934802C2
:104B90000F900F900F900F9080914E0390914F03C4
:104BA0009F938F9380912102909122029F938F93E4
:104BB0008FE098E09F938F93DF93CF93E09104046D
:104BC000F0910504099588E2809348026DB77EB79D
:104BD000685F7F4F6DBF80914C0390914D039F9311
:104BE0008F9380912302909124029F938F938EE163
:104BF00098E09F938F93DF93CF93E0910404F0911B
:104C0000050409958CE3809348028DB79EB70896FA
:104C10008DBF8091460390914703A0914803B091C6
:104C20004903BC01CD010E940576DC01CB019F93B5
:104C30008F9380915007909151079F938F938DE2AE
:104C400098E0B7CD1092480285E597E09F938F9347
:104C500005E712E2DF93CF93E0910404F09105049D
:104C60000995809102010F900F900F900F908A305C
:104C700009F405C68B3009F42CC5843109F429C523
:104C80008D3009F0ADC684E18093480280911A010D
:104C900099279F938F934091580350915903CA01CC
:104CA00057FD97C695958795959587959595879581
:104CB000959587959F938F939A0157FD87C6359554
:104CC00027953595279535952795809129029091BF
:104CD0002A02821B930B9F938F9386EC97E09F93FE
:104CE0008F931F930F93E0910404F09105040995AD
:104CF00088E2809348026DB77EB7665F7F4F6DBFD5
:104D00008091190199279F938F9340915603509159
:104D10005703CA0157FD62C6959587959595879566
:104D200095958795959587959F938F939A0157FDB4
:104D300052C63595279535952795359527958091B8
:104D4000270290912802821B930B9F938F938AEDE9
:104D500097E09F938F931F930F93E0910404F0913A
:104D6000050409958CE3809348028DB79EB70A9697
:104D70008DBF8091180199279F938F9320915403A1
:104D800030915503C90137FD1FC6959587959F93AF
:104D90008F938091250290912602281B390B3F9317
:104DA0002F938EEE97E09F938F931F930F93E09135
:104DB0000404F091050409952DB73EB7265F3F4FD7
:104DC0002DBF0EC61092480287E59AE09F938F93FD
:104DD000DF93CF93E0910404F0910504099584E1F9
:104DE000809348020F900F900F900F908091D60102
:104DF0009091D7019F938F9385E69AE09F938F932D
:104E0000DF93CF93E0910404F0910504099588E2C3
:104E1000809348026DB77EB76A5F7F4F6DBF809108
:104E2000D8019091D9019F938F9382E79AE09F9345
:104E30008F93DF93CF93E0910404F09105040995DB
:104E400089E4809348028DB79EB706968DBF8FE7A1
:104E50009AE09F938F93DF93CF93E0910404F091B6
:104E600005040995809146020F900F900F900F90C6
:104E700083FFB6C51092D9011092D801AEE0B0E020
:104E800080E0082E0E947577AFE0B0E08091D801F5
:104E9000082E0E947577A4C51092480283EC99E011
:104EA0009F938F93DF93CF93E0910404F0910504D7
:104EB000099584E1809348020F900F900F900F9016
:104EC0008091350699278F7790709F938F9380916B
:104ED000310699278F7790709F938F9380912D063D
:104EE00099278F7790709F938F93809129069927A8
:104EF0008F7790709F938F9383ED99E09F938F931B
:104F0000DF93CF93E0910404F0910504099588E2C2
:104F1000809348026DB77EB7645F7F4F6DBF80910D
:104F2000450699278F7790709F938F9380914106C4
:104F300099278F7790709F938F9380913D06992743
:104F40008F7790709F938F938091390699278F77F1
:104F500090709F938F9384EE99E09F938F93DF934C
:104F6000CF93E0910404F091050409958CE38093BC
:104F700048028DB79EB70C968DBF80915506992734
:104F80008F7790709F938F938091510699278F7799
:104F900090709F938F9380914D0699278F77907093
:104FA0009F938F938091490699278F7790709F9355
:104FB0008F9385EF99E09F938F93DF93CF93E09149
:104FC0000404F091050409952DB73EB7245F3F4FC7
:104FD0002DBF06C51092480283E899E09F938F93F6
:104FE000DF93CF93E0910404F0910504099584E1E7
:104FF000809348020F900F900F900F9080918B0438
:10500000992787FD90959F938F9380918A04992784
:1050100087FD90959F938F9383E999E09F938F935A
:10502000DF93CF93E0910404F0910504099588E2A1
:10503000809348026DB77EB7685F7F4F6DBF8091E8
:105040008C04992787FD90959F938F9380918D0471
:1050500099279F938F9383EA99E09F938F93DF9390
:10506000CF93E0910404F091050409958CE38093BB
:1050700048028DB79EB708968DBF809191049927FD
:105080009F938F9380918E04992787FD90959F938E
:105090008F9383EB99E08DCB109248028BE996E0D9
:1050A0009F938F9305E712E2DF93CF93E09104047F
:1050B000F0910504099584E1809348020F900F90C8
:1050C0000F900F908091400390914103A091420373
:1050D000B0914303B7FD5DC43AE0B595A7959795A8
:1050E00087953A95D1F7BF93AF939F938F9388EAB3
:1050F00096E09F938F931F930F93E0910404F09198
:105100000504099588E2809348022DB73EB7285FD1
:105110003F4F2DBF8091380390913903A0913A03FE
:10512000B0913B03B7FD30C42AE0B595A79597959C
:1051300087952A95D1F7BF93AF939F938F9387EB72
:1051400096E09F938F931F930F93E0910404F09147
:10515000050409958CE3809348026DB77EB7685FBC
:105160007F4F6DBF80910603909107039F938F93AC
:1051700086EC96E09F938F931F930F93DECB8091E5
:10518000D40680FF67C2109248028091E602909197
:10519000E702A091E802B091E902BC01CD0125E04F
:1051A00030E040E050E00E9410773F932F9387E378
:1051B00096E09F938F93DF93CF93E0910404F09157
:1051C0000504099584E1809348028DB79EB7069641
:1051D0008DBF8091E2029091E302A091E402B09130
:1051E000E502BC01CD0125E030E040E050E00E9446
:1051F00010773F932F9384E496E09F938F93DF93F0
:10520000CF93E0910404F0910504099588E280931E
:1052100048022DB73EB72A5F3F4F2DBF80911B013B
:1052200090911C019F938F9381E596E09F938F93BC
:10523000DF93CF93E0910404F091050409958CE38A
:10524000809348026DB77EB76A5F7F4F6DBF87B5A9
:1052500099279F938F938EE596E06BCB109248022F
:105260008091C906E82FFF27EE0FFF1FE75AF94F7D
:10527000808191819F938F938091C806E82FFF27AB
:10528000EE0FFF1FE75AF94F808191819F938F9313
:1052900085E197E09F938F93DF93CF93E091040490
:1052A000F0910504099584E1809348026DB77EB7BB
:1052B000685F7F4F6DBF8091CB06E82FFF27EE0F11
:1052C000FF1FE75AF94F808191819F938F938091BF
:1052D000CA06E82FFF27EE0FFF1FE75AF94F80811C
:1052E000918188589F4F9F938F9385E297E09F937A
:1052F0008F93DF93CF93E0910404F0910504099517
:1053000088E2809348028DB79EB708968DBF809142
:10531000CD06E82FFF27EE0FFF1FE75AF94F8081D8
:10532000918182599F4F9F938F938091CC06E82F54
:10533000FF27EE0FFF1FE75AF94F808191818259B5
:105340009F4F9F938F9385E397E09F938F93DF9376
:10535000CF93E0910404F091050409958CE38093C8
:1053600048022DB73EB7285F3F4F2DBF8091CF0633
:10537000E82FFF27EE0FFF1FE75AF94F8081918139
:1053800082599F4F9F938F938091CE06E82FFF27DE
:10539000EE0FFF1FE75AF94F8081918182599F4F8D
:1053A0009F938F9385E497E09F938F93DF93CF93A1
:1053B000E0910404F091050409956DB77EB7685F2C
:1053C0007F4F6DBF0DC31092480280915D06909192
:1053D0005E069F938F9380915B0690915C069F93EE
:1053E0008F9385ED96E09F938F93DF93CF93E0911A
:1053F0000404F0910504099584E1809348022DB7D7
:105400003EB7285F3F4F2DBF8091610690916206A5
:105410009F938F9380915F06909160069F938F93E7
:1054200085EE96E09F938F93DF93CF93E0910404F2
:10543000F0910504099588E2809348026DB77EB724
:10544000685F7F4F6DBF80916506909166069F9360
:105450008F9380916306909164069F938F9385EF5D
:1054600096E09F938F93DF93CF93E0910404F091A4
:10547000050409958CE3809348028DB79EB7089682
:105480008DBF8091690690916A069F938F9380915A
:105490006706909168069F938F9385E097E089C98E
:1054A0001092480286E09AE09F938F9305E712E2FC
:1054B000DF93CF93E0910404F0910504099584E112
:1054C000809348020F900F900F900F9080913506B7
:1054D000881F8827881F97E0899FC00111248D9617
:1054E0009F938F9380913106881F8827881F96E0AD
:1054F000899FC00111248D969F938F9380912D06D3
:10550000881F8827881F95E0899FC00111248D96E8
:105510009F938F9380912906881F8827881F99273A
:10552000880F991F880F991F8D969F938F9385E100
:105530009AE09F938F93DF93CF93E0910404F091CF
:105540000504099588E2809348026DB77EB7645FD1
:105550007F4F6DBF80914506881F8827881F9BE07D
:10556000899FC00111248D969F938F93809141064E
:10557000881F8827881F9AE0899FC00111248D9673
:105580009F938F9380913D06881F8827881F99E0FD
:10559000899FC00111248D969F938F938091390626
:1055A000881F8827881F9927880F991F880F991FA0
:1055B000880F991F8D969F938F9389E29AE09F930E
:1055C0008F93DF93CF93E0910404F0910504099544
:1055D0008CE3809348028DB79EB70C968DBF809167
:1055E0004906881F8827881F9CE0899FC0011124D5
:1055F0008D969F938F938DE39AE09F938F93DF9384
:10560000CF93E0910404F0910504099580914D0633
:105610002DB73EB72A5F3F4F2DBF87FD1DC180913B
:10562000510687FD06C18091550687FFD9C188E4E0
:105630008093480284E59AE09F938F931F930F9382
:10564000E0910404F091050409950F900F900F90DC
:105650000F90C6C1109248028BE696E09F938F93FD
:10566000DF93CF93E0910404F0910504099584E160
:10567000809348020F900F900F900F908AE796E06A
:105680009F938F93DF93CF93E0910404F0910504EF
:10569000099588E2809348020F900F900F900F9029
:1056A00083E896E09F938F93DF93CF93E091040478
:1056B000F091050409958CE3809348020F900F90B8
:1056C0000F900F9082E996E09F938F93DF93CF9393
:1056D000B7CF84E180934802409158035091590319
:1056E000CA0157FD69C19C013595279535952795C8
:1056F0003595279535952795C90182959295907F87
:105700009827807F9827BA01681B790BCB0177FD1A
:1057100051C1959587959F938F933F932F939A01AE
:1057200057FD45C13595279535952795359527958D
:105730008091290290912A02821B930B9F938F9351
:1057400083E997E09F938F931F930F93E091040455
:10575000F0910504099588E2809348028DB79EB7C1
:105760000A968DBF4091560350915703CA0157FDC9
:105770001CC19C013595279535952795359527951D
:1057800035952795C90182959295907F9827807FBE
:105790009827BA01681B790BCB0177FD04C1959559
:1057A00087959F938F933F932F939A0157FDF8C04E
:1057B000359527953595279535952795809127021D
:1057C00090912802821B930B9F938F9385EA97E019
:1057D0009F938F931F930F93E0910404F09105041E
:1057E00009958CE3809348028DB79EB70A968DBFCA
:1057F0002091540330915503C90137FDCFC09595D1
:1058000087959F938F938091250290912602281B64
:10581000390B3F932F9387EB97E09F938F931F93C1
:105820000F930C94DD238CE38093480285E196E08E
:105830004BCF84E48093480281E59AE09F938F9355
:105840001F930F93E0910404F091050409950F90C4
:105850000F900F900F90E7CE80E4809348028EE483
:105860009AE09F938F93DF93CF93E0910404F0919C
:10587000050409950F900F900F900F90D0CE84E102
:105880008093480240915803509159039A0157FD63
:1058900098C0359527953595279535952795C90154
:1058A000880F991F880F991F880F991F481B590B44
:1058B0005F934F933F932F938091290290912A02F7
:1058C000821B930B9F938F9383E697E09F938F9315
:1058D0001F930F93E0910404F0910504099588E269
:1058E000809348028DB79EB70A968DBF40915603AC
:1058F000509157039A0157FD61C03595279535950D
:10590000279535952795C901880F991F880F991FED
:10591000880F991F481B590B5F934F933F932F9309
:105920008091270290912802821B930B9F938F9363
:1059300084E797E09F938F931F930F93E091040464
:10594000F091050409958CE3809348022DB73EB78A
:10595000265F3F4F2DBF80915403909155039F9335
:105960008F9380915403909155032091250230919B
:105970002602821B930B9F938F9385E897E09F935A
:105980008F931F930F9314CD81509C4FAF4FBF4FF8
:10599000CBCB81509C4FAF4FBF4F9ECB01962FCFAB
:1059A000295F3F4F05CF0196FACE0F96E2CE295FD1
:1059B0003F4FB8CE0196ADCE0F9695CE295F3F4FA3
:1059C0009CCF295F3F4F65CF0196DFC9295F3F4FCD
:1059D00076C90F9667C9295F3F4FABC90F969CC91F
:1059E00010924602DF91CF911F910F91089510926E
:1059F000B9008AE28093B800089585EA8093BC00DC
:105A0000089584E98093BC0008951092B9008093B2
:105A1000BB0085E88093BC0008950E94012D109280
:105A20004E028091BB0010924D0280E88093BC0032
:105A30001092BD001092BA001092BB001092B900F3
:105A40001092B8000E94F72C0E94FD2C80E00E946A
:105A5000052D08958093BB0085E88093BC000895D0
:105A600085EC8093BC00089585E88093BC00089580
:105A70001F920F920FB60F9211242F933F934F93C3
:105A80005F936F937F938F939F93AF93BF93EF93A6
:105A9000FF9380914E02282F3327442755278F5F8D
:105AA00080934E02F90127313105C8F4E454FF4FC9
:105AB0000C94627780914C02E82FFF27EE0FFF1FB6
:105AC000EE0FFF1FE85DF94F9091BB0093838F5F4E
:105AD0008C3008F4ABC010924C020E94012D109241
:105AE0004E02FDC080E80E94052DF9C088E90E94A1
:105AF000052DF5C00E94012D8AE090E09093A5014C
:105B00008093A4010E94FD2CEAC084E10E94052D2F
:105B1000E6C082E10E94052DE2C080911A010E9438
:105B2000052DDDC080E10E94052DD9C080911901AD
:105B30000E94052DD4C0809118010E94052DCFC070
:105B400080914D02E82FFF27EE0FFF1FEE0FFF1F82
:105B5000E85DF94F8F5F80934D0280810E94052D93
:105B6000BEC090914D02292FE92FFF27EE0FFF1F96
:105B7000EE0FFF1FEA5FFB4F858518160CF05EC025
:105B80009C3009F471C0990F892F8E5A0E94052DFF
:105B9000A6C080914C02E82FFF27EE0FFF1FEE0FEB
:105BA000FF1FE85DF94F8091BB0082830E94342D76
:105BB00096C08091B900803409F47EC080914C0277
:105BC000E82FFF27EE0FFF1FEE0FFF1FE85DF94FD5
:105BD00091819F7791838F5F8C3068F110924C0296
:105BE0000E94012D10924E0280914F0280934B0231
:105BF00010924F0274C08091B900803309F440C004
:105C00000E94012D8AE090E09093A5018093A40169
:105C100010924E020E94FD2C62C00E94012D8AE06B
:105C200090E09093A5018093A40159CF80934C02FA
:105C30000E94012D54CF80934C02D2CF9C3008F0AB
:105C40009FCF922F9F5FE92FFF27EE0FFF1FEE0FD1
:105C5000FF1FEA5FFB4F858518161CF0292F9C302B
:105C600080F390934D028CCF10924D0283E080938D
:105C70004E0280914C02880F8D5A0E94052D2FC034
:105C800080914F02882341F590914D0290934F02ED
:105C9000E92FFF27EE0FFF1FEE0FFF1FEB5DF94F00
:105CA0002081822F99278F7790708F3791050CF084
:105CB000A7CF2F5F2083A4CF80914C02E82FFF272E
:105CC000EE0FFF1FEE0FFF1FE85DF94F8181806827
:105CD00081830E94302D88CF90914D02D9CF809141
:105CE000BC0080688093BC00FF91EF91BF91AF91A1
:105CF0009F918F917F916F915F914F913F912F91E4
:105D00000F900FBE0F901F90189589E1ADE8B6E097
:105D1000E9E5F6E011821082329611961C921E92ED
:105D20001296815087FFF6CF1092550310925403BC
:105D30001092570310925603109259031092580371
:105D400008951F920F920FB60F921124EF92FF92B7
:105D50000F931F932F933F934F935F936F937F9373
:105D60008F939F93AF93BF93CF93DF93EF93FF9363
:105D70008091270782FD2CC02091860030918700FA
:105D80008091510290915202281B390B809186001C
:105D9000909187009093520280935102C9018D54D3
:105DA0009440835F9A4108F0B7C08091530280937A
:105DB00058068091530290915402049714F0109267
:105DC0007801C1E0D0E0D0935402C093530219C2CD
:105DD0004091860050918700809155029091560223
:105DE000481B590B80918600909187009093560232
:105DF00080935502CA018D549440835F9A4138F5CF
:105E00008091BF028093500280915002843008F04C
:105E100010C18091C002853608F47DC18AE080936C
:105E2000C002809102018A3009F478C1843109F4FA
:105E300075C1289881E08093BF028091EA0288238F
:105E400009F0DFC18091500280935806DAC1C091F9
:105E5000BF02CD3008F0E6C0CA018B5F9040845B82
:105E6000914008F05DC1425D5140EC2FFF27EE0FDD
:105E7000FF1FE95AFD4F80819181FA01E81BF90B60
:105E8000CF0105960B9708F45EC1EC2FFF27EE0FAC
:105E9000FF1FE95AFD4F808191819C01220F331F22
:105EA000280F391F240F351F37FDA8C17901F5943C
:105EB000E794F594E794CA0101968E159F050CF0BE
:105EC00073C10894E108F1088091F4028E3B08F454
:105ED00062C1EC2FFF27EE0FFF1FDF01A95ABD4F54
:105EE0008D919C919701281B390BC90163E070E0EB
:105EF0000E94DB76CB01880F991F860F971FEF5802
:105F0000FD4F91838083EC2FFF27EE0FFF1FE95A8F
:105F1000FD4FF182E0820BC1C0915302D091540237
:105F2000CD30D1050CF06DC1C9018B5F9040845B11
:105F3000914008F060C0225D3140FE01EC0FFD1F72
:105F4000E75AF94F80819181D901A81BB90BCD0186
:105F5000B7FD0EC1069754F48091F402883C08F016
:105F600048C18091F402865F8093F402FE01EC0F39
:105F7000FD1FE75AF94F80819181AC01440F551FF5
:105F8000480F591F420F531F57FD35C17A01F59431
:105F9000E794F594E794C90101968E159F050CF0DE
:105FA00015C10894E108F1088091F402833C08F4DB
:105FB00005C18E010C0F1D1FF801E75AF94F8081B2
:105FC0009181F701E81BF90BCF0163E070E00E94BB
:105FD000DB76CB01880F991F860F971F0357194F48
:105FE000D80111969C938E93FE01EC0FFD1FE75A8A
:105FF000F94FF182E082FE013196F0935402E09372
:106000005302E530F10509F4B9C05D98E630F105B9
:1060100009F4BFC05C98379709F4B9C05B98F1C028
:106020005C9A5B98C43108F054C0CF5FC093BF0244
:10603000E8C09091580680915002981709F0E9CE77
:106040004091C0024B3008F49BC01092780110922E
:10605000BF023AC0C091BF02EC2FFF27EE0FFF1F17
:106060009F0125573D4FDF01A75AB94F8D919C9154
:10607000D9018D939C93DF01A357B94F8D919C91CA
:10608000EB55FD4F91838083EC2FFF27EE0FFF1F11
:106090009F01275A394FDF01A95ABD4F8D919C911D
:1060A000D90111969C938E93DF01AF58BD4F8D910E
:1060B0009C91E357F94F91838083EC2FEF5FED3094
:1060C00008F05EC0E093BF024F3120F6C091BF02DE
:1060D000DBCFC43109F095C0809102018A3009F408
:1060E0007FC0843109F47CC028988EE18093BF0280
:1060F0002CE0CDE8D6E0ABE8B2E0E9E5F6E08D9142
:106100009D91918380833296198218822296215024
:1061100027FFF5CF76C01092C00283CE289A8ACE90
:10612000809102018A3011F1843101F12898C53043
:1061300019F15D98C63009F473CF5C98C73009F047
:1061400070CF5B9A72CF8091C0028A3108F44AC046
:106150008091F402865F8093F4028091F402893C7E
:1061600008F493CE88EC8093F4028FCE289ADFCF88
:10617000909581959F4FEECE5D9ADFCF5D9A46CF89
:106180004F3F09F457CE4F5F4093C00253CE5B9A06
:1061900038C05C9A40CFEC2FFF27EE0FFF1FEF585F
:1061A000FD4F11821082AFCE41505040E416F506EB
:1061B0000CF08ACE0894E11CF11C86CEFE01EC0F97
:1061C000FD1FE357F94F118210820ECF215030404E
:1061D000E216F3060CF0E8CE0894E11CF11CE4CEC4
:1061E000289A83CF8B3008F4B8CF8091F4028E5F69
:1061F000B2CF88ECB9CE4D5F5F4FC8CE2D5F3F4F19
:1062000055CEFF91EF91DF91CF91BF91AF919F91CB
:106210008F917F916F915F914F913F912F911F913E
:106220000F91FF90EF900F900FBE0F901F90189559
:1062300081E08093CA0682E08093C90683E0809360
:10624000C80684E08093CB0685E08093CC0686E088
:106250008093CD0687E08093CE0688E08093CF06BA
:1062600089E08093D0068AE08093D1068BE080930A
:10627000D2068CE08093D30608951F938AE680931C
:10628000D40661E0609327075EE15093D5068FEF57
:106290008093D7068AE08093D8065093D606509311
:1062A000DA0685E08093DB0680E48093DC061092BA
:1062B000DD0684E18093D9068EE08093DE06F0E16E
:1062C000F093DF061CE01093E006A8E0A093E1063F
:1062D00086EE8093E2065093E30680E88093E4061E
:1062E00040E54093E50696E99093E60683E08093C7
:1062F000E7064093E8069093E90681E28093EA0678
:1063000083E28093EB065093EC0670E27093EE0606
:106310001092EF061092F0061092F1061092F2061B
:1063200010920A0710920B0710920C0710920D079B
:1063300024E62093F30638E23093F40660932607B0
:106340001092F50697EF9093F606E6E0E093FB06D1
:106350008DE78093FC068093FD068093FE062093D4
:10636000F7063093F8061092F9069093FA0682E346
:106370008093FF069AE5909300078093010710929F
:10638000250790930207409303076093040785E570
:106390008093050780930607F0930707709308071B
:1063A000209309078FE580930E0783EF80931007F2
:1063B0008AEA80931207809313078FE080930F0778
:1063C000809311078EEF8093140720931507909305
:1063D000160790931707909318078BE4809319077B
:1063E00080931A0780931B0710921C07E0931D07E8
:1063F000A0931E0790931F07509320072093210717
:106400002093220784E0809323076093ED06A6EA99
:10641000B1E0E8E2F7E00D9001921A95E1F71F91E3
:1064200008958AE68093D406E1E0E09327076EE1C1
:106430006093D5068FEF8093D7069AE09093D806A5
:106440006093D6066093DA0685E08093DB0680E4ED
:106450008093DC061092DD068FE08093D90690933E
:10646000DE0680E18093DF0676E07093E006F8E0D8
:10647000F093E10686EE8093E2066093E30680E8FF
:106480008093E4062AE52093E50698E79093E606D4
:1064900083E08093E7062093E8069093E90681E283
:1064A0008093EA0683E28093EB066093EC0650E269
:1064B0005093EE061092EF061092F0061092F1063D
:1064C0001092F20610920A0710920B0710920C0716
:1064D00010920D0744E64093F30638E23093F40639
:1064E000E09326071092F50697EF9093F6067093C7
:1064F000FB068DE78093FC068093FD068093FE06E5
:106500004093F7063093F8061092F9069093FA0636
:1065100082E38093FF062093000780930107109287
:1065200025072093020780E5809303078CE380937F
:10653000040785E5809305078093060750930707B6
:10654000509308079BE4909309078FE580930E070B
:1065500083EF809310078AEA8093120780931307D2
:1065600084E180930F07809311078EEF80931407C7
:1065700040931507209316072093170720931807B9
:106580009093190790931A0790931B0710921C077A
:1065900070931D07F0931E0720931F076093200739
:1065A000409321074093220784E080932307E093E0
:1065B000ED068CE0ADEAB1E0E8E2F7E00D90019283
:1065C0008A95E1F708958AE68093D40671E0709386
:1065D00027074EE14093D5068FEF8093D7068AE0D8
:1065E0008093D8064093D6064093DA0685E08093E0
:1065F000DB0680E48093DC061092DD068FE080935A
:10660000D90668E06093DE0620E12093DF0656E0BD
:106610005093E0066093E10686EE8093E206409395
:10662000E30680E88093E40634E63093E50698E7D5
:106630009093E60683E08093E7063093E806909314
:10664000E90681E28093EA0683E28093EB0684E127
:106650008093EC062093EE061092EF061092F0065F
:106660001092F1061092F20610920A0710920B0790
:1066700010920C0710920D073093F30628E2209336
:10668000F406709326071092F50697EF9093F6069E
:106690005093FB068DE78093FC068093FD06809364
:1066A000FE063093F7062093F8061092F9069093B1
:1066B000FA0692E39093FF062AE520930007909351
:1066C0000107109225072093020780E580930307B6
:1066D00086E48093040785E5809305078093060789
:1066E00080E28093070780930807909309078FE55E
:1066F00080930E0783EF809310078AEA8093120736
:106700008093130740930F07409311078EEF8093F8
:10671000140730931507209316072093170720932B
:1067200018078BE48093190780931A0780931B073F
:1067300010921C0750931D0760931E0720931F079C
:1067400040932007309321073093220784E0809301
:1067500023077093ED068CE0A5EBB1E0E8E2F7E0EB
:106760000D9001928A95E1F708956817790744F42E
:10677000680F791F77FD09C0CB019595879508951E
:10678000681B790B861B970B08956F5F7F4FCB01BA
:10679000959587950895EF92FF920F931F93CF934E
:1067A000C82F8B018091EA028823A9F4C150CF3F02
:1067B00091F07B01E60EF71E109303020093020294
:1067C0008091020290910302892BD1F7C7010E94A8
:1067D0002B18C15088F7CF911F910F91FF90EF9028
:1067E0000895ADE3B0E0E7EFF3E30C942B7720914D
:1067F0005403309155038091250290912602281B65
:10680000390B3A872987309389072093880720918D
:106810002F023091300237FDBFC73595279535954A
:106820002795359527953FA32EA33C872B87790184
:1068300020912D0230912E0237FDABC7359527955B
:1068400035952795359527953CA32BA33E872D8716
:10685000F0925307E092520730934907209348077C
:106860008091830790918407AA2797FDA095BA2F5E
:106870007C018D01EE0CFF1C001F111FE80EF91E9C
:106880000A1F1B1F80912102909122029C01442724
:1068900037FD4095542FDA01C901880F991FAA1FAF
:1068A000BB1F880F991FAA1FBB1F820F931FA41F16
:1068B000B51F820F931FA41FB51FE80EF91E0A1FF4
:1068C0001B1F17FD8BC715950795F794E794159532
:1068D0000795F794E794F0928407E09283078091FC
:1068E000930790919407AA2797FDA095BA2F7C0152
:1068F0008D01EE0CFF1C001F111FE80EF91E0A1F70
:106900001B1F80912302909124029C01442737FD94
:106910004095542FDA01C901880F991FAA1FBB1F88
:10692000880F991FAA1FBB1F820F931FA41FB51F9B
:10693000820F931FA41FB51FE80EF91E0A1F1B1F0D
:1069400017FD43C715950795F794E7941595079597
:10695000F794E794F0929407E092930780915007A0
:1069600090915107AA2797FDA095BA2F9C01AD01E0
:10697000220F331F441F551F280F391F4A1F5B1F4B
:1069800080911F0290912002AA2797FDA095BA2F0F
:10699000280F391F4A1F5B1F57FD12C75595479592
:1069A00037952795559547953795279530935107F6
:1069B000209350072091210230912202C901880FB3
:1069C000991F880F991F820F931F820F931FAA2769
:1069D00097FDA095BA2F209130033091310340915B
:1069E000320350913303820F931FA41FB51F80936E
:1069F000300390933103A0933203B093330320917B
:106A0000230230912402C901880F991F880F991F12
:106A1000820F931F820F931FAA2797FDA095BA2F6D
:106A200020912C0330912D0340912E0350912F0380
:106A3000820F931FA41FB51F80932C0390932D03E7
:106A4000A0932E03B0932F0380915C0790915D0774
:106A50002091210230912202820F931F90935D07B3
:106A600080935C0780918B0790918C072091230283
:106A700030912402820F931F90938C0780938B0791
:106A800080914A0390914B03019690934B0380931E
:106A90004A038091280390912903A0912A03B09181
:106AA0002B03BC01CD010E9422765B016C01809119
:106AB0001B0690911C06AA2797FDA095BA2FBC0132
:106AC000CD010E9422767B018C018091460390913A
:106AD0004703A0914803B09149039C01AD01C8014F
:106AE000B7010E94C275DC01CB019C01AD01C6015A
:106AF000B5010E94C375DC01CB01BC01CD010E9430
:106B00000576DC01CB018093280390932903A093A1
:106B10002A03B0932B038FEC80937A001092170115
:106B2000209018033090190340901A0350901B03D3
:106B300039E423163BE6330631E0430630E05306E2
:106B40000CF4AEC188E49BE6A1E0B0E08D839E83A7
:106B5000AF83B88760902003709021038090220358
:106B60009090230339E463163BE6730631E0830615
:106B700030E093060CF40FC588E49BE6A1E0B0E09A
:106B800089839A83AB83BC8349855A85CA01AA2726
:106B900097FDA095BA2F20911003309111034091D9
:106BA000120350911303280F391F4A1F5B1F28A798
:106BB00039A74AA75BA7A0908F07B0909007C09015
:106BC0009107D0909207A80EB91ECA1EDB1E86013F
:106BD00075013091DD023CA7332309F074C1809127
:106BE000DC02882309F0F5C44091D4064DA746FF86
:106BF000FEC5EBA1FCA1CF01AA2797FDA095BA2F56
:106C0000BC01CD0129813A814B815C810E949C7637
:106C10009B01AC0197FD59C6BBE05595479537954B
:106C20002795BA95D1F780918601E82EFF24002799
:106C30001127C801B7010E949C7697FD68C6ACE099
:106C40009595879577956795AA95D1F76F87788BF6
:106C5000898B9A8B609364037093650380936603BA
:106C6000909367032EA13FA1C901AA2797FDA09584
:106C7000BA2FBC01CD012D813E814F8158850E94E4
:106C80009C769B01AC0197FD3DC6FBE05595479571
:106C900037952795FA95D1F7C801B7010E949C76E0
:106CA00097FD2BC6DC01CB01ECE0B595A795979538
:106CB0008795EA95D1F78093680390936903A09331
:106CC0006A03B0936B0320916403309165033093A2
:106CD000C2062093C1062091680330916903309366
:106CE000C6062093C5062F85388949895A89821B93
:106CF000930BA40BB50B8AAF9BAFACAFBDAF80932A
:106D0000680390936903A0936A03B0936B03A80E82
:106D1000B91ECA1EDB1E86017501309185013DA397
:106D2000332309F08EC58EA79FA7A8ABB9ABB7FDDB
:106D300000C62EA53FA548A959A955954795379551
:106D4000279588A599A5AAA5BBA5821B930BA40B83
:106D5000B50B88A799A7AAA7BBA780931003909308
:106D60001103A0931203B093130389859A85AA2770
:106D700097FDA095BA2F2AAD3BAD4CAD5DAD820F0E
:106D8000931FA41FB51F8B8B9C8BAD8BBE8BBC013F
:106D9000CD0129813A814B815C810E949C769B01C7
:106DA000AC0197FD8DC56BE05595479537952795B7
:106DB0006A95D1F760918701862F9927AA27BB276B
:106DC0008F8B988FA98FBA8FBC01CD010E949C76C2
:106DD00097FD71C52CE095958795779567952A95D0
:106DE000D1F76B8F7C8F8D8F9E8F60935C03709338
:106DF0005D0380935E0390935F036B897C898D892B
:106E00009E892D813E814F8158850E949C769B01F1
:106E1000AC0197FD4BC58BE0559547953795279568
:106E20008A95D1F76F89788D898D9A8D0E949C768D
:106E300097FD37C5BCE09595879577956795BA9589
:106E4000D1F76AAB7BAB8CAB9DAB60936003709367
:106E50006103809362039093630329853A8537FD2C
:106E60001CC5213431050CF458C06B8D7C8D8D8D83
:106E70009E8D97FD56C5613871058105910564F4B5
:106E80006AA97BA98CA99DA997FD60C56138710588
:106E9000810591050CF441C081E0809300033DC061
:106EA00098EB291694E939069EEF49069FEF59069B
:106EB0000CF08AC328EB34E94EEF5FEF2D833E835D
:106EC0004F83588747CE28A539A54AA55BA52093AF
:106ED0001003309311034093120350931303309126
:106EE000D4063DA71092C6061092C5061092C2069F
:106EF0001092C10610926003109261031092620317
:106F00001092630310925C0310925D0310925E0373
:106F100010925F03309185013DA3809160039091B1
:106F20006103A0916203B0916303BC01CD0124E62B
:106F300030E040E050E00E941077DA01C901409152
:106F40005C0350915D03481B590B58A34F8F8091F0
:106F50005C0390915D03A0915E03B0915F03BC015F
:106F6000CD0124E630E040E050E00E941077DA01E5
:106F7000C9012091600330916103821B930B9AA396
:106F800089A380917E0190917F01A0918001B091B1
:106F90008101BC01CD0128E631E040E050E00E94D3
:106FA0009C76E616F7060807190744F057016801B2
:106FB000A61AB70AC80AD90A8601750117FDF3C3D4
:106FC000A0928F07B0929007C0929107D09292073B
:106FD0002BA13CA18F8D98A1280F391F7901002783
:106FE000F7FC0095102F8091140390911503A09148
:106FF0001603B0911703E80EF91E0A1F1B1F570155
:1070000068018091E0029091E102281B390BC901CF
:10701000AA2797FDA095BA2F280E391E4A1E5B1E7F
:1070200020919A0130919B0140919C0150919D01CA
:10703000221533054405550574F4A8EAEA2EA1E6A5
:10704000FA2E012D112DE21AF30A040B150B17016C
:1070500028015701680188279927DC01821B930BBF
:10706000A40BB50B281639064A065B060CF082C243
:10707000F8E52F2EFEE93F2EFFEF4F2EFFEF5F2E9C
:10708000220E331E441E551E2092180330921903FF
:1070900040921A0350921B03820171012092140343
:1070A0003092150340921603509217032EA13FA170
:1070B000A9A1BAA12A0F3B1FA901662757FD609518
:1070C000762F80911C0390911D03A0911E03B09117
:1070D0001F03480F591F6A1F7B1F5A016B018091C4
:1070E000DE029091DF02281B390BC901AA2797FD08
:1070F000A095BA2F680E791E8A1E9B1E80919E0154
:1071000090919F01A091A001B091A1018EAB9FAB86
:10711000A8AFB9AF86159705A805B90564F448EA84
:1071200051E660E070E0481B590B6A0B7B0B3A019B
:107130004B015A016B018EA99FA9A8ADB9ADB095BD
:10714000A095909581959F4FAF4FBF4F68167906D8
:107150008A069B060CF0FDC1E8E56E2EEEE97E2E58
:10716000EFEF8E2EEFEF9E2E2EA93FA948AD59AD21
:10717000620E731E841E951E60922003709221037E
:107180008092220390922303B401A30160921C0316
:1071900070921D0380921E0390921F0388A599A5EB
:1071A000AAA5BBA58093240390932503A09326034F
:1071B000B093270360924003709241038092420390
:1071C00090924303209238033092390340923A035D
:1071D00050923B0340933C0350933D0360933E0326
:1071E00070933F03E0923403F0923503009336032B
:1071F00010933703809123019091240197FDD1C210
:107200007C01F594E794F594E794F594E794FFA254
:10721000EEA2809121019091220197FDC0C28C01C4
:107220001595079515950795159507951CA30BA31F
:107230008091290290912A020F9734F458E1E52EAB
:107240005CEFF52EFFA2EEA28091290290912A0216
:10725000079734F440E3E42E48EFF42EFFA2EEA2A9
:10726000209102012A3009F4D2C180912902909123
:107270002A02815D97400CF0A0C180912902909173
:107280002A02805E974034F080EDE82E87E0F82EE9
:10729000FFA2EEA280912702909128020F9724F47A
:1072A00008E11CEF1CA30BA38091270290912802F8
:1072B000079724F400E318EF1CA30BA32A3009F46A
:1072C000BCC18091270290912802815D974024F0F3
:1072D00008EE13E01CA30BA38091270290912802D3
:1072E000805E974024F000ED17E01CA30BA3A09153
:1072F0009101AA2309F497C06091230170912401A0
:1073000080916C0390916D03681B790B2091230190
:1073100030912401280F391F37FD90C235952795EC
:1073200030936D0320936C03613871050CF4A1C197
:1073300060E870E070937303609372038A2F99275B
:10734000869FF001879FF00D969FF00D1124CF01CD
:10735000F7FD72C27C01F594E794F594E794F594F7
:10736000E794F594E7942EA13FA1E20EF31EFFA24D
:10737000EEA2409121015091220180916E039091E3
:107380006F03481B590B2091210130912201280FD6
:10739000391F37FD4EC23595279530936F032093E3
:1073A0006E03413851050CF45CC140E850E0509345
:1073B0007103409370038A2F9927849FD001859F82
:1073C000B00D949FB00D1124AD019D01B7FD2EC2EB
:1073D00089011595079515950795159507951595A7
:1073E0000795EBA1FCA10E0F1F1F1CA30BA3869FEB
:1073F0009001879F300D969F300D1124C901209177
:10740000230130912401820F931F909324018093D4
:1074100023018091210190912201480F591F50931F
:107420002201409321014D855E85141615060CF04E
:1074300028C18091C1069091C20697FDF3C1AA2789
:1074400097FDA095BA2F6DA1262F332744275527E6
:10745000BC01CD010E949C7697FDDFC1F6E09595B9
:10746000879577956795FA95D1F7AF8DB8A1A60F57
:10747000B71FB0934407A09343074B855C85141650
:1074800015060CF028C18091C5069091C60697FD9F
:10749000C0C1AA2797FDA095BA2F6DA1262F33272B
:1074A00044275527BC01CD010E949C7697FDACC1B5
:1074B00056E095958795779567955A95D1F7A9A147
:1074C000BAA1A60FB71FB0933907A09338073DA5FF
:1074D00037FD28C11093370700933607F09246070F
:1074E000E0924507A5EFB2E06CEC76E057E0FB01D7
:1074F0008191BF01E82FFF27EE0FFF1FE75AF94FD9
:107500000190F081E02DE259FF4FEF3FF10509F0C6
:107510000CF474C0EFEFF0E04C91242F33272E17BA
:107520003F0709F41BC2CF01821B930B97FD6DC06F
:10753000959587959595879595958795242F280FEF
:10754000822F9927E817F9070CF05DC021502C9382
:1075500005C26092200370922103809222039092D0
:107560002303A0921C03B0921D03C0921E03D0926D
:107570001F0314CE209218033092190340921A036D
:1075800050921B03A0921403B0921503C0921603ED
:10759000D09217038BCD98EB691694E979069EEF8C
:1075A00089069FEF99062CF528EB34E94EEF5FEF43
:1075B00029833A834B835C83E7CA98EEE92E93E0F4
:1075C000F92EFFA2EEA259CE2D823E824F8258861E
:1075D000C1CA88A599A5AAA5BBA5809310039093BD
:1075E0001103A0931203B09313039091D4069DA7A7
:1075F00079CC69827A828B829C82C6CAF7FF8CCF53
:10760000E0E0F0E089CF2F5FA2CF079691CF809185
:10761000290290912A02835F934034F038EEE32EE2
:1076200033E0F32EFFA2EEA28091290290912A026C
:107630008A5F93400CF42ECE27CE80912702909142
:107640002802835F934024F008EE13E01CA30BA3F1
:1076500080912702909128028A5F93400CF447CED4
:1076600042CE3FEF403853070CF0A1CE40E85FEF29
:107670009ECE8FEF603878070CF05CCE60E87FEF2D
:1076800059CE8091C1069091C20697FDE7C0AA2706
:1076900097FDA095BA2FEDA12E2F3327442755270C
:1076A000BC01CD010E949C7697FDF2C0E6E0959565
:1076B000879577956795EA95D1F72F8D38A1261B89
:1076C000370B30934407209343074B855C85141692
:1076D00015060CF4D8CE8091C5069091C60697FD8C
:1076E000C1C0AA2797FDA095BA2FEDA12E2F332751
:1076F00044275527BC01CD010E949C7697FDC3C04D
:1077000046E095958795779567954A95D1F729A194
:107710003AA1261B370B30933907209338073DA534
:1077200037FFD8CE4CA5442309F0D4CE8091DC029B
:10773000882309F0CFCE8B859C85A1E081309A0704
:107740000CF094C02B853C854FEF203034070CF0B3
:10775000E3C08EA19FA1280F391F3C872B872050A3
:107760003F4F3093460720934507AD85BE85E1E046
:10777000A130BE070CF4AEC02BA13CA1A20FB31FD9
:10778000BE87AD87A050B140B0933707A0933607AE
:10779000A9CE295F3F4F52C8295F3F4F3EC8079689
:1077A0003ECD07962DCDE60EF71E081F191FE0925D
:1077B0008F07F0929007009391071093920708CCDF
:1077C0002D5F3F4F4F4F5F4FE9C823E030E040E06F
:1077D00050E0E20EF31E041F151FB4C883E090E0D2
:1077E000A0E0B0E0E80EF91E0A1F1B1F6CC828A518
:1077F00039A54AA55BA5209310033093110340934C
:107800001203509313036ECB615C7F4F8F4F9F4FDA
:107810004FCE909581959F4F3CCE615C7F4F8F4FAF
:107820009F4F1CCE909581959F4F09CE215F3F4F72
:10783000CFCD2F5F3F4FAFCD0F968CCD2F5F3F4FFA
:107840006DCD28A539A54AA55BA5209310033093DB
:107850001103409312035093130387CA90958195A7
:107860009F4F15CF909581959F4F3BCFEEA1FFA1E4
:107870008E0F9F1F9C878B87805091409093460767
:107880008093450772CF615C7F4F8F4F9F4F38CFFA
:10789000615C7F4F8F4F9F4F09CF309521953F4FB0
:1078A000E0CA6150704F8F4F9F4FC4CA2150384F6C
:1078B0004F4F5F4FB0CA6150704F8F4F9F4F8ACA72
:1078C0002150384F4F4F5F4F6ECA2150384F4F4FA6
:1078D0005F4FA2C94D855E856FEF403056078CF52E
:1078E0008BA19CA1480F591F5E874D8740505F4F69
:1078F0005093370740933607F5CD6150704F8F4F47
:107900009F4FD0C92150384F4F4F5F4FBEC9615074
:10791000704F8F4F9F4F93C9F0924607E0924507F3
:1079200024CF90958095709561957F4F8F4F9F4F95
:10793000A2CA0196A11DB11D8EA79FA7A8ABB9AB86
:10794000F8C91093370700933607CCCD90958095F2
:10795000709561957F4F8F4F9F4F98CA51501196E8
:1079600057FFC5CDE2E1C35C0C944777CF93DF931B
:10797000809102018D3009F491C010927A008091BB
:10798000290290912A02909346078093450780919F
:1079900027029091280290933707809336078091B1
:1079A0002502909126029093890780938807809101
:1079B0002102909122029C01442737FD4095542FCB
:1079C000DA01C901880F991FAA1FBB1F880F991FD1
:1079D000AA1FBB1F820F931FA41FB51F820F931FE7
:1079E000A41FB51F9093840780938307809123027F
:1079F000909124029C01442737FD4095542FDA01D1
:107A0000C901880F991FAA1FBB1F880F991FAA1FA2
:107A1000BB1F820F931FA41FB51F820F931FA41FAC
:107A2000B51F909394078093930780911F029091C4
:107A3000200290935107809350078FEC80937A0037
:107A4000A5EFB2E0CCECD6E037E08991E82FFF2734
:107A5000EE0FFF1FE75AF94F0190F081E02DE25938
:107A6000FF4F1E161F06BCF4EF3FF10514F0EFEFB9
:107A7000F0E02C91822F9927E817F9073CF4215068
:107A80002C933150119637FFE0CF0BC08E179F0714
:107A9000C4F72F5FF5CFE0E0F0E0EBCF0E94FC1CD5
:107AA0006CCF809105079927AA27BB27BC01CD0180
:107AB00024EC39E040E050E00E949C76DC01CB01F0
:107AC00080939E0190939F01A093A001B093A10188
:107AD000809106079927AA27BB27BC01CD010E94E8
:107AE0009C76DC01CB0180939A0190939B01A0933B
:107AF0009C01B0939D01DF91CF9108956F927F9289
:107B00008F929F92AF92BF92CF92DF92EF92FF92AD
:107B10000F931F93CF9300E010E078016801469A1D
:107B200010934F0300934E0310934D0300934C03A7
:107B300080E090E0A0E0B0E080934603909347039C
:107B4000A0934803B093490310935903009358033B
:107B50001093570300935603109355030093540357
:107B600010936407009363071092870110928601B7
:107B7000109219020E94B63C84E690E00E943818E8
:107B80000E94B63C8091D40680FF10C080911B01FA
:107B900090911C01875B934008F0D0C180911B013C
:107BA00090911C018E5E924008F4C8C1CFE18AE03A
:107BB00090E00E9438188091250290912602080FCB
:107BC000191F8091290290912A02E80EF91E8091D6
:107BD000270290912802C80ED91EC150C7FFE7CFD7
:107BE000A701405F5F4F569547955695479550932F
:107BF0005903409358039601205F3F4F36952795D0
:107C0000369527953093570320935603C801409625
:107C100096958795929582958F7089279F70892771
:107C20009093550380935403909364078093630764
:107C300030935303209352035093510340935003C6
:107C400044E050E0DA010E946877802D853008F426
:107C500078C1809193079091940797FDABC16CE038
:107C600070E00E94DB7670934D0360934C0380912B
:107C700083079091840797FD99C16CE070E00E94A2
:107C8000DB7670934F0360934E0380911B069091B7
:107C90001C06AA2797FDA095BA2FBC01CD010E9412
:107CA0002276DC01CB018093460390934703A09397
:107CB0004803B0934903109246071092450710926B
:107CC000370710923607109289071092880784E6CA
:107CD00090E00E9438188091210290912202AA27F8
:107CE00097FDA095BA2F9C01AD01220F331F441FB1
:107CF000551F220F331F441F551F280F391F4A1FBE
:107D00005B1F280F391F4A1F5B1F30938407209386
:107D100083078091230290912402AA2797FDA095C2
:107D2000BA2F7C018D01EE0CFF1C001F111FEE0C01
:107D3000FF1C001F111FE80EF91E0A1F1B1FE80E73
:107D4000F91E0A1F1B1FF0929407E092930780917F
:107D5000E306682E772488249924C9019C014427CE
:107D600037FD4095542FC401B3010E949C765B01FE
:107D70006C0160934003709341038093420390939E
:107D800043039701442737FD4095542FC401B301A5
:107D90000E949C76DC01CB018093380390933903D9
:107DA000A0933A03B0933B03A0921C03B0921D032F
:107DB000C0921E03D0921F03809314039093150367
:107DC000A0931603B093170310921003109211039F
:107DD000109212031092130380911D0190911E01C5
:107DE000A0911F01B091200190931E0680931D0663
:107DF00010921802109217021092080310920903B1
:107E000010920A0310920B038091060390910703CE
:107E100090930503809304030E94D86182E390E06D
:107E20009093030280930202809105079927AA2765
:107E3000BB27BC01CD0124EC39E040E050E00E94BA
:107E40009C76DC01CB018856954CAF4FBF4F809399
:107E50009E0190939F01A093A001B093A1018091F6
:107E600006079927AA27BB27BC01CD010E949C7653
:107E7000DC01CB018856954CAF4FBF4F80939A01E0
:107E800090939B01A0939C01B0939D01109283015C
:107E9000109282018091060390910703AA2797FD13
:107EA000A095BA2F20917E0130917F0140918001F1
:107EB00050918101BC01CD010E949C76DC01CB0177
:107EC00080938F0790939007A0939107B0939207A8
:107ED0001092FF021092FE0281E0809301010E9445
:107EE00022668091C30284608093C3028FEF8093E7
:107EF00000081092010880E28093020825EF32E02A
:107F0000ACECB6E0C7E08D91E82FFF27EE0FFF1F26
:107F1000E75AF94F808191818259F90181939F013C
:107F2000C150C7FFF0CF84E68093F4028091000235
:107F3000882309F443C0469A579A40C00E94A31C64
:107F400035CEDA010E946877802D9927982F8827EF
:107F5000DA0111960E946877202D820F911D90936F
:107F60004F0380934E03DA0112960E946877802DAA
:107F70009927982F8827DA0113960E946877202D79
:107F8000820F911D90934D0380934C03DA01149658
:107F90000E946877802D9927982F8827DA011596F7
:107FA0000E946877202D820F911D73CE9095819548
:107FB0009F4F63CE909581959F4F51CECF911F914A
:107FC0000F91FF90EF90DF90CF90BF90AF909F9078
:107FD0008F907F906F9008959091EA02992309F510
:107FE0008091C3028C7F8093C30214C0A92FBB274A
:107FF000FD01E159FB4F8083FD01EE0FFF1FEE0FE6
:10800000FF1FE85DF94FA159BB4F8C9180839F5FA3
:108010009C3068F48091E301882341F3A92FBB27AA
:10802000EBCF8091C30281608093C30209C080912D
:10803000E301882329F08091E30181508093E301DB
:108040008091280699279093F1058093F0058091FF
:108050002C0699279093F3058093F20580913006C2
:1080600099279093F5058093F4058091340699271C
:108070009093F7058093F60510924E0210924D02F0
:108080000E94FD2C08958091D606883F08F007C213
:10809000E82F882321F0843608F40DC284E680930B
:1080A00097018091D806883F08F0F0C1E82F882317
:1080B00021F0843608F4FCC184E680939501809118
:1080C000E506883F08F0D9C1E82F8B3008F0CFC112
:1080D0008AE08093900180910F07883F08F0BEC12D
:1080E000E82F823008F0B4C181E080935E07809170
:1080F0001107883F08F0A3C1E82F823008F099C12A
:1081000081E0809386078091FC06883F38F0EFEF8E
:10811000F0E0E81BF109EB50FD4F808180935B0795
:108120008091FD06883F38F0EFEFF0E0E81BF109A1
:10813000EB50FD4F80818093C7068091FE06883FFB
:1081400038F0EFEFF0E0E81BF109EB50FD4F8081D4
:10815000809365078091D706883F38F0EFEFF0E015
:10816000E81BF109EB50FD4F8081809396018091CF
:10817000DA06883F38F0EFEFF0E0E81BF109EB504A
:10818000FD4F8081809394018091DC06883F38F018
:10819000EFEFF0E0E81BF109EB50FD4F8081809399
:1081A00092018091E406883F38F0EFEFF0E0E81BA1
:1081B000F109EB50FD4F8081809393018091E60699
:1081C000883F38F0EFEFF0E0E81BF109EB50FD4F8E
:1081D000808180938F018091E706883F38F0EFEF30
:1081E000F0E0E81BF109EB50FD4F80818093910195
:1081F0008091E806883F38F0EFEFF0E0E81BF109E6
:10820000EB50FD4F808180938E018091E906883F7D
:1082100038F0EFEFF0E0E81BF109EB50FD4F808103
:1082200080938D012091EE06283F38F0EFEFF0E0CB
:10823000E21BF109EB50FD4F208120938B018091CF
:10824000EF06883F08F0EDC0482F4093D702809199
:10825000F006883F38F0EFEFF0E0E81BF109EB5053
:10826000FD4F80818093D6028091F106883F38F0DF
:10827000EFEFF0E0E81BF109EB50FD4F80818093B8
:10828000D5028091F206883F38F0EFEFF0E0E81B6E
:10829000F109EB50FD4F80818093D40280910A0751
:1082A000883F38F0EFEFF0E0E81BF109EB50FD4FAD
:1082B00080818093D30280910B07883F38F0EFEFE5
:1082C000F0E0E81BF109EB50FD4F80818093D20272
:1082D00080910C07883F38F0EFEFF0E0E81BF109E0
:1082E000EB50FD4F80818093D10280910D07883F34
:1082F00038F0EFEFF0E0E81BF109EB50FD4F808123
:108300008093D0028091F306883F38F0EFEFF0E0E1
:10831000E81BF109EB50FD4F808180938A01809129
:10832000F706883F38F0EFEFF0E0E81BF109EB507B
:10833000FD4F8081809389018091FF06883F38F04E
:10834000EFEFF0E0E81BF109EB50FD4F80818093E7
:10835000880180910207883F38F0EFEFF0E0E81BDA
:10836000F109EB50FD4F80818093870180910307D5
:10837000883F38F0EFEFF0E0E81BF109EB50FD4FDC
:1083800080818093860180910407883F38F0EFEF69
:10839000F0E0E81BF109EB50FD4F808180938501EF
:1083A00080910907883F38F0EFEFF0E0E81BF10912
:1083B000EB50FD4F80818093840180912407883F9A
:1083C00038F0EFEFF0E0E81BF109EB50FD4F808152
:1083D0008093960733272F5F3F4F8CE398E2B901D4
:1083E0000E94DB7670939901609398018091E20678
:1083F000809387078091E10680934A07413009F412
:108400005DC0443009F45AC083E090E090937C0151
:1084100080937B0181E090E090937A0180937901D1
:108420000895EFEFF0E0E81BF109EB50FD4F4081BC
:108430000CCF8F3F09F465CEE093860764CEEFEF53
:10844000F0E0E81BF109EB50FD4FE0818E2F55CE97
:108450008F3F09F44ACEE0935E0749CEEFEFF0E09C
:10846000E81BF109EB50FD4FE0818E2F3ACE8F3F94
:1084700009F42FCEE09390012ECEEFEFF0E0E81B51
:10848000F109EB50FD4FE0818E2F1FCEEFEFF0E0B2
:10849000E81BF109EB50FD4FE0818E2F08CEEFEF86
:1084A000F0E0E81BF109EB50FD4FE0818E2FF1CD9C
:1084B000E093950104CEE0939701F3CD81E090E045
:1084C00090937C0180937B0183E090E090937A010C
:1084D000809379010895ACE3B0E0E1E7F2E40C9415
:1084E0002B770E94F133209102012C3008F0BAC2A0
:1084F000299AA090EB02B090EC02BA82A9828091F6
:108500004A0799270A96A816B90614F49A8389830C
:108510008091F402843608F0A7C280919003909174
:108520009103009709F0B6C41092EA028091C30249
:108530008F7E8093C3022A3009F4B4C4243109F435
:10854000B1C428988091C4029091C502895E93407D
:1085500008F4B1C48091EB06282F33273A8329838E
:108560008091C30280618093C3028091C806A82FC6
:10857000BB27AA0FBB1FFD01E357F94F11821082E1
:108580008091C906282F3327220F331FC901835733
:10859000994FFC0111821082A75AB94F11961C9273
:1085A0001E92275A394FD90111961C921E92809122
:1085B000CB06E82FFF27EE0FFF1FE75AF94F118276
:1085C00010828091780181508093780180917801A8
:1085D0008F3F21F08091C30284FF70C40E9443400A
:1085E00080919F039091A003AC01440F551F480F49
:1085F000591F0091C806A02FBB27AA0FBB1FFD0162
:10860000E75AF94FE090DE06CE2CDD24808191817F
:108610008C9D50018D9DB00C9C9DB00C11244A0D79
:108620005B1D57FF02C00C946C57559547955595A7
:108630004795A357B94F8091DF06682F77278D9113
:108640009C91869F9001879F300D969F300D11243D
:10865000240F351F3093A00320939F038091D603EE
:108660009091D7034091D2035091D303840F951F6B
:10867000281B390B3093F2022093F1028091A10361
:108680009091A203AC01440F551F480F591F109140
:10869000C906A12FBB27AA0FBB1FFD01E75AF94F3F
:1086A000808191818C9D90018D9D300D9C9D300D20
:1086B0001124420F531F57FF02C00C946857559561
:1086C000479555954795A357B94F8D919C91869F96
:1086D0009001879F300D969F300D1124240F351F78
:1086E0003093A2032093A1038091D4039091D503EA
:1086F0004091D0035091D103840F951F281B390B53
:108700003093F0022093EF028091CB06E82FFF27F1
:10871000EE0FFF1FE75AF94F808191819095819567
:108720009F4F8330910514F40C94364E029790932A
:10873000EE028093ED028091CA06E82FFF27EE0F2C
:10874000FF1FE75AF94FC080D18048E750E0C40EC0
:10875000D51E809190019927AA2797FDA095BA2F41
:10876000BC01CD010E942276DC01CB0120E030E08B
:1087700040E251E4BC01CD010E94C375DC01CB0194
:10878000BC01CD010E940576DC01CB0180938D07F1
:10879000F0908F0180918E019927AA2797FDA095CF
:1087A000BA2FBC01CD010E942276DC01CB0120E072
:1087B00030E040E251E4BC01CD010E94C375DC0110
:1087C000CB01BC01CD010E940576DC01CB01809379
:1087D0003D0750918D01509354078091910480FF83
:1087E00006C080919607813810F00C94994ED09273
:1087F000EC02C092EB028091EB029091EC0297FFA9
:1088000002C00C946257F091D406F9A3F2FD02C0A5
:108810000C94804E109266074091F1025091F20242
:10882000CA0157FF02C00C948B4E9595879595957C
:10883000879597FF02C00C94944E2091C802309106
:10884000C9022817390714F00C943E4ECA0157FF8D
:1088500002C00C94ED5A97FF02C00C94F25ABC016E
:1088600075956795759567956536710514F40C9443
:10887000414E64E670E04091EF025091F002CA016F
:1088800057FD02C00C944A4E039695958795959591
:10889000879597FD02C00C94524E909581959F4FFD
:1088A0002091C6023091C7022817390714F40C949E
:1088B0005B4E215030408091C30284FD02C00C9475
:1088C000764E1092C9021092C8021092C7021092FE
:1088D000C602E12FFF27EE0FFF1FE75AF94F409125
:1088E0000007242F3327808191812817390734F41A
:1088F0008091250782FF02C00C940D4FE12FFF27C6
:10890000EE0FFF1FE75AF94F842F99272091010797
:10891000821B9109208131812817390714F41092A4
:10892000DB02E12FFF27EE0FFF1FE75AF94F842FDD
:10893000992722273327281B390B808191818217A1
:10894000930734F48091250783FF02C00C94084FED
:108950008091DA02882391F0E12FFF27EE0FFF1FAD
:10896000E75AF94F809101079927841B91092081CB
:1089700031818217930714F40C94394FE02FFF27AD
:10898000EE0FFF1FE75AF94F242F33278081918183
:108990002817390734F48091250780FF02C00C9412
:1089A000024F5091D802552399F0E02FFF27EE0F88
:1089B000FF1FE75AF94F842F992720910107821B47
:1089C0009109208131812817390714F40C94344F10
:1089D000E02FFF27EE0FFF1FE75AF94F842F99274B
:1089E00022273327281B390B808191818217930717
:1089F00034F48091250781FF02C00C94FD4E8091D4
:108A0000D902882391F0E02FFF27EE0FFF1FE75ACE
:108A1000F94F809101079927841B910920813181A9
:108A20008217930714F40C943D4F8091DB02882346
:108A300031F48091DA02882311F40C94FA4E91E01B
:108A4000552331F48091D902882311F40C94184FE6
:108A500081E08093DD021092DC021092DB02109222
:108A6000DA022FC2299845CD8091F4028D3808F49E
:108A7000A8CD8091C3028F7E8093C3029091EC06B3
:108A800082E3989FC00111249093910380939003F7
:108A9000E981FA81B99714F00C941D4F8091C402BA
:108AA0009091C5028F3F910519F010F00C945B571F
:108AB000109274031092750310927603109277034C
:108AC000109278031092790310927A0310927B032C
:108AD0008A3F910511F40C944F5C3091CA06E32F44
:108AE000FF27EE0FFF1FE75AF94F808191818135F3
:108AF00091050CF409C14091EA02442309F004C134
:108B0000E0917B01F0917C01E853F94F8081E82FDF
:108B1000FF27EE0FFF1FE75AF94F808191818C34B8
:108B2000910514F40C948A5B809192038F5F893CC9
:108B300010F40C94AC5C2C3010F00C94FA5D299875
:108B40001092EA02109292031092C5021092C4028F
:108B50000091C806E02FFF27EE0FFF1FE75AF94FDD
:108B6000808191818734910514F00C94F45D4091DB
:108B7000790150917A01FA01E853F94F8081E82F89
:108B8000FF27EE0FFF1FE75AF94F80819181019077
:108B9000F081E02DF7FF02C00C940E61E734F1057F
:108BA0000CF482C021E0FA01E853F94F8081A82F2C
:108BB000BB27AA0FBB1FA75AB94F8D919C91119744
:108BC0008734910544F0E02FFF27EE0FFF1FE75A8F
:108BD000F94F808191818D919C918734910564F04A
:108BE000E02FFF27EE0FFF1FE75AF94F8081918199
:108BF000873491050CF022E0FA01E853F94F8081A7
:108C0000E82FFF27EE0FFF1FE75AF94F8081918170
:108C10008634910564F4E02FFF27EE0FFF1FE75A1B
:108C2000F94F80819181873491050CF023E0FA019E
:108C3000E853F94F8081E82FFF27EE0FFF1FE75A17
:108C4000F94F808191818A5B9F4F64F4E02FFF2769
:108C5000EE0FFF1FE75AF94F80819181873491050C
:108C60000CF024E04853594FDA018C91E82FFF278C
:108C7000EE0FFF1FE75AF94F808191818A5B9F4F6A
:108C800064F4E02FFF27EE0FFF1FE75AF94F8081B2
:108C90009181863491050CF425E0822F0E945F07B4
:108CA0004091790150917A014853594FFA018081DE
:108CB000E82FFF27EE0FFF1FE75AF94F80819181C0
:108CC0008081918197FF02C00C941D604E9714F033
:108CD0000C94A85D8091C806E82FFF27EE0FFF1FB8
:108CE000E75AF94F808191818A5B9F4F14F00C9471
:108CF000A85D81E08093850488EE93E09093030261
:108D0000809302023091CA06E32FFF27EE0FFF1F68
:108D1000E75AF94F808191818B5A9F4F0CF051CCCB
:108D20002091EA02222311F00C947E58E0917B01FD
:108D3000F0917C01E853F94F8081E82FFF27EE0F77
:108D4000FF1FE75AF94F80819181855B9F4F14F097
:108D50000C94725B8091D602882341F08091C1020D
:108D60009091C202019711F00C94725B8091930371
:108D70008F5F893C10F40C94A45D2093930381E0F1
:108D800090E09093C5028093C40281E08093EA0250
:108D900010927C0310927D0310927E0310927F0349
:108DA00010921003109211031092120310921303E9
:108DB00010920C0310920D0310920E0310920F03E9
:108DC0008091E306E82EFF24002711278091830776
:108DD000909184079C01442737FD4095542FC8018A
:108DE000B7010E949C76DC01CB0180932003909315
:108DF0002103A0932203B0932303809193079091C2
:108E000094079C01442737FD4095542FC801B701B2
:108E10000E949C76DC01CB01809318039093190388
:108E2000A0931A03B0931B038091400390914103D8
:108E3000A0914203B091430380931C0390931D03C0
:108E4000A0931E03B0931F038091380390913903C0
:108E5000A0913A03B0913B038093140390931503C0
:108E6000A0931603B0931703109274031092750326
:108E70001092760310927703109278031092790380
:108E800010927A0310927B038091C30288608093D2
:108E9000C30297CB019790939103809390032A305C
:108EA00009F04CCB289A8091C4029091C502895E4A
:108EB000934008F04FCB1092EA0283CBA090D406E7
:108EC000A9A20091DC020A8F002321F48091DD0227
:108ED000882369F08091FF06992729813A818217BA
:108EE000930714F49A83898381E08093000380912F
:108EF000C30284FFB7C61092EE021092ED021092E8
:108F0000F2021092F1021092F0021092EF029AE532
:108F100090938D0788E78093660790933D078C8731
:108F2000809354071092DC021092DD021A8E209179
:108F30005707309158074091590750915A0760914F
:108F400040037091410380914203909143036E8BE3
:108F50007F8B888F998F260F371F481F591F80914D
:108F60005F0790916007A0916107B0916207A090A0
:108F70003803B0903903C0903A03D0903B03AE86DB
:108F8000BF86C88AD98A8A0D9B1DAC1DBD1DC090A5
:108F90004C07D0904D07E0904E07F0904F07CFA6BA
:108FA000D8AAE9AAFAAAE0903C03F0903D03009108
:108FB0003E0310913F03EA8AFB8A0C8B1D8BAFA402
:108FC000B8A8C9A8DAA8AE0CBF1CC01ED11EAFA697
:108FD000B8AAC9AADAAAC0903E07D0903F07E0908D
:108FE0004007F0904107CBA6DCA6EDA6FEA6E090D8
:108FF0003403F09035030091360310913703EBA250
:10900000FCA20DA31EA3ABA4BCA4CDA4DEA4AE0CF5
:10901000BF1CC01ED11EABA6BCA6CDA6DEA6B090BE
:10902000DD02BB8EBB2009F0BCC50A8D002309F010
:10903000B8C580935F0790936007A0936107B093D2
:10904000620720935707309358074093590750936E
:109050005A0780911B0690911C06815092400CF09B
:109060006AC48091EA02882309F065C480911502E0
:10907000909116028F3F910509F008F46BC5BB8DE6
:10908000BB2309F003C7EA8DEE2309F0FFC6F09178
:109090000003FD87FF2309F0F9C6A0900807AAA2E4
:1090A000AA2009F4F3C6CFA4D8A8E9A8FAA8C092C8
:1090B0004C07D0924D07E0924E07F0924F07EBA479
:1090C000FCA40DA51EA5E0923E07F0923F07009379
:1090D0004007109341078091570790915807A0913E
:1090E0005907B0915A07B7FF02C00C949D5F292E13
:1090F0003A2E4B2E552447FC5A9420925707309213
:1091000058074092590750925A0780915F079091F3
:109110006007A0916107B0916207B7FF02C00C948D
:10912000975F892F9A2FAB2FBB27A7FDBA958C830A
:109130009D83AE83BF8380935F0790936007A09366
:109140006107B09362078091E306E82EFF240027B1
:109150001127209130033091310340913203509117
:109160003303C801B7010E949C7697FF02C00C949C
:10917000915F672E782E892E992487FC9A942091EE
:109180002C0330912D0340912E0350912F03C801E1
:10919000B7010E949C7697FF02C00C948B5FA72EAC
:1091A000B82EC92EDD24C7FCDA94D201C10186197C
:1091B0009709A809B90920910707E22EFF24002783
:1091C0001127BC01CD01A80197010E941077390138
:1091D0004A012FA338A749A75AA78C819D81AE8148
:1091E000BF818A199B09AC09BD09BC01CD01A80149
:1091F00097010E941077D401C30197FE02C00C941E
:10920000775F892F9A2FAB2FBB27A7FDBA95BC019B
:10921000DA01C90157FF02C00C94715F892F9A2FA0
:10922000AB2FBB27A7FDBA952C018091C802909166
:10923000C90281349105D4F48091C6029091C7028D
:10924000813491059CF48091CB06E82FFF27EE0F27
:10925000FF1FE75AF94F808191810190F081E02D45
:10926000F7FF02C00C9416617A9734F080910008E1
:109270008F3F11F40C94FD5DEA88FB880C891D89F1
:109280002E893F89488D598DE21AF30A040B150B7C
:10929000E0928003F0928103009382031093830392
:1092A0008BA19CA1ADA1BEA1AE84BF84C888D98882
:1092B0008A199B09AC09BD0988879987AA87BB874A
:1092C0008093840390938503A0938603B0938703D0
:1092D000E0928803F092890300938A0310938B0332
:1092E00080938C0390938D03A0938E03B0938F0390
:1092F00080911C0390911D03A0911E03B0911F0348
:109300008E199F09A00BB10B80931C0390931D0332
:10931000A0931E03B0931F03809114039091150333
:10932000A0911603B0911703288539854A855B857E
:10933000821B930BA40BB50B80931403909315031E
:10934000A0931603B09317033AA1332371F1209130
:10935000FE023091FF022138310594F080915403D0
:1093600090915503019690935503809354038091F7
:109370006307909164070196909364078093630755
:1093800020583F4F94F480915403909155030197D6
:1093900090935503809354038091630790916407E1
:1093A000019790936407809363071092FF021092D5
:1093B000FE0291E0292E312CD801C70117FF02C00F
:1093C0000C94825F81509240A040B0401CF084E039
:1093D000282E312C8091A9039091AA03A091AB0370
:1093E000B091AC03A0905707B0905807C0905907B0
:1093F000D0905A078A199B09AC09BD09815E914B2F
:10940000AF4FBF4F8F539C49A040B04010F40C9415
:10941000865CF0910108F8A3F93114F40C94DA5D3C
:109420003092A4032092A30331E0E31630E1F30667
:1094300030E0030730E0130714F40C94B45C80911F
:10944000A503882311F40C947D5F7093DF02609371
:10945000DE02D801C70117FF02C00C946A619C01AB
:10946000AD01B7FF02C00C943F61B9E05595479537
:1094700037952795BA95D1F78091A3039091A403CE
:10948000820F931F9093A4038093A303A8019701D5
:1094900017FF02C00C94396139014A01A3E0959489
:1094A000879477946794AA95D1F76FA278A689A636
:1094B0009AA649E8641643E1740640E0840640E059
:1094C000940654F0F8E86F2EF3E17F2E812C912C56
:1094D0006FA278A689A69AA6D401C30197FE02C0FE
:1094E0000C944961892F9A2FAB2FBB27A7FDBA9502
:1094F000680F791F50E0E51650EFF5065FEF05079E
:109500005FEF150714F00C94945D8091A6038823F7
:1095100011F40C94605F7093DF026093DE02D80157
:10952000C70117FF02C00C9424619C01AD01B7FF75
:1095300002C00C94336169E055954795379527959E
:109540006A95D1F78091A3039091A403820F931F92
:109550009093A4038093A303A801970117FF02C06F
:109560000C942D6139014A0143E0959487947794D6
:1095700067944A95D1F768E766166CEE76066FEF4A
:1095800086066FEF960644F438E7632E3CEE732EA2
:109590003FEF832E3FEF932E6092970370929803D4
:1095A0008092990390929A03D401C30197FE02C05E
:1095B0000C94F660892F9A2FAB2FBB27A7FDBA9585
:1095C0006091DE027091DF02680F791F4AA1242F9B
:1095D00033278091A3039091A4032817390724F41B
:1095E0003093A4032093A30358A1552379F0252F8A
:1095F000332727FD30958091A3039091A40328176A
:10960000390724F43093A4032093A30381E8E816D8
:10961000F1040105110574F08091580390915903EC
:109620002091A3033091A403820F931F90935903B9
:109630008093580390E8E9169FEFF9069FEF09071A
:109640009FEF190774F4809158039091590320916A
:10965000A3033091A403821B930B9093590380932F
:109660005803B1E02B2E312C88859985AA85BB85BE
:10967000B7FF02C00C944A5F81509240A040B040B6
:109680001CF0A4E02A2E312C20E030E040E050E035
:109690008091AD039091AE03A091AF03B091B00360
:1096A000E0905F07F09060070091610710916207FA
:1096B0008E199F09A00BB10B815E914BAF4FBF4F2D
:1096C0008F539C49A040B04028F088A1893114F400
:1096D0000C94135E3092A4032092A303888599858D
:1096E000AA85BB8581509041A040B04014F40C94F1
:1096F000885D8091A703882311F40C94535F5092E6
:10970000E1024092E00288859985AA85BB85B7FF72
:1097100002C00C941B61B7FF02C00C940861F9E011
:10972000B595A79597958795FA95D1F7280E391E87
:109730003092A4032092A303288539854A855B854E
:1097400057FF02C00C940261E3E0559547953795A9
:109750002795EA95D1F72938F3E13F07F0E04F0765
:10976000F0E05F0714F40C94C96088E893E1A0E08E
:10977000B0E080939B0390939C03A0939D03B093D0
:109780009E0380919B0390919C03A0919D03B091B7
:109790009E03B7FF02C00C947361892F9A2FAB2FE1
:1097A000BB27A7FDBA954090E0025090E102480E19
:1097B000591E288539854A855B85203080EF38071A
:1097C0008FEF48078FEF580714F00C94B05C80912E
:1097D000A803882311F40C94E05F5092E1024092B8
:1097E000E002DA01C90157FF02C00C945B619C01E1
:1097F000AD01B7FF02C00C945561B9E0559547958E
:1098000037952795BA95D1F78091A3039091A4033A
:10981000820F931F9093A4038093A3032885398517
:109820004A855B8557FF02C00C944F61A3E05595B4
:10983000479537952795AA95D1F728379CEE390794
:109840009FEF49079FEF590714F00C94E76088E7F2
:109850009CEEAFEFBFEF80939B0390939C03A0938C
:109860009D03B0939E0380919B0390919C03A091D4
:109870009D03B0919E03B7FF02C00C946461892FD1
:109880009A2FAB2FBB27A7FDBA954090E0025090CE
:10989000E102480E591EAAA12A2F33278091A30363
:1098A0009091A4032817390724F43093A40320933C
:1098B000A303B8A1BB2379F02B2F332727FD3095C5
:1098C0008091A3039091A4032817390724F43093BF
:1098D000A4032093A303288539854A855B85213815
:1098E00031054105510574F080915603909157035D
:1098F0002091A3033091A403820F931F90935703E9
:109900008093560388859985AA85BB8580589F4F8B
:10991000AF4FBF4F0CF0D0C28091560390915703C8
:109920002091A3033091A403821B930B90935703C0
:1099300080935603C1C2909000086FEF961611F401
:109940000C9472578091E306A82EBB24CC24DD240E
:109950006E897F89888D998DA60195010E94107767
:1099600079018A018091830790918407AA2797FD46
:10997000A095BA2FE81AF90A0A0B1B0B6E857F8592
:1099800088899989A60195010E94107759016A0179
:109990008091930790919407AA2797FDA095BA2FDD
:1099A000A81AB90ACA0ADB0A292C332427FC3094E6
:1099B000432C532CC201B101A80197010E949C764F
:1099C00097FD5FC23B014C01F9E095948794779431
:1099D0006794FA95D1F7C201B101A60195010E94E1
:1099E0009C7697FF02C00C94465B5B016C01E9E03A
:1099F000D594C794B794A794EA95D1F78091C802FB
:109A00009091C902813491053CF48091C6029091F5
:109A1000C70281349105C4F0D401C30197FE02C08E
:109A20000C944A5C3C014D0195948794779467941B
:109A3000D601C501D7FE02C00C94455C5C016D01E6
:109A4000D594C794B794A7948091CB06E82FFF27AD
:109A5000EE0FFF1FE75AF94F808191810190F0814D
:109A6000E02DF7FF02C00C94415B7A97A4F0C4018B
:109A7000B30123E030E040E050E00E94107739016C
:109A80004A01C601B50123E030E040E050E00E9409
:109A9000107759016A0180910208282F332727FD8A
:109AA0003095432F532F261537054805590514F4D3
:109AB00039014A01992787FD9095909581959F4F8F
:109AC000AA2797FDA095BA2F681679068A069B06E5
:109AD00014F43C014D012A153B054C055D0514F4B9
:109AE00059016A01A816B906CA06DB0614F45C011E
:109AF0006D018091200390912103A0912203B091E8
:109B0000230386199709A809B90980932003909324
:109B10002103A0932203B093230380911803909113
:109B20001903A0911A03B0911B038A199B09AC0970
:109B3000BD098093180390931903A0931A03B0935F
:109B40001B0380911502909116028F3F910511F031
:109B500008F095CAAFA4B8A8C9A8DAA8A0924C0783
:109B6000B0924D07C0924E07D0924F07CBA4DCA411
:109B7000EDA4FEA4C0923E07D0923F07E0924007BA
:109B8000F0924107009100030D87A090ED02B09084
:109B9000EE02C501B7FEF0C1882799278A199B09F3
:109BA000EBC11092300310923103109232031092E5
:109BB000330310922C0310922D0310922E03109257
:109BC0002F031092570710925807109259071092BE
:109BD0005A0710925F071092600710926107109267
:109BE00062071BA61CA61DA61EA620E030E040E0D2
:109BF00050E02FA738AB49AB5AAB8091200390912E
:109C00002103A0912203B091230380931C0390931E
:109C10001D03A0931E03B0931F038091180390911E
:109C20001903A0911A03B0911B038093140390931E
:109C30001503A0931603B093170310921602109207
:109C400015021092DF021092DE021092E1021092D1
:109C5000E0023B8D332309F009CA4A8D442309F001
:109C600005CAF7C9309154073C8761C93FEF8E3F61
:109C700093070CF0D7C002960C949743B90161503A
:109C800070404091EF025091F002CA0157FF02C0AC
:109C90000C944444959587959595879597FF02C0B8
:109CA0000C944D442091C6023091C7022817390701
:109CB00014F00C945944CA0157FF02C00C94F85A8E
:109CC00097FF02C00C94F55A9C0135952795359560
:109CD00027952536310514F40C945B4424E630E0D6
:109CE0008091C30284FF02C00C9461443093C70288
:109CF0002093C6027093C9026093C8020C94694411
:109D0000F09266074091F1025091F202CA0157FDAC
:109D100002C00C9415440396959587959595879563
:109D200097FD02C00C941D44909581959F4F0C9413
:109D30001D4480918A04992787FD90954E2D5527C3
:109D4000849FB001859F700D949F700D1124CB01ED
:109D50002091F1023091F202820F931F9093F20250
:109D60008093F10280918B04992787FD9095849FC1
:109D7000D001859FB00D949FB00D1124CD0120918D
:109D8000EF023091F002820F931F9093F0028093C4
:109D9000EF0280918C04992787FD90952091ED0228
:109DA0003091EE02820F931F9093EE028093ED02AA
:109DB00080918E04282F332727FD30958091D90676
:109DC0009927289FF001299FF00D389FF00D11244D
:109DD000F0938301E093820180918D0499278C1583
:109DE0009D0514F00C94F7439093EC028093EB02E2
:109DF0000C94FB43982F0C94204581E08093D9026A
:109E00000C94154581E08093D802582F0C94E844B7
:109E100081E08093DA020C94BE4481E08093DB02FF
:109E20000C9491441092EE021092ED020C949B431C
:109E30009093DC028093DD0244C88091EA0288237B
:109E400011F40C944E458091C4029091C502FFEF2D
:109E50008F3F9F0711F40C94524501969093C502D1
:109E60008093C4020C9452451092D80250E00C9496
:109E7000E8441092DA020C94BE441092D9020C9479
:109E8000154561507E4F8F4F9F4F9CCD60E070E035
:109E90002B01109200031D86A0905707B090580721
:109EA000C0905907D0905A07E0905F07F090600784
:109EB000009161071091620780916607882309F07D
:109EC000B8C71092E1021092E0021092DF021092E5
:109ED000DE02A092A903B092AA03C092AB03D09273
:109EE000AC03E092AD03F092AE030093AF03109386
:109EF000B00310923003109231031092320310928B
:109F0000330310922C0310922D0310922E03109203
:109F10002F03109228031092290310922A03109203
:109F20002B0310925707109258071092590710925E
:109F30005A0710925F071092600710926107109203
:109F4000620710924C0710924D0710924E07109224
:109F50004F0710923E0710923F0710924007109251
:109F600041071092160210921502A090ED02B090D7
:109F7000EE02C501B7FC10CE409774F068EE262EB5
:109F800063E0362E3092A3012092A20119A114FDA4
:109F900003C081E080939603D090E006ED2CFF246F
:109FA00000271127B501882777FD8095982F950107
:109FB000B7FC7CC7442737FD4095542F0E949C7600
:109FC0009B01AC01C801B7010E949C7697FD69C74F
:109FD00059E095958795779567955A95D1F79B01A7
:109FE0008D2D99278A9DA0018B9D500D9A9D500D16
:109FF0001124CA0157FD46C7959587959595879574
:10A00000280F391FC901AA2797FDA095BA2F809361
:10A010007C0390937D03A0937E03B0937F032091F4
:10A020001003309111034091120350911303281B28
:10A03000390B4A0B5B0B213563EC360760E04607B2
:10A0400060E056070CF4ECC680E593ECA0E0B0E0CD
:10A050008093100390931103A0931203B093130302
:10A060008091100390911103A0911203B0911303FA
:10A07000805B9C43AF4FBF4F64F480EB9CE3AFEF3A
:10A08000BFEF8093100390931103A0931203B0933A
:10A090001303C0900603D0900703C114D10409F440
:10A0A000A3C589A183FFA0C58E899F89A88DB98D7D
:10A0B000B7FF02C00C940F5B09E0B595A795979583
:10A0C00087950A95D1F798AF8FAB97FF02C00C9494
:10A0D0001B5B8E859F85A889B989B7FF02C00C9448
:10A0E000155B19E0B595A795979587951A95D1F7C2
:10A0F000BC0197FF02C00C940A5BEFA9F8ADE6170C
:10A10000F70714F478AF6FAB6FA978AD77FF02C093
:10A110000C94065B2B0155944794559447945594A1
:10A1200047940894411C511CACE1AA2EA2E0BA2E1F
:10A13000CA0CDB1C76010027F7FC0095102F24EEDB
:10A140003DEFC20ED31E60908F07709090078090F5
:10A1500091079090920740917E0150917F0160910C
:10A160008001709181014C8F5D8F6E8F7F8FC40154
:10A17000B3012C8D3D8D4E8D5F8D0E941077E21ABC
:10A18000F30A040B150BC801B70128E631E040E0E3
:10A1900050E00E941077DC01CB018C01045B104081
:10A1A000A0908807B0908907C501B7FE02C00C9443
:10A1B000005B8138910514F000E010E02090A201CE
:10A1C0003090A30121143104A9F46FA978AD69314D
:10A1D000710584F48091FE029091FF02800F911F1F
:10A1E0009093FF028093FE0280919603882311F0E2
:10A1F0000C94145CC801880F991F880F991F880F51
:10A20000991FB2010E94DB769B01442737FD4095E0
:10A21000542F260D371D481D591D20938F0730934D
:10A2200090074093910750939207F09093016F2D00
:10A230007727AFA9B8AD6A9FC0016B9F900D7A9F39
:10A24000900D112497FF02C00C94FD5A95958795A7
:10A2500095958795959587959595879595958795E6
:10A26000681B790B78AF6FAB77FF02C00C94235B50
:10A270002114310411F00C94385B0091C802109144
:10A28000C9028091C6029091C702080F191F17FFDB
:10A2900002C00C947B5C159507951595079515954F
:10A2A0000795005C1F4FCA01B9012C8D3D8D4E8D65
:10A2B0005F8D0E941077DA01C9012091040330916B
:10A2C0000503442737FD4095542F821B930BA40BA5
:10A2D000B50B845E9D4FAF4FBF4FBC01CD0128E64B
:10A2E00031E040E050E00E941077DC01CB01845B5C
:10A2F00090402FA938AD829FF001839FF00D929F6F
:10A30000F00D1124CF01B8010E94DB7683E0F89EA6
:10A31000A001112458AF4FAB4617570714F00C9407
:10A320002B5BBA01CB01AA2797FDA095BA2F2091EC
:10A330001003309111034091120350911303820FC7
:10A34000931FA41FB51F8093100390931103A09334
:10A350001203B09313038091950381508F3F09F44A
:10A360004CC4809395035D85552381F0109278034A
:10A370001092790310927A0310927B031092740367
:10A380001092750310927603109277036B8D6623FB
:10A3900009F043C5809166079927AA27BB27BC010E
:10A3A000CD012E893F89488D598D0E949C76DC0114
:10A3B000CB01BC01CD0128EF3AE240E050E00E9421
:10A3C000107729017A8D772309F024C580916607DB
:10A3D0009927AA27BB27BC01CD012E853F85488937
:10A3E00059890E949C76DC01CB01BC01CD0128EF8C
:10A3F0003AE240E050E00E9410771901809038075F
:10A400009090390789EC881691040CF4F8C4B8ECE4
:10A410008B2E912C90923907809238070091430738
:10A4200010914407093C11050CF4E1C408EC10E05C
:10A430001093440700934307809145079091460786
:10A44000AA2797FDA095BA2F20918D07C22EDD2453
:10A45000EE24FF24BC01CD01A70196010E949C7649
:10A460009B01AC01C401AA2797FDA095BA2FF7E084
:10A47000880F991FAA1FBB1FFA95D1F7280F391F04
:10A480004A1F5B1F57FDECC4E6E05595479537958D
:10A490002795EA95D1F7F201E20FF31FFAAFE9AF82
:10A4A0003F018091360790913707AA2797FDA09525
:10A4B000BA2FBC01CD01A70196010E949C769B0199
:10A4C000AC01C801AA2797FDA095BA2F77E0880FA5
:10A4D000991FAA1FBB1F7A95D1F7280F391F4A1F52
:10A4E0005B1F57FDB8C466E055954795379527958E
:10A4F0006A95D1F76101C20ED31E4601AA0CBB1C9E
:10A50000C501AA2797FDA095BA2F20913D073327B3
:10A5100044275527BC01CD010E949C767B018C010C
:10A5200097FD90C436E015950795F794E7943A9512
:10A53000D1F73C85832F9927AA27BB272091240395
:10A54000309125034091260350912703BC01CD0192
:10A550000E949C76DC01CB01BC01CD0120EF35E5EA
:10A5600040E050E00E9410775701A20EB31EC501D3
:10A5700049AD5AAD415050442CF0A0E0B0E4BAAF20
:10A58000A9AF3D01E9ADFAADE050F04C0CF02AC4A2
:10A5900020E030EC3AAF29AF3093460720934507CF
:10A5A00031E0C31630E4D30624F0C12C20E4D22ECF
:10A5B000460140E0C41640ECD4060CF00EC4C12C99
:10A5C00000ECD02ED0923707C092360751E0A51686
:10A5D00050E4B50624F0A12C10E4B12EC50160E0D2
:10A5E000A61660ECB6060CF0F3C3A12CB0ECBB2EA3
:10A5F000B0928907A092880780910001482F5527C3
:10A6000080912501909126014817590794F42091D3
:10A61000250130912601A981BA814A9FC0014B9F33
:10A62000900D5A9F900D1124B9010E94C7767A832C
:10A630006983E981FA81EE0FFF1FEE0FFF1FFA8396
:10A64000E983F9A1F0FF53C00A8D002309F04FC040
:10A650001B8D112309F04BC0882499248091B503E8
:10A660009091B6039093030680930206809117029F
:10A67000909118029093FD058093FC0520915A0358
:10A6800030915B032115310509F0F5C480911B0160
:10A6900090911C018959934010F00C94815B80913A
:10A6A0001B0190911C018436910510F00C94A25C62
:10A6B00087B58B3010F40C94F05D809119028F5F98
:10A6C000809319029AE08902900111248091250655
:10A6D000821B87BD8CE291E090930302809302027B
:10A6E0008EE591E090935B0380935A03E5C47090EC
:10A6F000870760904A07262D3327C901880F991FC5
:10A70000880F991F889649815A818417950714F0FC
:10A710009A838983872D9927880F991F880F991FFE
:10A720008055904069817A818617970714F49A833F
:10A73000898380914B028823A1F08091C40290917B
:10A74000C5020297C09768F489819A811816190684
:10A7500044F481E090E09093C5028093C4023A8370
:10A760002983A981BA81B093E705A093E60580917A
:10A770007C0390917D03A0917E03B0917F03880FAD
:10A78000991FAA1FBB1F880F991FAA1FBB1FA81ABA
:10A79000B90AE981FA81E13AF1050CF407C3CF0166
:10A7A000F7FD9EC3959587958A159B050CF45C0172
:10A7B000909581959F4FA816B9060CF45C01272D42
:10A7C0003327220F331F220F331FC90149815A81BA
:10A7D000841B950B8A159B050CF45C0169817A81B9
:10A7E000621B730BA616B7060CF45B018091F10295
:10A7F0009091F20209AD1AAD081B190B1093560780
:10A800000093550780906607882009F4C9C2481A4A
:10A81000590AC201AA2797FDA095BA2F2091740367
:10A82000309175034091760350917703820F931F07
:10A83000A41FB51F8093740390937503A0937603B0
:10A84000B0937703609174037091750380917603E0
:10A85000909177036130AAEF7A07A0E08A07A0E021
:10A860009A0774F080E09AEFA0E0B0E08093740360
:10A8700090937503A0937603B0937703BC01CD0149
:10A880006030B6E07B07BFEF8B07BFEF9B0774F428
:10A8900080E096E0AFEFBFEF809374039093750371
:10A8A000A0937603B0937703BC01CD01E0909801AB
:10A8B000F09099019701442737FD4095542F0E944D
:10A8C0001077020F131F90908401692D7727882736
:10A8D00099279501B7FCD1C237FDCCC23595279594
:10A8E000E981FA812E0F3F1F442737FD4095542FF1
:10A8F0000E949C7697FDB9C256E09595879577950D
:10A9000067955A95D1F79B01601771070CF48B017D
:10A91000309521953F4F021713070CF48901809160
:10A92000EF029091F002C81AD90AD0923507C0926E
:10A930003407882009F42EC2281A390AC101AA272F
:10A9400097FDA095BA2F209178033091790340911B
:10A950007A0350917B03820F931FA41FB51F80932E
:10A96000780390937903A0937A03B0937B0360916B
:10A9700078037091790380917A0390917B03613021
:10A98000FAEF7F07F0E08F07F0E09F0774F080E0B8
:10A990009AEFA0E0B0E08093780390937903A093BE
:10A9A0007A03B0937B03BC01CD01603026E07207CF
:10A9B0002FEF82072FEF920774F480E096E0AFEF5D
:10A9C000BFEF8093780390937903A0937A03B093B9
:10A9D0007B03BC01CD019701442737FD4095542FDF
:10A9E0000E9410777601E20EF31E692D77278827E3
:10A9F00099279501B7FC50C237FD4BC23595279575
:10AA000049815A81240F351F442737FD4095542F23
:10AA10000E949C7697FD38C226E09595879577959C
:10AA200067952A95D1F79B016E157F050CF47B0184
:10AA3000309521953F4FE216F3060CF47901180189
:10AA4000442437FC4094542C662D77277CAB6BABA9
:10AA5000872D99279EAB8DABB8E2CB2EB6E0DB2ECF
:10AA600006E014E03701882477FC8094982C9BE062
:10AA70009B83A7E6EA2EA7E0FA2E07C0F8AFEFAB5C
:10AA8000EFA9D601EC930C94C361F8012585121649
:10AA90000CF091C049815A81CA01AA2797FDA0955F
:10AAA000BA2F332727FD3095432F532FBC01CD01FB
:10AAB0000E949C7697FD93C0F6E0959587957795D3
:10AAC0006795FA95D1F778AF6FABF8018685282F97
:10AAD000332727FD3095432F532FC201B1010E9428
:10AAE0009C7697FD77C0E6E0959587957795679575
:10AAF000EA95D1F72FA938AD260F371F38AF2FAB06
:10AB0000F8018785282F332727FD3095432F532FB2
:10AB1000C401B3010E949C7697FD55C056E09595FF
:10AB20008795779567955A95D1F72FA938AD260F58
:10AB3000371F38AF2FABC501AA2797FDA095BA2FB5
:10AB4000F8012089332727FD3095432F532FBC016F
:10AB5000CD010E949C76DC01CB01B7FD30C046E000
:10AB6000B595A795979587954A95D1F7F701608197
:10AB700071812FA938AD820F931F0E94B533D70181
:10AB80008D939C9397FD24C0959587959595879572
:10AB900098AF8FABEBA9FCA98E179F070CF46ECF73
:10ABA0002DA93EA94FA958AD241735070CF068CF41
:10ABB00038AF2FAB65CFD6011C920C94C361CF96F2
:10ABC000A11DB11DCCCF615C7F4F8F4F9F4FA6CF92
:10ABD0000396DACF615C7F4F8F4F9F4F84CF615CCC
:10ABE0007F4F8F4F9F4F68CFA0908807B090890705
:10ABF00080919503815008F0B4CB88E18093950350
:10AC00008091E3069927880F991F880F991F7C016F
:10AC10000027F7FC0095102F6E897F89888D998D0C
:10AC2000A80197010E9410773093D9052093D80589
:10AC30006E857F8588899989A80197010E94107780
:10AC40003093DB052093DA05809183079091840788
:10AC500097FDC1C495958795959587959093DD054A
:10AC60008093DC05809193079091940797FDB1C480
:10AC700095958795959587959093DF058093DE054B
:10AC8000B092E105A092E0058091E6029091E70282
:10AC9000A091E802B091E902BC01CD0125E030E0CD
:10ACA00040E050E00E9410773093E3052093E205E6
:10ACB00080911B0690911C069093E5058093E40516
:10ACC000D092E905C092E805809125019091260176
:10ACD0009093EB058093EA058091F4029927909375
:10ACE000ED058093EC0580918F0790919007A091DE
:10ACF0009107B091920720917E0130917F014091A0
:10AD0000800150918101BC01CD010E9410773093E8
:10AD1000EF052093EE058091170290911802909311
:10AD2000FD058093FC058091850499279093FF058C
:10AD30008093FE058091FE019091FF0190930106A2
:10AD4000809300068091050890910608909305066F
:10AD5000809304068091090890910A089093070651
:10AD60008093060680910308992790931306809399
:10AD700012068091D6039091D70390931506809385
:10AD800014068091D4039091D50390931706809375
:10AD90001606E9CAC601AA2797FDA095BA2FD3CDFA
:10ADA000C801AA2797FDA095BA2F38CDF1E5AF16B7
:10ADB000B1041CF0B0E5AB2EB12C00EBA0160FEFE8
:10ADC000B0060CF0FCCCA0EBAA2EAFEFBA2EF7CC5D
:10ADD00090938907809388070FCC909237078092D1
:10ADE0003607F4CB7092460760924507D9CBAFEF98
:10ADF00008331A070CF020CB08E31FEF19CB98E3B8
:10AE000089169FEF99060CF009CBA8E38A2EAFEFC5
:10AE10009A2E00CB22243324F1CA44245524D2CACA
:10AE200020931003309311034093120350931303A4
:10AE300017C95092E1024092E0027093DF026093E2
:10AE4000DE0247C82FE330E040E050E0E20EF31EA0
:10AE5000041F151F67CB215C3F4F4F4F5F4F43CB04
:10AE6000215C3F4F4F4F5F4F0FCB615C7F4F8F4F48
:10AE70009F4F42CD2F5F3F4F31CD222733272A19D5
:10AE80003B092ACD0396B8C8615C7F4F8F4F9F4F17
:10AE9000C3CD2F5F3F4FB2CD222733272A193B095D
:10AEA000ABCD61507E4F8F4F9F4F92C822273327E3
:10AEB0002A193B097FC88091C30282608093C30234
:10AEC0000C946D451092EC021092EB020C9403442A
:10AED0004D5F5F4F0C945F434D5F5F4F0C94154384
:10AEE000019660CC8091E306E82EFF24002711270D
:10AEF0006E897F89888D998DA80197010E941077AE
:10AF000039014A018091830790918407AA2797FD10
:10AF1000A095BA2F681A790A8A0A9B0A6E857F85DE
:10AF200088899989A80197010E94107759016A01BF
:10AF30008091930790919407AA2797FDA095BA2F27
:10AF4000A81AB90ACA0ADB0AD401C30197FCCFC404
:10AF50003C014D0154E095948794779467945A95F9
:10AF6000D1F7D601C501D7FCBEC45C016D0144E038
:10AF7000D594C794B794A7944A95D1F78091C80205
:10AF80009091C902813491050CF486C3C401B301C8
:10AF900023E030E040E050E00E94107739014A01A0
:10AFA000C601B50123E030E040E050E00E94107798
:10AFB00059016A018091CB06E82FFF27EE0FFF1F92
:10AFC000E75AF94F808191810190F081E02DF7FDE2
:10AFD00086C47A97A4F0C401B30123E030E040E0D6
:10AFE00050E00E94107739014A01C601B50123E003
:10AFF00030E040E050E00E94107759016A0171E2B0
:10B0000067167104810491042CF030E2632E712CD8
:10B01000812C912C80EE68168FEF78068FEF8806D2
:10B020008FEF980644F420EE622E2FEF722E2FEF52
:10B03000822E2FEF922E91E2A916B104C104D10401
:10B040002CF090E2A92EB12CC12CD12CA0EEAA1686
:10B05000AFEFBA06AFEFCA06AFEFDA0614F00C9402
:10B06000794D80EEA82E8FEFB82E8FEFC82E8FEF80
:10B07000D82E0C94794D8091E6029091E702A09130
:10B08000E802B091E902E4E0880F991FAA1FBB1FF4
:10B09000EA95D1F780931A0290931B02A0931C02A9
:10B0A000B0931D02909218028092170221503040F6
:10B0B00030935B0320935A0349A141FF42C0809122
:10B0C0009601823308F016C38091C301815098F431
:10B0D000109201032091E6023091E7024091E802CC
:10B0E0005091E9022093E2023093E3024093E4029C
:10B0F0005093E50281E08093C30145C0E0917B015C
:10B10000F0917C01E853F94F8081E82FFF27EE0F83
:10B11000FF1FE75AF94F808191818C3491050CF41F
:10B12000E5C2809194038F5F893C08F4F8C31092C4
:10B13000EA02109294031092C5021092C4020C9479
:10B14000E142209196018091820190918301820FCA
:10B15000911D2091D9063327829FB001839F700DE6
:10B16000929F700D11249B01442737FD4095542F69
:10B170002093E2023093E3024093E4025093E5020D
:10B1800081E080930103E0907E01F0907F010091C7
:10B190008001109181016E897F89888D998DA80128
:10B1A00097010E94107759016A016E857F85888911
:10B1B0009989A80197010E941077B901C5010E94E1
:10B1C000B96D5C01CC971CF07CE3A72EB12CC501B6
:10B1D0000E94F5695C0140E280910103882309F433
:10B1E00024C18091C30299279C012071307084FD95
:10B1F0001CC16090270760FC04C08091D40681FDCB
:10B200005AC540937D01C980DA803093B203209300
:10B21000B1038091E6029091E702A091E802B0911B
:10B22000E90289AF9AAFABAFBCAF2091E202309197
:10B23000E3024091E4025091E502E9ACFAAC0BADB7
:10B240001CAD2E153F054007510714F060FC05C1E9
:10B2500080915A0390915B03892B09F4B0C3C0908D
:10B26000B503D090B60388249924E0900803F090A9
:10B27000090300910A0310910B0317FDA6C6A7E06E
:10B2800015950795F794E794AA95D1F780919401C5
:10B29000282F332744275527C801B7010E949C76E1
:10B2A00097FDA2C67B018C01F5E015950795F794F3
:10B2B000E794FA95D1F731E8E3163FEFF3063FEF55
:10B2C00003073FEF13070CF06CC3E0E8EE2EEFEF3F
:10B2D000FE2EEFEF0E2FEFEF1E2FE0928003F09285
:10B2E00081030093820310938303809180039091E4
:10B2F0008103C81AD90A80919201282F332780919F
:10B300000408992787FD9095289FB001299F700D0B
:10B31000389F700D11249B0177FD63C6220F232FE8
:10B32000221F330B7FEF213837070CF032C320E8A0
:10B330003FEFC21AD30A85E990E0880E991E9BE27E
:10B34000891691E09906E8F48091B1039091B203D7
:10B35000892BB9F48091B5039091B603181619069C
:10B3600084F48091B7039091B8038C159D050CF07F
:10B3700074C28091C1019091C201C816D9060CF027
:10B380006CC2C601AA2797FDA095BA2F5DE0880F71
:10B39000991FAA1FBB1F5A95D1F79501442737FD66
:10B3A0004095542FBC01CD010E9410772093840357
:10B3B000309385034093860350938703C0908403A2
:10B3C000D09085038091B3039091B4039C01220F28
:10B3D000331F280F391F2C0D3D1D37FDFFC5A90157
:10B3E0005595479555954795BA018091D506282FD3
:10B3F0003327220F331F220F331F241735070CF476
:10B40000B7C2A901B9017090870760FE78C2A9810F
:10B41000BA814A175B070CF472C2AD01B093B40352
:10B42000A093B3035A8349831AC040937D0160916E
:10B43000DD06662309F439C17727673471050CF0FE
:10B4400019C266E470E07093C0016093BF01C980C7
:10B45000DA80D092B403C092B303709087078091D2
:10B46000C30281FFFCC18091C30284FD2DC2E09024
:10B47000B903F090BA030091BB031091BC03E1142F
:10B48000F10401051105B1F429813A817901002700
:10B49000F7FC0095102FACE0EE0CFF1C001F111FF5
:10B4A000AA95D1F7E092B903F092BA030093BB03D7
:10B4B0001093BC038091170290911802809117029B
:10B4C0009091180297FDD8C4843691050CF02BC2D8
:10B4D00069817A819B01442737FD4095542FC5012E
:10B4E000AA2797FDA095BA2FBC01CD010E949C769A
:10B4F00097FD81C59B01AC01FDE0559547953795BA
:10B500002795FA95D1F720938403309385034093D0
:10B510008603509387038091C4029091C50277E01F
:10B52000803D970708F095C3D801C701E9E0B695BB
:10B53000A79597958795EA95D1F7E81AF90A0A0B26
:10B540001B0BDA01C90173E0880F991FAA1FBB1FEB
:10B550007A95D1F7E80EF91E0A1F1B1FE092B90376
:10B56000F092BA030093BB031093BC03D801C70148
:10B570006CE0B695A795979587956A95D1F79093C6
:10B58000B6038093B5034091DB06442309F47EC3E0
:10B5900055279C01BA010E94DB76C901861B970BD7
:10B5A0009093B8038093B703260F371F3093C201DF
:10B5B0002093C101A0908807B0908907E0914507CA
:10B5C000F0914607FAAFE9AFC0903607D090370741
:10B5D00090C803964DCB03963DCB909581959F4F98
:10B5E0000C942B4403960C942F4403960C94644EB5
:10B5F000909581959F4F0C94604E4F960C942651D8
:10B60000882799278A199B090C94D950695F7F4F25
:10B610000C948A50709561957F4F0C947D508150A9
:10B620009E4FAF4FBF4F0C945C5081509E4FAF4F19
:10B63000BF4F0C947150DC01B095A195BF4FB8AFCE
:10B64000AFAB0C94695084EF91E09093A301809389
:10B65000A2010C94AB518FA998AD909581959F4F05
:10B660006817790714F00C949251BC010C94925114
:10B670000894210831083092A3012092A2010C9471
:10B68000AB51F095E195FF4F0C94354D61507E4FD5
:10B690008F4F9F4F0C94F54C8091C6029091C7023A
:10B6A000813491050CF486CC71CC4091B503509156
:10B6B000B60357FD7CC255954795559547958091A2
:10B6C000250190912601209100013327489FF00128
:10B6D000499FF00D589FF00D1124CF01B9010E9430
:10B6E000DB76ABCE109293030C94E142109294035C
:10B6F0000C94E14281E08093010388EC8093C301C4
:10B7000042CD87B5853F08F023C180911902815051
:10B710000C94605380819181855B9F4F0CF00EC12A
:10B72000809192038F5F80939203893C10F40C9474
:10B7300084462C3008F05DC42998A4E0B0E08FEF77
:10B74000082E0E9475771092EA02109292031092CE
:10B75000C5021092C4020E947E3DA4E0B0E0809138
:10B760004E0390914F0397FD4AC5892F990F990B6E
:10B77000082E0E947577A5E0B0E080914E0390916D
:10B780004F03082E0E947577A6E0B0E080914C032D
:10B7900090914D0397FD30C5892F990F990B082E75
:10B7A0000E947577A7E0B0E080914C0390914D0323
:10B7B000082E0E94757708E010E080914603909172
:10B7C0004703A0914803B0914903BC01CD010E94F9
:10B7D0000576DC01CB019C0197FD25C5832F9927B8
:10B7E00087FD9A95D801082E0E94757709E010E030
:10B7F0008091460390914703A0914803B09149037B
:10B80000BC01CD010E940576DC01CB01D801082ED8
:10B810000E9475770E949A0768E770E00E94CB3318
:10B820003091CA060C948446C601AA2797FDA095BC
:10B83000BA2FBC01CD012C8D3D8D4E8D5F8D0E94A8
:10B840009C763B014C010E941077309305032093B6
:10B850000403109296030C94FA506C0192CDA090C0
:10B860008807B0908907E0904507F0904607FAAE48
:10B87000E9AEAACE663971050CF4E5CD86E990E013
:10B880009093C0018093BF01E2CD0196A11DB11D2F
:10B890000C941E4D0196A11DB11D0C94124D81E01A
:10B8A0008093960310927C0310927D0310927E0386
:10B8B00010927F0310921003109211031092120342
:10B8C000109213030C946D45A0908807B0908907DF
:10B8D00000914507109146071AAF09AF75CEF09554
:10B8E000E195FF4F76CB0F96A11DB11D3ECB0F9674
:10B8F000A11DB11D2DCB095F1F4F0C944B517093AF
:10B90000B4036093B3035A834983A9CD3092A4034F
:10B910002092A3032091010828A30C94144A809339
:10B9200094030C94E142A0908807B090890720917D
:10B930004507309146073AAF29AF46CE4093920370
:10B940000C9484463B8D3093BD033093BE03B4CB3F
:10B9500081E08093BE03B0CB809392030C94844625
:10B960001092A8030C944B4C1092A5030C947A4AA5
:10B9700070908707272D3327220F331F220F331F85
:10B9800020553040421753070CF43FCDA901B901AF
:10B990003CCD2F3F310509F00CF4CBCC20E031E059
:10B9A000C8CC4FEFE416F1040105110509F00CF4C1
:10B9B00094CCE12C71E0F72E012D112D8ECCE9AC49
:10B9C000FAAC0BAD1CADE21AF30A040B150B22E026
:10B9D000E21620E8F2062FEF02072FEF12070CF015
:10B9E000DEC251E0E52E50E8F52E5FEF052F5FEF48
:10B9F000152FE0928003F09281030093820310934D
:10BA00008303809080039090810380919501992712
:10BA1000AA27BB27BC01CD01A80197010E949C76F3
:10BA200097FDC6C37B018C0134E015950795F7940B
:10BA3000E7943A95D1F745E0E4164CEFF4064FEF62
:10BA400004074FEF14070CF099C224E0E22E2CEF0C
:10BA5000F22E2FEF022F2FEF122FE0928003F092A1
:10BA6000810300938203109383038091800390915C
:10BA70008103C81AD90A609117027091180277FDE4
:10BA800092C39B0135952795359527953595279533
:10BA90006FEF2C3436070CF06AC22BE43FEFC9017C
:10BAA000283031050CF44FC288E090E0889FD00127
:10BAB000899FB00D989FB00D1124CD01B7FD76C3BD
:10BAC0009595879595958795280F391FC901AA27C0
:10BAD00097FDA095BA2F209197013327442755272A
:10BAE000BC01CD010E949C7697FD7BC3B7E0959584
:10BAF000879577956795BA95D1F79B01BFEF613828
:10BB00007B070CF0BDC120E83FEFC21AD30AADCBD2
:10BB100020939B0330939C0340939D0350939E037B
:10BB20001092A7030C94D94B2FA138A549A55AA56B
:10BB300020939703309398034093990350939A036B
:10BB40001092A6030C94E64A809393030C94E1426E
:10BB50000E949A074CE668EC76E00E94420780E07B
:10BB60000E94E5070E9401748091D40680FF10C0F6
:10BB700080911B0190911C01875B934038F4809168
:10BB80001B0190911C018E5E924010F40E94A31C38
:10BB9000109200020E947E3D81E08093000281E0CD
:10BBA00090E09093C2028093C102579A33CE4D5FCA
:10BBB0005F4F81CD609297037092980380929903B2
:10BBC00090929A031092A4031092A30388EE282E59
:10BBD00083E0382E3092A3012092A2010C94E64A11
:10BBE00081E08093BD0368CA4091790150917A0148
:10BBF0000C94D245299A0C94A0457093DF0260936F
:10BC0000DE025092E1024092E002CB0177FD3FC399
:10BC1000BC0175956795C20157FC37C32C0155943B
:10BC200047940C943C4920939B0330939C0340938E
:10BC30009D0350939E031092A4031092A303E8EE79
:10BC40002E2EE3E03E2E3092A3012092A2010C940E
:10BC50004B4CAFE0803A9A0708F0D2C1D801C70137
:10BC60006AE0B695A795979587956A95D1F7E81AF2
:10BC7000F90A0A0B1B0BDA01C901880F991FAA1FC9
:10BC8000BB1F880F991FAA1FBB1F64CC1092B8035B
:10BC90001092B7038FEF93E09093C2018093C1019C
:10BCA000A0908807B0908907C0904507D0904607BC
:10BCB000DAAEC9AE89CC8091C30281FFC3C1609165
:10BCC000BF017091C001CB010F962091EB02309122
:10BCD000EC02821793070CF0E2C18091BD03882328
:10BCE00009F0DDC18091BF0381FF40C38D7FC0900B
:10BCF000E602D090E702E090E802F090E902C9AED7
:10BD0000DAAEEBAEFCAEC092E202D092E302E09279
:10BD1000E402F092E50281608093BF03261B370B9B
:10BD20002F50304037FD1EC38091B1039091B20374
:10BD3000280F391F3093B2032093B1038BE2809315
:10BD40007D012091B1033091B203C90137FDD1C209
:10BD5000815092400CF46CC18091D9069927829F42
:10BD6000B001839F700D929F700D1124CB0160E094
:10BD700075E00E94DB769B01442737FD4095542FE8
:10BD80008091E2029091E302A091E402B091E50279
:10BD9000280F391F4A1F5B1F1092B2031092B10384
:10BDA00089AD9AADABADBCAD80509440A040B040E1
:10BDB00082179307A407B50774F489AD9AADABADAC
:10BDC000BCAD80509C4FAF4FBF4F281739074A0773
:10BDD0005B070CF4A1C28093E2029093E302A0936C
:10BDE000E402B093E50261FE06C08BE490E090931C
:10BDF0000302809302028091DD06882309F018C1B6
:10BE00000091B5031091B603A80117FD97C255958F
:10BE10004795559547958091250190912601209150
:10BE200000013327489FD001499FB00D589FB00DA6
:10BE30001124CD01B9010E94DB76663471050CF046
:10BE400076C266E470E07093C0016093BF01809198
:10BE50005A0390915B03892B09F4AFC129AD3AAD28
:10BE60004BAD5CAD2093E2023093E3024093E402D9
:10BE70005093E5026801E1C9909581959F4F24CBCD
:10BE80006F3F710509F00CF440CE20E031E0C21A9A
:10BE9000D30AEBC9B095A095909581959F4FAF4F70
:10BEA000BF4F0C943C4B20939B0330939C034093D7
:10BEB0009D0350939E0381E08093A7030C94D94B7C
:10BEC0008FA198A5A9A5BAA58093970390939803ED
:10BED000A0939903B0939A0381E08093A6030C94F6
:10BEE000E64A81509F4FAF4FBF4F0C940E4981508F
:10BEF0009F4FAF4FBF4F0C94014981E08093A50342
:10BF00000C947A4A88279927DC018E199F09A00B87
:10BF1000B10B0C94E24961507F4F8F4F9F4F0C94AF
:10BF2000CF4861507F4F8F4F9F4F0C94B94881503D
:10BF30009F4FAF4FBF4F0C94914881509F4FAF4FD1
:10BF4000BF4F0C947748121613060CF4AFCD229F06
:10BF5000C001239F900D329F900D112497FDE5C1E4
:10BF60009595879595958795281B390BAFCD253BE2
:10BF700031050CF494CD25EB30E091CD5CEFE51666
:10BF800053E0F50650E0050750E015070CF465CDC9
:10BF90009CEFE92E93E0F92E012D112D5ECD3FEFA0
:10BFA000E3163FE7F30630E0030730E013070CF435
:10BFB00020CD4FEFE42E4FE7F42E012D112D19CD9A
:10BFC00081E08093A8030C944B4C2FE730E040E0D5
:10BFD00050E0E20EF31E041F151F51C92D5F3F4FA5
:10BFE000FEC921583F4F9AC9615E7F4F8F4F9F4FC7
:10BFF00059C9299AA2CB6150704E8F4F9F4F7ACA70
:10C0000080549F4108F0B3C0D801C701EBE0B6955A
:10C01000A79597958795EA95D1F7E81AF90A0A0B3B
:10C020001B0BDA01C901820F931FA41FB51F92CA0F
:10C030000091B5031091B6030ACF909581959F4F5B
:10C040000C94664640937D01C090E602D090E702D2
:10C05000E090E802F090E902C9AEDAAEEBAEFCAED9
:10C06000A701960120593140404050402093E20200
:10C070003093E3024093E4025093E5028091DD06A1
:10C08000882309F443C0682F77277093C001609319
:10C09000BF010091B5031091B6036801CEC8CB0172
:10C0A0000F9728173907ACF58091BE03882389F5CF
:10C0B0008091BF0380FF49C18E7FC090E602D0907F
:10C0C000E702E090E802F090E902C9AEDAAEEBAE2A
:10C0D000FCAEC092E202D092E302E092E402F0925F
:10C0E000E50282608093BF03261B370B215F3F4F21
:10C0F00037FD27C18091B1039091B203821B930B4E
:10C100009093B2038093B1038DE219CE68E770E09B
:10C11000BCCF2091BF03822F992783709070892B09
:10C1200009F4ECC02C7F2093BF031092B20310924D
:10C13000B1030091E6021091E7022091E8023091EC
:10C14000E90209AF1AAF2BAF3CAF0093E2021093A4
:10C15000E3022093E4023093E50261FE06C084EF1F
:10C1600091E090930302809302028DE3E8CDD80121
:10C17000C7017CE0B695A795979587957A95D1F7F5
:10C18000E81AF90A0A0B1B0BE20EF31E041F151F17
:10C19000E5C920939B0330939C0340939D035093E8
:10C1A0009E030C94C14B695F7F4F6BCC039688CC88
:10C1B000615F7F4F8F4F9F4F35CC2091E2023091CE
:10C1C000E3024091E4025091E502680136C82093F1
:10C1D0009B0330939C0340939D0350939E030C94C8
:10C1E000334C61587F4F8F4F9F4F80CC81509F4F72
:10C1F000AF4FBF4F0C94DA4A81509F4FCDCA815048
:10C200009F4FB3CA295F3F4F4F4F5F4F0C94A44BD2
:10C2100081509E4FAF4FBF4F0C948F4BF095E195DF
:10C22000FF4F0C94CE4521503F4FD8CAF095E19571
:10C23000FF4F0C943449B095A095909581959F4FF0
:10C24000AF4FBF4F0C948B4B88279927DC018E1979
:10C250009F09A00BB10B0C94954A295F3F4F4F4F9C
:10C260005F4F0C94B24A21503E4F4F4F5F4F0C949A
:10C270009B4A295F3F4F4F4F5F4F0C944C4A2150D0
:10C280003E4F4F4F5F4F0C94354A0196C7CC0196F5
:10C29000BFCC81509F4FAF4FBF4F0C94724A295F64
:10C2A0003F4F4F4F5F4F0C94164C21503E4F4F4F16
:10C2B0005F4F0C94FD4BB095A095909581959F4F45
:10C2C000AF4FBF4F0C94F74B81509F4FAF4FBF4FB5
:10C2D0000C943F4C88279927DC018E199F09A00BED
:10C2E000B10B0C942F4A81509F4FAF4FBF4F0C940E
:10C2F000CD4B88279927821B930B2ACD2091E602EC
:10C300003091E7024091E8025091E90229AF3AAF3B
:10C310004BAF5CAF8DE313CD2093E2023093E30289
:10C320004093E4025093E5025ECD039619CE67393F
:10C3300071050CF488CD66E970E085CD4D5F5F4FE7
:10C3400066CD309521953F4FD5CEE090E602F09036
:10C35000E7020091E8021091E902E9AEFAAE0BAFF4
:10C360001CAFBFCE309521953F4FDECCE090E6026A
:10C37000F090E7020091E8021091E902E9AEFAAE0E
:10C380000BAF1CAFC8CCBB81B150BB83E2E0F0E087
:10C39000EE0EFF1E0C5F1F4F24E030E0C20ED31ED6
:10C3A000B7FD02C00C944555E2E1C45C0C9447779C
:10C3B0008091CC039091CD03A091CE03B091CF0397
:10C3C0008093C4039093C503A093C603B093C7039F
:10C3D0008091C8039091C903A091CA03B091CB0387
:10C3E0008093C0039093C103A093C203B093C3038F
:10C3F00008951092D7031092D6031092D50310928D
:10C40000D403089584B1806A84B93D9A82E58CBDD5
:10C410001DBC459A81E0809399078AEA8093A90719
:10C4200083E88093AA078AE08093AB071092AD0758
:10C430001092AC071092AF071092AE07109203084B
:10C440001092CB070895EF92FF920F931F93809164
:10C45000E3069927880F991F880F991F7C010027F1
:10C46000F7FC0095102F8091400390914103A0911B
:10C470004203B0914303BC01CD01A80197010E9482
:10C4800010773093AD072093AC07809138039091DB
:10C490003903A0913A03B0913B03BC01CD01A8013F
:10C4A00097010E9410773093AF072093AE07209139
:10C4B0008F07309190074091910750919207DA01D0
:10C4C000C901E3E0880F991FAA1FBB1FEA95D1F7A6
:10C4D000820F931FA41FB51F820F931FA41FB51FA8
:10C4E00020917E0130917F01409180015091810126
:10C4F000BC01CD010E9410773093B5072093B4079B
:10C50000E0914A03F0914B0380915C0790915D07A5
:10C51000BF010E94DB76CB019B01220F331F220F4C
:10C52000331F280F391F280F391F37FD62C135957A
:10C530002795359527953093B1072093B0078091C3
:10C540008B0790918C07BF010E94DB769B01220F25
:10C55000331F220F331F260F371F260F371F37FDBC
:10C5600045C135952795359527953093B307209389
:10C57000B20710924B0310924A0310925D0710927B
:10C580005C0710928C0710928B078091AB0799275C
:10C590008D30910509F4EDC08E3091050CF0C3C0CB
:10C5A0008B30910509F4E3C18C3091050CF445C141
:10C5B00080918504863018F01092850485E0809380
:10C5C000BC07809123078093BD078091E20590917D
:10C5D000E3059093BF078093BE078091E20290919C
:10C5E000E302A091E402B091E502BC01CD0125E097
:10C5F00030E040E050E00E9410773093C107209374
:10C60000C007809119078093C20780911A07809311
:10C61000C30780911B078093C4078091F402809325
:10C62000C5078091F3028093C6078091E60590913B
:10C63000E70597FD27C295958795959587958093F2
:10C64000C7078091CB07882309F4C2C08AEF809383
:10C65000D9032091CD073091CE07C90181509E4F5B
:10C660008F5F934058F44091CF075091D007CA0193
:10C6700081509E4F8F5F934008F443C18091D30750
:10C680009091D40721E0893692070CF0AAC09C0152
:10C690009093070380930603809104039091050310
:10C6A000281B390BC901845E9D4F68E671E00E942A
:10C6B000DB76845B90409093030380930203209188
:10C6C000D7073091D8078091020290910302821718
:10C6D000930728F480918504882309F4F2C080919F
:10C6E000CC0799278836910509F4F6C0893691055B
:10C6F0000CF082C08736910509F0C6C18091D90738
:10C70000809300088091DA07809302088091DB070C
:10C71000809301088091DC07809303088091DD07F6
:10C7200080930408B1C18F30910509F4F7C08F30B0
:10C7300091050CF4B6C0409709F083CF80910508AD
:10C74000909106089093BD078093BC0780910908DB
:10C7500090910A089093BF078093BE0780912501AE
:10C76000909126018093C007809100018093C107BA
:10C7700068CF809114078093BC0780911507809340
:10C78000BD07809116078093BE078091170780939D
:10C79000BF07809118078093C00780911C07809382
:10C7A000C10780911D078093C20780911E07809367
:10C7B000C307809121078093C40780911F0780934E
:10C7C000C507809120078093C6078091220737CF45
:10C7D0001092D7031092D6031092D5031092D4036F
:10C7E00053C1209106033091070356CF2D5F3F4F71
:10C7F000B8CE2D5F3F4F9BCE8936910509F044C1DD
:10C800008091D90780939A078091DA0780939B07DC
:10C810008091DB0780939C078091DD079091DE0774
:10C8200090939E0780939D078091DF079091E0078A
:10C830009093A00780939F0727C10A9709F001CF23
:10C840008091D7028093BC078091D6028093BD0768
:10C850008091D5028093BE078091D4028093BF0758
:10C860008091D3028093C0078091D2028093C10748
:10C870008091D1028093C2078091D0028093C30738
:10C880008091C3028093C4078091C302837F809309
:10C89000C302A2E0B0E00E946877802D8093C507B4
:10C8A000D0CE1092BC078EE48093BD0785E08093C4
:10C8B000BE078CE08093BF07809102018093C00780
:10C8C000C0CE30930302209302028091CC079927B7
:10C8D0008836910509F00ACF8091D9078093A30784
:10C8E0008091DA078093A4078091DB078093A507E6
:10C8F0008091DC078093A6078091DD078093A707CE
:10C90000C3C08091D40685FFB9CE3093D70320935E
:10C91000D6035093D5034093D403B0CE8091FB0649
:10C920008093BC07809126078093BD0780918A0180
:10C930008093BE078091F4068093BF078091F5062F
:10C940008093C0078091F6068093C107809189018A
:10C950008093C2078091F8068093C3078091F906FF
:10C960008093C4078091FA068093C5076ACEF89435
:10C970008091CA06E82FFF27EE0FFF1FE75AF94FF5
:10C980000190F081E02DE038F1050CF45CC0EFE798
:10C99000F0E0E093BC078091CB06E82FFF27EE0F75
:10C9A000FF1FE75AF94F0190F081E02DE038F105C3
:10C9B0000CF460C0EFE7F0E0E093BD078091C9069A
:10C9C000E82FFF27EE0FFF1FE75AF94F0190F08184
:10C9D000E02DE038F1050CF445C0EFE7F0E0E0931E
:10C9E000BE078091C806E82FFF27EE0FFF1FE75A0A
:10C9F000F94F0190F081E02DE038F10564F1EFE7A7
:10CA0000F0E07894E093BF078091F5028093C0072F
:10CA10008091F6028093C1078091F7028093C2074C
:10CA20008091F8028093C3078091F9028093C40734
:10CA30008091FA028093C5078091FB028093C6071C
:10CA40008091FC02FCCD2FEFE138F2070CF0A1CF72
:10CA5000E1E8FFEF9ECF8FEFE138F80794F6E1E8C9
:10CA6000FFEFCFCF6FEFE138F6070CF0B8CFE1E87A
:10CA7000FFEFB5CF4FEFE138F4070CF09DCFE1E8C1
:10CA8000FFEF9ACF0396D7CD1F910F91FF90EF90B4
:10CA9000089580919907882309F43BC0459889EA55
:10CAA00097E09093A2078093A1078091D803E82F85
:10CAB000FF27EC53FE4F982F9F5F80818093AB0739
:10CAC000993008F027C09093D803109299070E94DC
:10CAD000236281E08093A8070000000000000000AE
:10CAE0000000000000000000000000000000000046
:10CAF0000000000000000000000000000000000036
:10CB000000000000000000008091A9078093C80782
:10CB10008EBD08951092D803D8CF20919907222373
:10CB200009F045C00DB407FE42C084E080930102C5
:10CB3000459A3EB58091DA0399278130910509F431
:10CB400037C0823091050CF451C0029709F439C006
:10CB50002091A807203208F030C04598000000005E
:10CB600000000000000000000000000000000000C5
:10CB700000000000000000000000000000000000B5
:10CB8000000000000000000000000000E091A1078C
:10CB9000F091A207E20FF11D80818EBD8091C80740
:10CBA0009081890F8093C8072F5F2093A80708956D
:10CBB000353551F12093DA03CBCF81E0809399078B
:10CBC000F3CF8091CA07E82FFF27EA51F84F30834F
:10CBD0008F5F8093CA078A3100F18091DB03381799
:10CBE00011F12093CB071092DA03B2CF892B09F011
:10CBF000AFCF2093CA073093DB03313809F0A8CFB9
:10CC000081E08093DA03A4CF8091DB03830F8093CC
:10CC1000DB0382E08093DA039BCF8091DB03830FF9
:10CC20008093DB0395CF8AE1E6EEF7E0ACECB7E06A
:10CC300001900D928A95E1F781E08093CB071092E5
:10CC4000DA0386CF87B18C6087B9429843981092F7
:10CC5000DD0380E88093CE011092DC038093CD0148
:10CC600008958091E20381508F3F19F08093E20391
:10CC7000089594E09093E2038091C302807BD9F4FD
:10CC80008093E503482F8093E60380910E078093FD
:10CC9000E303809110078093E40380912507282FF8
:10CCA000332724FF17C08091EA02882399F425FFD7
:10CCB00024C0429A2CC080911207882309F466C0D0
:10CCC0008091E503882311F49093DD0391E0909324
:10CCD000E5035EC090910F07983F28F080915E07B2
:10CCE0008D3D08F08DC0983F50F080915E078A30EE
:10CCF00030F48091E3038823E4F6429808C08091E1
:10CD0000DD0381508F3F09F486C08093DD03442307
:10CD1000A1F580912507282F332724FF05C0809196
:10CD2000EA02882309F473C090911107983F50F0EC
:10CD3000809186078D3D30F08091E4038823DCF0FC
:10CD400043980895983F08F04FC08091DC038150CC
:10CD5000D0F48091860781508093DC038091CD01CF
:10CD6000813009F484C0982F96959093CD018091DD
:10CD7000E403982329F3439A08958091DC038150BA
:10CD80008F3F09F45CC08093DC0308959091E50324
:10CD900080911307882359F08091E603882319F4C2
:10CDA00084E08093DC0341E04093E60302C04091BD
:10CDB000E603992309F471CF8091DD03815008F0D7
:10CDC000A4CF89E08093DD038091CE01813009F406
:10CDD0004CC0982F96959093CE018091120789238D
:10CDE00009F48BCF429A93CF809186078A3008F05E
:10CDF000ACCF8091E40388230CF4A2CF439A08952A
:10CE00008091E30388230CF454CF429880CF26FF0F
:10CE100097CF439A089580915E0781508093DD03F8
:10CE20008091CE018130F9F0982F96959093CE01A4
:10CE30008091E303982309F460CF429A68CF89E098
:10CE40008093DC038091CD01813059F0982F969525
:10CE50009093CD0180911307892309F471CF439AF0
:10CE6000089590E8F5CF90E8E1CF90E8B4CF90E84E
:10CE70007CCF4FB724E130E0F8948091C9008F77E0
:10CE80008093C9008091C9008F7B8093C9008091F5
:10CE9000C9008F7D8093C9005A9A52985B9A539A21
:10CEA000832F99278093CD002093CC008091C800D8
:10CEB00082608093C80080E18093C9008091CA009D
:10CEC0008F778093CA008091CA008F7B8093CA00BD
:10CED0008091CA008F7D8093CA008091CA008F7EA6
:10CEE0008093CA008091CA00877F8093CA00809196
:10CEF000C9008B7F8093C9008091CA0084608093B1
:10CF0000CA008091CA0082608093CA008091C800E4
:10CF100087FF0CC08091CE008091C800882334F434
:10CF20008091CE008091C8008823A4F38091C9002D
:10CF300080688093C9004FBF08950F931F93CF93CC
:10CF4000DF9380E197E20E941618EC018091C900FE
:10CF50008F778093C9008091C9008F7E8093C9002C
:10CF60005A9887E89AE09F938F9301E214E11F9308
:10CF70000F93E0910404F091050409950F900F9030
:10CF80000F900F90CE010E941F18882309F06BC0EC
:10CF90004A9BF8CF8AE590E00E941618EC018DEBD1
:10CFA0009AE09F938F931F930F93E0910404F09165
:10CFB00005040995529A0F900F900F900F90CE0193
:10CFC0000E941F188823D9F383E690E05A9A0197AC
:10CFD00097FFFCCF8FE891E05A98019797FFFCCF1D
:10CFE00089E090E05A9A019797FFFCCF89E090E0A2
:10CFF0005A98019797FFFCCF8FE891E05A9A0197D2
:10D0000097FFFCCF8FE891E05A98019797FFFCCFEC
:10D0100089E090E05A9A019797FFFCCF89E090E071
:10D020005A98019797FFFCCF8FE891E05A9A0197A1
:10D0300097FFFCCF8FE891E05A98019797FFFCCFBC
:10D0400089E090E05A9A019797FFFCCF89E090E041
:10D050005A98019797FFFCCF8FE891E05A9A019771
:10D0600097FFFCCF0FC083EC9AE09F938F931F93A1
:10D070000F93E0910404F091050409950F900F902F
:10D080000F900F9052985A980E943967DF91CF9174
:10D090001F910F910895CF92DF92EF92FF920F931D
:10D0A000CF93DF93482FE0E0F0E08091CF01813013
:10D0B00009F44AC08091E7038823C1F09F01809161
:10D0C000E8038823C9F4232B09F44AC081E0809344
:10D0D000E8038091E9038F5F8093E90303E0809187
:10D0E000E9038031E8F40093E7032AC121E030E04E
:10D0F0008091E803882339F3813009F44AC08230F3
:10D10000B9F1833009F44AC081E08093CF011092D5
:10D11000E9031092EB0304E48091E903803118F3F2
:10D120008091EB03882331F48091CF01882311F49F
:10D13000809378011092E9031092EB031092E803B8
:10D1400084E48093E703FCC01092CF0184E48093D1
:10D15000E7031092E9031092E8031092EA03F0C08B
:10D1600004E48093E9038093E8038093EA03D4CF37
:10D17000232B51F603E04093EA039091E9039230A8
:10D1800009F4A0C083E08093E8039F5F9093E903D4
:10D19000C3CF232B09F0B8CF82E099CF232B09F01E
:10D1A000B3CF082F82E08093E8038091E9038F5F7B
:10D1B0008093E9032091EA03822F9927782F66272D
:10D1C000842F9927682B792B8091ED06813009F403
:10D1D0007EC0823009F492C0737068567140CB01F2
:10D1E00077FDA1C0BC017595679526952695E22F20
:10D1F000FF27EF70F0703196ED30F10508F05BC05D
:10D200007F01EE0EFF1EF701E75AF94F80819181F1
:10D210009B01281B390BC90137FD8AC0069754F4BE
:10D220008091F402883C08F075C08091F402865F1A
:10D230008093F402F701E75AF94F808191819C01B4
:10D24000220F331F280F391F260F371F37FD6DC0E0
:10D25000E901D595C795D595C795CB0101968C1752
:10D260009D070CF043C021978091F402843BC0F1EC
:10D270005DE8C52E56E0D52ECE0CDF1CF701E75A2F
:10D28000F94F80819181FE01E81BF90BCF0163E02A
:10D2900070E00E94DB76CB01880F991F860F971FE5
:10D2A000F6019183808329E536E0E20EF31EF70153
:10D2B000D183C08331CF729708F42ECF81E0809361
:10D2C000CF012ACF47FD38C01092EB035BCF7370BC
:10D2D000CB018050924063E070E00E94DB7685CF06
:10D2E000F701E357F94F11821082DDCF6150704092
:10D2F000C617D7070CF0B8CF2196B6CF7770CB0101
:10D300008050944066E070E00E94DB76269526957A
:10D3100026956DCF88EC8093F40280916F008F7D0D
:10D3200080936F0087CF01965DCF2D5F3F4F90CFE9
:10D33000909581959F4F72CF81E08093EB0322CF30
:10D34000DF91CF910F91FF90EF90DF90CF900895F4
:10D35000CF93FC0197FD21C0C1E028E631E0CF0169
:10D36000B9010E94DB76FC018B35910554F08B5599
:10D3700090408A35910538F484EB90E08E1B9F0B2A
:10D38000FC0141E013C0CF01855B90408A359105D7
:10D3900048F4E45BF0404FEF09C0CFEFF095E19522
:10D3A000FF4FDBCF2E1B3F0BF9014FEFEE0FFF1F9F
:10D3B000E253F54F259134918C2F992787FD909555
:10D3C000829FB001839F700D929F700D1124842F56
:10D3D000992787FD9095689FA001699F500D789FC0
:10D3E000500D1124CA01CF9108952AE530E0281B81
:10D3F000390BC9010E94A8690895CF93DF9380E09B
:10D400000E949D6F80912501909126016AE070E055
:10D410000E94DB769F938F93809125019091260146
:10D420006AE070E00E94DB767F936F938CE99BE06B
:10D430009F938F93C0E9DFE6DF93CF93E0910404DD
:10D44000F091050409952DB73EB7285F3F4F2DBFDA
:10D450008091D903882309F458C086E00E949D6F0B
:10D460008FED90E09F938F9380919F079091A007FD
:10D470009F938F9380919D0790919E076AE070E043
:10D480000E94C7767F936F9385EA9BE09F938F936B
:10D49000DF93CF93E0910404F091050409958DB7D3
:10D4A0009EB70A968DBF80E10E949D6F8091D40146
:10D4B0009091D5016CE370E00E94C7769F938F93A3
:10D4C0008091D4019091D5016CE370E00E94C77601
:10D4D0007F936F938091090890910A089F938F938F
:10D4E00089EB9BE09F938F93DF93CF93E0910404AC
:10D4F000F091050409958091D4062DB73EB7265FBB
:10D500003F4F2DBF80FF3DC013C086E00E949D6F3E
:10D5100082EB9BE09F938F93DF93CF93E091040482
:10D52000F091050409950F900F900F900F90BBCFCD
:10D530008AE10E949D6F80917D0199279F938F932F
:10D540008091E6029091E702A091E802B091E90291
:10D55000BC01CD0124E630E040E050E00E941077AD
:10D560003F932F9386EC9BE09F938F93DF93CF9312
:10D57000E0910404F091050409958DB79EB70896D3
:10D580008DBFDF91CF910895CF93DF9380E00E940C
:10D590009D6F8DEC9BE09F938F93C0E9DFE6DF9357
:10D5A000CF93E0910404F0910504099580E10E9475
:10D5B0009D6F0F900F900F900F9080918F0790911B
:10D5C0009007A0919107B091920720917E01309130
:10D5D0007F014091800150918101BC01CD010E94E9
:10D5E00010773F932F938091380390913903A09146
:10D5F0003A03B0913B03B7FD14C03AE0B595A79547
:10D60000979587953A95D1F79F938F938091400393
:10D6100090914103A0914203B0914303B7FF0AC028
:10D6200005C081509C4FAF4FBF4FE7CF81509C4FFB
:10D63000AF4FBF4F2AE0B595A795979587952A9547
:10D64000D1F79F938F938CED9BE09F938F93DF9304
:10D65000CF93E0910404F091050409958DB79EB72E
:10D660000A968DBFDF91CF9108950F931F9380E0AD
:10D670000E949D6F2AE030E0809105089091060895
:10D68000B9010E94C7769F938F938091050890916E
:10D690000608B9010E94C7767F936F938091250198
:10D6A00090912601B9010E94DB769F938F93809120
:10D6B000250190912601B9010E94DB767F936F933B
:10D6C00088EE9BE09F938F9300E91FE61F930F93D3
:10D6D000E0910404F0910504099580E10E949D6F9A
:10D6E0008DB79EB70C968DBF8091090890910A085E
:10D6F0009F938F9380910708909108089F938F9331
:10D700008BEF9BE09F938F931F930F93E091040403
:10D71000F091050409958DB79EB708968DBF1F91AE
:10D720000F910895CF93DF938091D903882309F453
:10D7300064C080E00E949D6F80919B0799279F9312
:10D740008F9387E09CE09F938F93C0E9DFE6DF93A0
:10D75000CF93E0910404F091050409958DB79EB72D
:10D7600006968DBF80919C0799278230910509F418
:10D7700062C0833091050CF055C0892B09F461C05B
:10D7800087E00E949D6F82E29CE09F938F93DF93DE
:10D79000CF93E0910404F091050409950F900F9048
:10D7A0000F900F9080919A0781FD51C080E10E94F7
:10D7B0009D6F8FED90E09F938F9380919F07909145
:10D7C000A0079F938F9380919D0790919E076AE099
:10D7D00070E00E94C7767F936F938EE29CE09F93E8
:10D7E0008F93DF93CF93E0910404F09105040995A2
:10D7F0008DB79EB70A968DBF3DC082E00E949D6F97
:10D8000080E49CE09F938F9380E99FE69F938F93A2
:10D81000E0910404F091050409950F900F900F908A
:10D820000F9028C0039709F0ABCF87E00E949D6F4F
:10D830008CE19CE0AACF87E00E949D6F86E19CE08E
:10D84000A4CF87E00E949D6F80E19CE09ECF89E09D
:10D850000E949D6F88E29CE09F938F93DF93CF930C
:10D86000E0910404F091050409950F900F900F903A
:10D870000F909CCFDF91CF910895CF93C82F209127
:10D88000EC03322F2093ED0399278F32910521F17C
:10D8900080339105B4F44F9799F12313C0E00E94AF
:10D8A000A36F9091EC0386E0989FF0011124E85754
:10D8B000F44F259134918C2FF901099580E090E087
:10D8C00033C08F34910591F08F38910531F72223C1
:10D8D00009F581E090E028C086E0289FF00111243E
:10D8E000EA57F44F24912093EC03D7CF86E0289F8A
:10D8F000F0011124E957F44F24912093EC03CDCF8C
:10D9000086E0289FF0011124EB57F44F24912093D7
:10D91000EC03C3CF86E0289FF0011124EC57F44FAD
:10D9200024912093EC03B9CFCF910895109206086B
:10D930001092050810920A0810920908109208081F
:10D94000109207088AE090E00E9416189093EF0367
:10D950008093EE030895CF93DF938091EE0390912F
:10D96000EF030E941F18882309F4AAC08091EE03D8
:10D970009091EF030A969093EF038093EE03C0E03B
:10D98000D0E0AE0190E0E8E2F6E02BE004C02150E8
:10D99000349627FD0EC0818187FFF9CF9F5F82817A
:10D9A000C80FD11D8081480F511D2150349627FF8B
:10D9B000F2CF452B09F070C02091F4033091F503AC
:10D9C0004091F6035091F703BB27A52F942F832F87
:10D9D0009093F3038093F203AA27BB27281B390BEC
:10D9E0004A0B5B0BCE01AA27BB27820F931FA41FF4
:10D9F000B51F8093F4039093F503A093F603B093BF
:10DA0000F703C5E0D0E0D0930608C0930508CF3FE8
:10DA1000D10570F580912501909126018C9F900190
:10DA20008D9F300D9C9F300D1124C90164E670E07C
:10DA30000E94C77670930808609307082091F0034E
:10DA40003091F1032C0F3D1F5EE02131350758F076
:10DA50008091090890910A08019690930A08809392
:10DA6000090820513E403093F1032093F00328C071
:10DA7000CE019695879596958795209125013091B1
:10DA80002601829FA001839F500D929F500D11246B
:10DA9000CA0169E170E0CCCF2091F2033091F30329
:10DAA0002C173D0750F0C0E0D0E0892F9927880F50
:10DAB000991FC80FD91F2596A6CFC21BD30BF5CF30
:10DAC000DF91CF910895002422273327442751E086
:10DAD000BB27EE27FF27A0E1660F771F881F991F3E
:10DAE000001C221F331F441F660F771F881F991FBA
:10DAF000001C221F331F441F2AF4050E2B1F3E1F3C
:10DB00004F1F04C0051A2B0B3E0B4F0B550FBB1FAD
:10DB1000EE1F587F556047FD5250AA95E9F6E695ED
:10DB2000B7955795E695B7955795852F9B2F0895EF
:10DB30002227332741E0552768E0880F991F221FCD
:10DB4000331F880F991F221F331F1AF4240F351F0C
:10DB500002C0241B350B440F551F487F456037FD1D
:10DB600042506A9551F75695479556954795842F9B
:10DB70000895AA2797FF04C0809590958A1F9A1F41
:10DB800077FF04C0609570956A1F7A1F669F9001A9
:10DB9000779FA001679F300D411D5A1F300D411D19
:10DBA0005A1F889FF001999F2E0F3F1F401D511D46
:10DBB000899F300D411D5A1F300D411D5A1FCA014A
:10DBC000B901112480CF4FB720E430E0F894809160
:10DBD000C9008F778093C9008091C9008F7B8093A3
:10DBE000C9008091C9008F7D8093C9005A9A5298CC
:10DBF0005B9A539A832F99278093CD002093CC0072
:10DC00008091C80082608093C80088E18093C90039
:10DC10008091CA008F778093CA008091CA008F7B61
:10DC20008093CA008091CA008F7D8093CA00809142
:10DC3000CA008F7E8093CA008091CA00877F80933C
:10DC4000CA008091C9008B7F8093C9008091CA006F
:10DC500084608093CA008091CA0082608093CA0069
:10DC60008091C80087FF03C08091CE00F9CF8091DA
:10DC7000C90080688093C9004FBF08950F931F9318
:10DC8000CF93DF93482F4F5F893108F089C080918F
:10DC90005806841710F440935806CB0183539B42D7
:10DCA00068E170E00E94DB76A42FBB27FD01EA0F3C
:10DCB000FB1FE75AF94F808191819B01281B390B8B
:10DCC000C90137FF03C0909581959F4F069794F443
:10DCD0008091F402883C30F48091F402865F809356
:10DCE000F40208C088EC8093F40280916F008F7D6D
:10DCF00080936F00FD01EA0FFB1FE75AF94F808107
:10DD000091819C01220F331F280F391F260F371FC7
:10DD100037FF02C02D5F3F4FE901D595C795D595D7
:10DD2000C795CB0101968C179D0714F4219706C067
:10DD300061507040C617D7070CF421968091F40209
:10DD4000843BD8F08D010A0F1B1FF801E75AF94FE9
:10DD500080819181FE01E81BF90BCF0163E070E047
:10DD60000E94DB76CB01880F991F860F971F035700
:10DD7000194FF8019183808307C0AA0FBB1FA357D7
:10DD8000B94F11961C921E92E42FFF27EE0FFF1F32
:10DD9000E75AF94FD183C083443011F410927801CF
:10DDA000DF91CF911F910F910895CF93DF93209131
:10DDB0000B08822F9927807F9070409709F06CC0E4
:10DDC0002F3109F046C080910C088093FC0320910C
:10DDD0000E082093FE0380910F088093FD03822F8D
:10DDE000992790935A0680935906222309F054C02C
:10DDF0008091C806282F3327220F331FF901E357DC
:10DE0000F94F118210828091C906A82FBB27AA0F53
:10DE1000BB1FFD01E357F94F118210828091CB06A1
:10DE2000E82FFF27EE0FFF1FCF018357994FEC011B
:10DE300019821882275A394FE90119821882A75A84
:10DE4000B94F11961C921E92E75AF94F1182108217
:10DE500023C0C22FCF70CA30F8F480910C08809391
:10DE6000350880910D088093340880910E088093C6
:10DE7000370880910F0880933608609134087091BC
:10DE800035088C2F0E943E6E6091360870913708DD
:10DE90008C2F8F5F0E943E6EDF91CF910895CF93BC
:10DEA000C82F8F3F49F48091FF038F3F29F41092D0
:10DEB00001041092000432C020910104222339F49D
:10DEC000CF3111F485E001C084E080930204809199
:10DED0000204909100048217A0F4892F809580930A
:10DEE00000048F3F19F48EEF8093000480910004AA
:10DEF000C81711F40E94D56E10920104109200040C
:10DF00000BC0E22FFF27E55FF74FC0832F5F209301
:10DF100001049C0F90930004C093FF03CF910895D8
:10DF20009091FB03933240F4E92FFF27EF5EF74F08
:10DF300080839F5F9093FB030895833218F48D5F75
:10DF40008093FB03089590E2E4E1F8E08FE1919380
:10DF5000815087FFFCCF0895CF93CFB723E031E006
:10DF6000F8948091C9008F778093C9008091C9008F
:10DF70008F7B8093C9008091C9008F7D8093C900F9
:10DF80005A9A52985B9A539A832F99278093CD007F
:10DF90002093CC008091C80082608093C80088E103
:10DFA0008093C9008091CA008F778093CA008091C6
:10DFB000CA008F7B8093CA008091CA0080628093E0
:10DFC000CA008091CA0080618093CA008091CA0013
:10DFD00088608093CA008091C90084608093C900E2
:10DFE0008091CA0084608093CA008091CA008260D8
:10DFF0008093CA008091C80087FF03C08091CE0043
:10E00000F9CF8091C90080688093C9008091C900D0
:10E0100080648093C9000E94A36FCFBFCF91089501
:10E02000282F99278F709070892B31F4209580913B
:10E03000FA03822B8093FA0308958091D1018823FB
:10E0400009F441C08091C30285FF0AC082E9809330
:10E05000110883E28093120885E58093130802C0BB
:10E06000109211088091D2018F3071F48091FA03DF
:10E070000E943D6C882341F081E9809311088093D0
:10E08000120881E3809313081092D1018091C80097
:10E0900085FFFCCF8091C9008F7E8093C90080915D
:10E0A000C9008E7F8093C90080911108882311F4E4
:10E0B0008EEF01C08EE78093CE008091FA038093AB
:10E0C000D2011092FA0308951F920F920FB60F9289
:10E0D00011248F939F93EF93FF939091D1019923F4
:10E0E00009F040C080910304882361F480911108F5
:10E0F000882311F483E003C0813999F481E080938F
:10E1000003040FC0833099F480911108882349F0EB
:10E11000909311088091C9008E7F8093C9008EEF83
:10E120001EC08091C90081608093C9000EC08332F7
:10E1300061F48091C9008E7F8093C9008FEF809336
:10E14000CE0081E08093D10114C080910304E82FB8
:10E15000FF27EF5EF74F8F5F8093030480818093EA
:10E16000CE0007C0109203048091C90080618093A3
:10E17000C900FF91EF919F918F910F900FBE0F906B
:10E180001F901895EF92FF920F931F93CF93DF93F9
:10E190007C018B01EA01452B39F0F80181918F0157
:10E1A000F70109952197C9F7E6E0CDB7DEB70C94E2
:10E1B0005377EF92FF920F931F93CF93DF937C01DE
:10E1C0008B01EA01452B41F0F8010F5F1F4F84914D
:10E1D000F70109952197C1F7E6E0CDB7DEB70C94BA
:10E1E00053770F931F93CF938C01C62F161634F4D9
:10E1F00080E2F8010995C1501C16D4F3CF911F910C
:10E200000F9108950F931F93CF938C01C62F16166D
:10E2100034F480E3F8010995C1501C16D4F3CF9172
:10E220001F910F910895A5E3B0E0E9E1F1E70C94A7
:10E230002B772E96EEADFFAD2E97882499245401AE
:10E240008091F903882321F42C961FAE1EAE2C97E3
:10E250005EE4452E512C4C0E5D1E6F01B60105C0CB
:10E26000153239F00894C11CD11CF6011491112308
:10E27000B9F7A601461B570B31F02C968EAD9FAD1A
:10E280002C970E94D970112309F46AC20894C11C0A
:10E29000D11CFF24FDA6FCA64FEFE42EF9A6F60143
:10E2A0000894C11CD11C1491153721F0812F806274
:10E2B0008837B1F4F0FE0AC0F20124E030E0420EEB
:10E2C000531E80809180A280B3800AC0F20142E098
:10E2D00050E0440E551E808191814C01AA24BB243C
:10E2E000103221F489A58823D1F61DC0133219F408
:10E2F00058E0F52AD4CF1A3211F01D3291F41A32B7
:10E3000059F4F20182E090E0480E591EE081ECA73A
:10E31000EE232CF6E195ECA790E1F92AAFEDFA2275
:10E32000BECF1B3211F419A7BACF1E32C1F5F601C8
:10E330000894C11CD11C14911A3279F4F20122E024
:10E3400030E0420E531E408151813FEF4F3F530753
:10E3500014F44FEF5FEFE42EA2CF40E050E0812FA6
:10E3600080538A30A0F4CA0133E0880F991F3A9590
:10E37000E1F7840F951F480F591F410F511D40535E
:10E380005040F6010894C11CD11C1491E8CF8FEFC6
:10E390004F3F580714F44FEF5FEFE42E85CF103353
:10E3A00029F4F4FC7CCF90E2F92A79CF812F8153B4
:10E3B0008930D8F440E050E0CA0123E0880F991F6B
:10E3C0002A95E1F7840F951F480F591F410F511DE2
:10E3D00040535040F6010894C11CD11C1491812F68
:10E3E00080538A3048F34CA75FCF183619F4A4E065
:10E3F000FA2A55CF1C3619F4B1E0FB2A50CF133658
:10E4000061F43E010894611C711CF20122E030E0CD
:10E41000420E531E808189833CC1143421F014368E
:10E4200011F0193651F5143411F431E0F32AF0FEED
:10E430000AC0F20144E050E0440E551E80809180F5
:10E44000A280B3800CC0F20182E090E0480E591E19
:10E45000808191814C01AA2497FCA094BA2CB7FE2C
:10E460000AC0B094A09490948094811C911CA11C2B
:10E47000B11C8DE289A70AE06FC01F3411F01F366E
:10E4800031F41F3411F491E0F92A08E064C0103728
:10E4900079F4F201A2E0B0E04A0E5B1E8081918126
:10E4A0004C01AA24BB2400E1B0E4FB2A18E753C0C6
:10E4B0001337C1F5F20122E030E0420E531E6080B6
:10E4C00071806114710489F43E010894611C711C0F
:10E4D00088E289838EE6F301818385E78B838CE66E
:10E4E0008C838D8389E28E831F82E7FC13C08E2D7F
:10E4F000992787FD9095AC0160E070E0C3010E9410
:10E50000B575009729F0382E3618E3140CF0C3C007
:10E510003E2CC1C0F30101900020E9F731973E2E57
:10E520003618B9C0153511F0153731F4153511F419
:10E53000F1E0FF2A0AE00FC0183519F0183709F08A
:10E54000A0C000E1F3FE07C081149104A104B1044E
:10E5500011F020E4F22A19A6EDA6E7FC02C03FED77
:10E56000F32289E2682E712C6C0E7D1E81149104B9
:10E57000A104B10421F44DA5442309F47BC0802FEC
:10E580009927AA27BB278EA79FA7A8ABB9AB202E98
:10E59000332490E0891690E0990691E0A90690E076
:10E5A000B90648F0C501B4012EA53FA548A959A94F
:10E5B0000E94EE7617C0AFEF8A169104A104B10451
:10E5C00049F040F0C401B1010E94C7769B01442785
:10E5D000552708C0882D602F0E94BB76282F33272F
:10E5E000442755272AAB3BAB4CAB5DAB0A3059F403
:10E5F0008AA9880F880F880F9AA9990F890F382D3B
:10E60000381B832F10C0003139F48AA98295807F8E
:10E61000482D481B842F07C08AA9880F880F880FB0
:10E62000582D581B852F90E02EA53FA548A959A924
:10E6300082169306A406B50608F091E08AA89BA866
:10E64000ACA8BDA88A3010F4805D04C0895A183582
:10E6500009F48F7DD3018E933D01992309F099CF61
:10E66000083041F4F3FE06C0803321F080E3FD0161
:10E6700082933F01CE010196382E3618F8E23F0E04
:10E680000BC0112309F46CC03E010894611C711C7D
:10E690001983B1E03B2E19A6032D2DA4231827FCC6
:10E6A000222489A5882311F00F5F02C0F6FC0E5FBB
:10E6B000020DEF2CFF24C70180739070892B49F461
:10E6C0008CA5801B682F2C968EAD9FAD2C970E9439
:10E6D000F17089A5882331F041E050E0BE01675D0B
:10E6E0007F4F0AC0E6FE0EC080E38AA71BA742E068
:10E6F00050E0BE01665D7F4F2C968EAD9FAD2C978E
:10E700000E94C270C70180739070809749F48CA5F5
:10E71000801B682F2C968EAD9FAD2C970E940271A6
:10E72000622D2C968EAD9FAD2C970E940271832D89
:10E73000992787FD9095AC01B3012C968EAD9FADC6
:10E740002C970E94C270E4FE89CD2CA5201B2CA71B
:10E75000622F2C968EAD9FAD2C970E94F1707ECDCE
:10E76000E2E1CB5C0C9447772FB740E0F894E0E00F
:10E77000F0E081E2809357009491E2E0F0E0809332
:10E7800057003491E4E0F0E08093570084912FBF6C
:10E790009E3199F4363941F4893011F441E00DC0CD
:10E7A0008A3059F442E009C0373939F4863011F41F
:10E7B00043E003C0853009F444E0842F992708958D
:10E7C0009FB7F8948091C900877F8093C90080919A
:10E7D000C9008F7E8093C9008091C9008F77809394
:10E7E000C9008091C9008F7B8093C9008091C900C6
:10E7F0008F7D8093C90052985A9A53985B9A9FBF15
:10E800000895CF93DF938091F903882309F497C08B
:10E810009091ED068091D301981709F490C08091F2
:10E82000F803882321F40E94B4738093F80389E3EA
:10E830009DE09F938F93C1E2D4E1DF93CF93E0916A
:10E840000404F091050409950F900F900F900F901C
:10E850008091ED0699278230910501F18330910571
:10E860002CF4009761F0019769F024C08430910581
:10E87000D9F084309105ACF00597C9F01BC089E24E
:10E880009DE002C087E19DE09F938F93DF93CF933C
:10E89000E0910404F0910504099519C08EEF9CE005
:10E8A000F3CF8BED9CE0F0CF8DEC9CE0EDCF85ECD1
:10E8B0009CE0EACF86E49DE09F938F93DF93CF9314
:10E8C000E0910404F091050409951092ED060F9073
:10E8D0000F900F900F908091F803843011F08230E8
:10E8E000A9F40E94E0739091ED06892F8150833046
:10E8F00018F40E9439671FC0943019F40E94AC6F5D
:10E900001AC09530C1F40E94E36D15C08091ED06E8
:10E91000882389F08CE59DE09F938F9381E294E1B9
:10E920009F938F93E0910404F091050409950F9053
:10E930000F900F900F908091ED068093D301DF919F
:10E94000CF9108950F931F9381E08093F903409135
:10E95000D001E5E7FCE020E030E05FE48491992716
:10E960002F5F3F4F829FB001839F700D929F700D6C
:10E97000112446275150319657FFF0CF4093D001D4
:10E98000EDE4FCE020E030E057E2849199272F5F2E
:10E990003F4F829FB001839F700D929F700D112495
:10E9A00046275150319657FFF0CF4093D0018091C8
:10E9B000F803882321F40E94B4738093F8038091B4
:10E9C000D001833459F088E190E029E20FB6F89441
:10E9D000A895809360000FBE2093600083E191E7CB
:10E9E000909305048093040487E79DE09F938F93A1
:10E9F00001E214E11F930F93E0910404F0910504E8
:10EA000009950F900F900F900F9086E690E09F93DE
:10EA10008F938EE490E09F938F931F921F9280912B
:10EA200002016AE00E94BB76892F99279F938F93FA
:10EA3000809102010E94BB7699279F938F938DE965
:10EA40009DE09F938F931F930F93E0910404F091A7
:10EA50000504099585E79CE09F938F931F930F937F
:10EA6000E0910404F091050409958DE49CE09F93E6
:10EA70008F931F930F93E0910404F091050409957F
:10EA80008DB79EB746968DBF81ED9DE09F938F9386
:10EA90001F930F93E0910404F0910504099583EC12
:10EAA0008093810080916F00806280936F000F904F
:10EAB0000F900F900F901F910F9108958091F9037F
:10EAC000882361F08091ED06843011F40E941D705E
:10EAD0008091D001833411F01092F90308951F92B0
:10EAE0000F920FB60F9211242F933F934F935F9382
:10EAF0006F937F938F939F93AF93BF93EF93FF9306
:10EB00002091CE009091ED06892F8150833020F422
:10EB1000822F0E944B680BC0943021F4822F0E94F8
:10EB2000107005C0953019F4822F0E944F6FFF912D
:10EB3000EF91BF91AF919F918F917F916F915F9175
:10EB40004F913F912F910F900FBE0F901F901895EE
:10EB5000FB01DC0140FF05C002C005900D9205904D
:10EB60000D9242505040C8F70895FC01415050406A
:10EB700030F001900616D1F73197CF01089588271C
:10EB8000992708955058192EA6D001D08CC0BA17D5
:10EB90006207730784079507B1F188F40EF41094A7
:10EBA0000B2EBA2FA02D062E622F202D072E732F8D
:10EBB000302D082E842F402D092E952F502DFF2704
:10EBC0005523B9F0591B49F0573E98F046953795B3
:10EBD0002795A795F0405395C9F776F0BA0F621FB5
:10EBE000731F841F30F4879577956795B795F0402C
:10EBF000939517FA0F2E0895BF1BBB27BA0B620B14
:10EC0000730B840BF6CFDEF692C097FB70D09F3764
:10EC100038F0FEE9F91B982F872F762F6B2F05C050
:10EC200083C09695879577956795F150D0F73EF418
:10EC300090958095709561957F4F8F4F9F4F089568
:10EC4000E89403C097FB0EF4F3DFB62F672F782FFD
:10EC5000892F9EE9002427C00ED05EF004C00BD09F
:10EC600026F001C008D019F020F48FEF089580E05D
:10EC7000089581E0089597FB092E052600F8689411
:10EC80002DD0E89407FC07C0621773078407950727
:10EC900021F008F400940794989408959A95BB0F76
:10ECA000661F771F881F11249923A1F08823B2F7CC
:10ECB0009F3F59F0BB0F48F421F4002011F460FF8E
:10ECC00004C06F5F7F4F8F4F9F4F881F9795879529
:10ECD00097F9089529C0052E092607FA440F551FF4
:10ECE0005F3F79F0AA27A51708F051E04795880FF4
:10ECF000991F9F3F31F0BB27B91708F091E0879526
:10ED000008959F919F91112414C097FB880F991F1C
:10ED10009F3F31F0BB27B91708F091E08795089520
:10ED20009F919F91112405C06627772788279927EF
:10ED300008959FEF80EC0895629FD001739FF001CA
:10ED4000829FE00DF11D649FE00DF11D929FF00D7B
:10ED5000839FF00D749FF00D659FF00D9927729FB2
:10ED6000B00DE11DF91F639FB00DE11DF91FBD013D
:10ED7000CF0111240895991B79E004C0991F9617BB
:10ED800008F0961B881F7A95C9F780950895AA1BED
:10ED9000BB1B51E107C0AA1FBB1FA617B70710F086
:10EDA000A61BB70B881F991F5A95A9F780959095B8
:10EDB000BC01CD01089597FB092E07260AD077FDE7
:10EDC00004D0E5DF06D000201AF4709561957F4FDE
:10EDD0000895F6F7909581959F4F0895A1E21A2E18
:10EDE000AA1BBB1BFD010DC0AA1FBB1FEE1FFF1FEF
:10EDF000A217B307E407F50720F0A21BB30BE40B3F
:10EE0000F50B661F771F881F991F1A9469F7609585
:10EE10007095809590959B01AC01BD01CF0108953F
:10EE200097FB092E05260ED057FD04D0D7DF0AD058
:10EE3000001C38F450954095309521953F4F4F4F29
:10EE40005F4F0895F6F790958095709561957F4F87
:10EE50008F4F9F4F08952F923F924F925F926F92E4
:10EE60007F928F929F92AF92BF92CF92DF92EF925A
:10EE7000FF920F931F93CF93DF93CDB7DEB7CA1BDB
:10EE8000DB0B0FB6F894DEBF0FBECDBF09942A8806
:10EE9000398848885F846E847D848C849B84AA84AE
:10EEA000B984C884DF80EE80FD800C811B81AA813B
:10EEB000B981CE0FD11D0FB6F894DEBF0FBECDBF06
:10EEC000ED010895EE0FFF1F0590F491E02D0994D8
:10EED000F999FECFB2BDA1BDF89A119600B408957C
:10EEE000F7DF01921A94E1F70895F999FECFB2BDC8
:10EEF000A1BD00BC11960FB6F894FA9AF99A0FBE0C
:0CEF000008950190F2DF1A94E1F70895E3
:10EF0C005E010A0151756164726F00000164FF01BA
:10EF1C00FFFF01FC01FC0101737373FF03007D0013
:10EF2C0000C409C40964001048616C6C6F205765FB
:10EF3C006C740000000000000000000000000000E5
:10EF4C0000000000000000000000000000000000B5
:10EF5C0000000000000000000000000000000000A5
:10EF6C000000000000000000000000000000000095
:10EF7C0000000000000000000101000300200B0550
:10EF8C000000ECFF6440415A4664640A029696966F
:10EF9C00960840403A10FB30380190D0030090D0D6
:10EFAC000300F401640053706F727400004E6F72B2
:10EFBC006D616C0000426567696E6E657200007869
:10EFCC0000FF03640B0A0D0B0C0E0B0F100101015B
:04EFDC0070010FFFB2
:00000001FF
